:020000040000FA
:10000000E80E0020D5000000DD000000DF00000049
:1000100000000000000000000000000000000000E0
:10002000000000000000000000000000E1000000EF
:100030000000000000000000E3000000E5000000F8
:10004000519D00000BC20000C5A10000D7A1000017
:1000500081A10000A3A1000075AA00005DAB000013
:100060000FBC000067BC0000C1BC00001BBD00004D
:1000700035C3000055C30000E7000000E7000000A2
:10008000E7000000E7000000E7000000E7000000D4
:10009000E70000000000000000000000E700000092
:1000A000E7000000E7000000E7000000E7000000B4
:1000B000D19E0000ABA9000000000000C9B4000000
:1000C000034885460CF070FC00480047E91B00001F
:1000D000E80E00200448804704480047FEE7FEE79A
:1000E000FEE7FEE7FEE7FEE75D010000C10000005D
:1000F00070B51B4D28694007400F052800D9042022
:10010000022803D017498000085817E0286A000425
:10011000840F012C00D9641E286A000301D51248FF
:1001200000E01248296AC905C90D891C4843296A9B
:100130008904C90E891C0CF0E9FBE040A969090794
:10014000090F491C0CF0E2FB064C083C20600849F2
:100150004A1080180CF0DAFB606070BD7047000038
:10016000000200500800002000805101001BB70071
:1001700040420F00FFB581B005460E461746164CAB
:100180000120A840C0B20AF0EAFB01200AF0FAFB05
:1001900000200AF0EBFB0AF034FC01E0641E15D3EA
:1001A0000AF03BFC0028F9D0E8B20AF03EFC0499C2
:1001B00088420ED90A99002906D031683A68891A0E
:1001C000081830600009386005B0F0BD0020C04359
:1001D000FAE70020C043F7E7F401000038B56B4CA4
:1001E00059202060162020608820206017200AF007
:1001F000E7F818200AF0E4F819200AF0E1F81B20CB
:100200000AF0DEF81C200AF0DBF81D200AF0D8F80E
:100210001020002200900223012110460AF03CFB2E
:100220000020206038BD38B50120594A00900023D5
:10023000111F0520FFF79EFF411C08D0554C206080
:10024000554948437D21C9000CF060FB606038BD12
:1002500038B54F4A0120083200900023111F0620B4
:10026000FFF788FF411C09D04A4CA0604A492C3155
:1002700048437D21C9000CF049FBE06038BD38B52A
:10028000434A0120103200900023111F0420FFF781
:1002900071FF411C09D03F4C20613F492C3148433C
:1002A0007D21C9000CF032FB606138BD38B5384A99
:1002B0000120183200900023111F0220FFF75AFF7F
:1002C000411C09D0334CA06133492C3148437D2176
:1002D000C9000CF01BFBE06138BD38B52C4A012089
:1002E000002320320090111F1846FFF743FF411CE6
:1002F00008D0284C2062294948437D21C9000CF0D0
:1003000005FB606238BD38B5214A01202832002340
:10031000111F0090FFF72EFF411C08D01D4CA0625A
:100320001E4948437D21C9000CF0F0FAE06238BD57
:1003300070B5174C083C2078411C2170002806D06D
:10034000012807D00025022807D0257070BDFFF7CF
:100350006AFF70BDFFF793FF70BDFFF7D4FF2570F4
:1003600070BD70B50A4C083C6078411C6170002873
:1003700004D00025012804D0657070BDFFF768FF28
:1003800070BDFFF7AAFF657070BD0000000100504E
:1003900028000020280300204C090000250300004D
:1003A000FB48C0687047FA4880687047F848406862
:1003B0007047F749C8607047F54988607047F4494D
:1003C0004860704770B50446F14D226800212869E5
:1003D00013000CF026FB08F205333D95F1F0EF32E7
:1003E000242001F0B9FC002827D12420616801F005
:1003F000AFFC0CF0A1FAFC210CF088FA08460321AE
:100400000CF084FA29788142F3D02870E04A143243
:1004100041004318D05C64214843000AFFF7CFFF36
:100420009A18507864214843000AFFF7C5FF907876
:1004300064214843000AFFF7BCFFF1E16069FFF760
:10044000BEFFA069FFF7B8FFE069FFF7B2FFE7E181
:1004500000280AD001281DD0022836D0E0680128E3
:10046000EBD9401EE0602961DAE10020FFF7A7FF29
:100470000020FFF7A1FF0020FFF79BFF2420616809
:1004800001F066FC2520A16801F062FC2869401C8F
:100490002861C5E1242001F05FFC002809D06069D3
:1004A000FFF78DFFA069FFF787FFE069FFF781FF86
:1004B000B6E12420616801F04BFC2520A16801F021
:1004C00047FC2869401C2861AAE1252001F044FC72
:1004D000002809D00020FFF772FF0020FFF76CFF13
:1004E0000020FFF766FF9BE12420616801F030FCEB
:1004F0002520A16801F02CFC2869401C28618FE1AF
:1005000003000CF08EFA0504112B456370000020E7
:10051000FFF755FF0020FFF74FFF0020FFF749FFCF
:100520002869401C28617BE1242001F015FC00288B
:100530000CD00020FFF743FF0020FFF73DFF002015
:10054000FFF737FF6320FFF73AFF69E12420616876
:1005500001F0FEFB2869401C286161E1242001F0C4
:10056000FBFB00280CD00020FFF729FF0020FFF73D
:1005700023FF0020FFF71DFF6320FFF71DFF4FE162
:100580002420616801F0E4FB2869401C286147E1F0
:10059000242001F0E1FB002810D00020FFF70FFF1E
:1005A0000020FFF709FF0020FFF703FF6320FFF79C
:1005B00000FF35E150E01DE080E026E12420616885
:1005C00001F0C6FB2869401C286129E10020FFF7E3
:1005D000F6FE0020FFF7F0FE0020FFF7EAFE286994
:1005E000401C28611CE1E068012888D9401EE060B9
:1005F000296115E1002806D0E068012893D9401E42
:10060000E06029610CE1242001F0A6FB00288AD1DA
:10061000206963281CD22420616801F099FB2569B8
:100620006D1C25616069642168430CF06FF9FFF768
:10063000C6FEA069642168430CF068F9FFF7BCFEB0
:10064000E069642168430CF061F9FFF7B2FEE7E06E
:100650002869401C2861E3E0002806D0E0680128F2
:100660008DD9401EE0602961DAE0242001F074FB9E
:10067000002884D1206900281CD02420616801F062
:1006800067FB25696D1E25616069642168430CF074
:100690003DF9FFF794FEA069642168430CF036F938
:1006A000FFF78AFEE069642168430CF02FF9FFF739
:1006B00080FEB5E02869401C2861B1E06322030098
:1006C0000CF0AFF906042038516B849C2069632834
:1006D00014D2242001F040FB00280ED124206168B0
:1006E00001F036FB2069401C2061FFF768FE002006
:1006F000FFF762FE6320FFF75CFE91E022610120BC
:1007000028618DE02069002811D0242001F024FB0D
:1007100000280BD12420616801F01AFB6320FFF749
:100720004EFE2069401E2061FFF743FE78E0022064
:10073000286175E02069632811D2242001F00CFBA8
:1007400000286DD12420616801F002FB6320FFF7CF
:1007500036FE2069401C2061FFF72EFE60E022611A
:10076000032028615CE02069002813D0242001F0D8
:10077000F3FA002854D12420616801F0E9FA2069D5
:10078000401E2061FFF71BFE6320FFF715FE47E0C8
:10079000540000200420286142E02069632811D21F
:1007A000242001F0D9FA00283AD12420616801F010
:1007B000CFFA6320FFF700FE2069401C2061FFF79D
:1007C000F8FD2DE022610520286129E0206900283C
:1007D00011D0242001F0C0FA002821D12420616822
:1007E00001F0B6FA2069401E2061FFF7E5FD6320A5
:1007F000FFF7DFFD14E00620286111E0E068012822
:100800000ED9401EE06029610AE0216129610020C3
:10081000FFF7D5FD0020FFF7CFFD0020FFF7C9FD52
:1008200002F09FF8012809D0002001F0D2FB00203F
:1008300001F008FC002001F03DFC70BDFFF7B6FDA3
:1008400001F0C7FBFFF7AFFD01F0FCFBFFF7A8FDD0
:1008500001F030FC70BD0149086170475400002070
:1008600010B5002001F0B5FB002001F0EBFB0020EB
:1008700001F020FC10BD10B5874C0422226061609D
:10088000A160E06063206061A061E061242001F06C
:100890005FFA2520A16801F05BFA0020FFF7DBFF7B
:1008A0002046FFF78FFD10BD10B57B4905220A6079
:1008B000486088607948C8600021242001F048FA27
:1008C0000021252001F044FA0020FFF7C4FF724800
:1008D000FFF778FD10BD10B56F4901220A6048602E
:1008E00088606E48C8600021242001F031FA0021A0
:1008F000252001F02DFA0020FFF7ADFF6648FFF735
:1009000061FD10BD70B5644C062525606360A36071
:100910000125E56064256843000A60616420414365
:10092000080AA06164204243100AE06119462420AD
:1009300001F00EFA2520A16801F00AFA0020FFF765
:100940008AFF2046FFF73EFD70BD002806D05449BF
:10095000012810D0022813D1C868A5E750484038B4
:10096000C16B4A008B18816B5B1CCAB2416B006B78
:10097000C9B2C0B2C6E788687821401C4843AAE7DC
:10098000704710B5444C002020606061A061E061B8
:100990002420616801F0DCF92520A16801F0D8F974
:1009A0000020FFF758FF2046FFF70CFD10BD70B583
:1009B0000D46394C0721216059086160A16001236F
:1009C000E36064235843000A606164204543280AB9
:1009D000A06164204243100AE061242001F0B8F9CC
:1009E0002520A16801F0B4F90020FFF734FF20466C
:1009F000FFF7E8FC70BD002804D0012801D00228D0
:100A00000BD1BEE726484038816BC36BCAB2416B3D
:100A1000006BDB1CC9B2C0B2C9E7704710B51E4CF1
:100A2000022323600123E36064235843000A6061CA
:100A300064204143080AA06164204243100AE06137
:100A40002420616801F084F92520A16801F080F973
:100A50000020FFF700FF2046FFF7B4FC10BD10B5E3
:100A60000D4C03202060FA216160A1600F20E0603E
:100A7000632060610020A061E061242001F068F93A
:100A80002520A16801F064F90020FFF7E4FE20466C
:100A9000FFF798FC10BD000058030020102700004D
:100AA000FC0B002070B5054600240821002009F049
:100AB000E0FB280604D50B21002009F0BFFB03E072
:100AC0000B21002009F0D5FB0A21002009F0B6FB1C
:100AD000012001F067FB0A21002009F0CAFB012078
:100AE00001F060FB6806050E641C082CE1D30821A8
:100AF000002009F0A3FB70BD10B5044604210120BD
:100B000009F0B7FBE0B2FFF7CDFF10BD10B504460A
:100B10000421012009F092FBE0B2FFF7C3FF10BDF2
:100B200010B50C46B030FFF7E7FF20091230FFF791
:100B3000E3FF2007000FFFF7DFFF10BDF7B50E46FC
:100B4000002500F0D4F9002801D0771C10E0022025
:100B5000FEBD30460099FFF7E3FF002428460299C6
:100B60006D1C085CFFF7D2FF641C052CF6D3761CC5
:100B7000BE42EED30020FEBDF7B50E46002500F0C4
:100B8000B6F9002801D0B71C10E00220FEBD3046A7
:100B90000099FFF7C5FF0024284602996D1C085CE8
:100BA000FFF7B4FF641C052CF6D3761CBE42EED3CF
:100BB0000020FEBDF7B50E46002500F098F900288C
:100BC00001D0B71C10E00220FEBD30460099FFF7AF
:100BD000A7FF0024284602996D1C085CFFF796FFCA
:100BE000641C0A2CF6D3761CBE42EED30020FEBD58
:100BF000F7B50E46002500F07AF9002801D0F71C61
:100C000010E00220FEBD30460099FFF789FF002466
:100C1000284602996D1C085CFFF778FF641C0E2CB7
:100C2000F6D3761CBE42EED30020FEBDFFB581B0E8
:100C30000F461646002500F05AF9002812D102206E
:100C400005B0F0BD30460199FFF76AFF019C06E050
:100C500028460A996D1C085CFFF758FF641CBC42CB
:100C6000F6D3761C04988642ECD30020E8E7FFB563
:100C700081B00646174600240091002500F037F9A0
:100C8000002807D00498002813D0012822D0052876
:100C900034D130E00220D3E7385D2038810041189C
:100CA00017480A1830460099FFF748FFF61D6D1CDB
:100CB000641C785D0A28EFD120E0385D0A212038D5
:100CC00048431049421830460099FFF755FFF61D7A
:100CD0006D1C641C785D0A28EFD10FE0385D14218B
:100CE000203848430849421830460099FFF762FF10
:100CF0000A366D1C641C785D0A28EFD100209FE73E
:100D00000EE2000035E3000083E5000010B5002886
:100D10000ED001280BD1A120FFF7EEFEA820FFF78F
:100D2000EBFE2F20FFF7E8FEC820FFF7E5FE10BD21
:100D3000A020FFF7E1FEA820FFF7DEFE2F20FFF73F
:100D4000DBFEC020FFF7D8FE10BD10B5AE20FFF7C8
:100D5000D3FE0020FFF7D0FE1020FFF7CDFE40208D
:100D6000FFF7CAFEB020FFF7C7FE8120FFF7C4FEE1
:100D70008020FFF7C1FEA020FFF7BEFEA620FFF7F0
:100D8000BBFEA820FFF7B8FE2F20FFF7B5FEC0205E
:100D9000FFF7B2FED320FFF7AFFE0020FFF7ACFE57
:100DA000D520FFF7A9FE8020FFF7A6FED920FFF788
:100DB000A3FE2220FFF7A0FEDA20FFF79DFE1220FF
:100DC000FFF79AFEDB20FFF797FE3020FFF794FE37
:100DD0008D20FFF791FE9520FFF78EFEAF20FFF7E5
:100DE0008BFE10BD10B503242402204601F0DAF971
:100DF0000521012009F03DFA204601F0D3F9052133
:100E0000012009F01BFA204601F0CCF910BD10B505
:100E100001220521104609F0E7F901220A210020EC
:100E200009F0E2F901220B21002009F0DDF901228D
:100E30000821002009F0D8F901220421104609F008
:100E4000D3F9FFF7CFFFFFF780FF2A488069C0B2D0
:100E5000FFF75CFF10BD70B500252846B030FFF7E6
:100E60004BFE1220FFF748FE0020FFF745FE00244E
:100E70000020FFF74BFE641C402CF9D36D1C062D9F
:100E8000EBD370BDFFB581B007460E4615460CE0AA
:100E900039462846FFF744FE3C4603E00020FFF7B2
:100EA00035FE641CB442F9D36D1C04988542EFD31F
:100EB00005B0F0BD10B5044607F0BFFF60436421E4
:100EC0000BF024FDC4B2642C00D964241E2C00D283
:100ED0001E248120FFF710FE2046FFF70DFE10BDF7
:100EE00010B5FFF709FE10BD0349087070470248AE
:100EF000007870473C0B0020640100203EB5134C85
:100F00005920206016202060882020602A2009F0C7
:100F100057FA0F48009003206946087100254D716B
:100F20008D71CD7100200BF07BFA0A4A012100205F
:100F30000BF07EFB03220021022009F055F900216D
:100F4000022009F07BF925603EBD00000001005041
:100F500000C20100590F000010B51422FF49002003
:100F60000BF0D1FB10BDFE4908707047FC490871B9
:100F70007047FB480078704710B5FFF7FAFF00286C
:100F800005D001280ED00020FFF7EDFF10BD002195
:100F9000022009F053F90020FFF7E8FFF149002093
:100FA000486010BD0021022009F063F910BDEC4932
:100FB00088707047F8B50024EB4EE94F3546FF3591
:100FC000F1354D206102800209188022E64801F0C7
:100FD0001EF9FE60F868C17B962907D0A84207D3A6
:100FE000FE60641C5A2CECD30020F8BD0120F8BD33
:100FF0001030F860EEE7F0B58FB000200222DB4B36
:10100000D64919600E91097800297ED00B020E99FD
:10101000D24C4978257A0B43A178E4780D942402C8
:101020000C430C94AC467D24E400CE4D4C43D04F91
:1010300080350B942C46DE1B4034BB4266D028DC46
:10104000CC4FDE1BBB427ED012DCCB4A981A9342B7
:101050007AD008DCC948181877D0C94A80182CD033
:10106000012831D131E0052870D00628F9D136E1C8
:10107000BA4B0C2E9B7B6AD006DC012E68D0072E63
:1010800067D00B2EEDD14DE10D2E7DD00E2EE8D187
:10109000B8E1B24A3300177B12790BF0C2FC1A1583
:1010A000F1151515151515F0EFEEEDECEBEAE9E885
:1010B000E7151515151515E6E515FF29D1D10322FC
:1010C000B04900200BF055FB28E26046FF28FBD119
:1010D000A3480022427182710120FFF747FFA34815
:1010E0009F4E0368303698783070D97871700A91C5
:1010F0001979B1708E465979F1708C4699793171B0
:10110000DB79737101266F4601E00BE281E13E71EC
:101110007A7102930391614604910592714606919A
:101120000A99079198494018089008AF3A7101A9A7
:1011300000200AF0DBFB002804D0032293490020A2
:101140000BF017FB06E0D1E06BE0E2E170E03EE17E
:10115000CEE0DEE08E49E0690870206A48708D4F6D
:10116000AB213868017013214170FF2181730C227B
:10117000874989480BF0F2FB87490F22891E00201E
:101180000BF0F7FA032000E032E101F013F86421DC
:10119000686A0BF0BBFB7E4E0C3E30707F4800212E
:1011A000406A08F02DFD70702068B070286BF070F8
:1011B000686B3071A86B70717949E86A0BF0A6FB17
:1011C000B0717D25ED002946606A0BF09FFBF07140
:1011D0002946A0690BF09AFB3072A0207072C820DB
:1011E000B0720020F0723968AB200870FFF7E2FEA1
:1011F000002803D039680C20487002E038680B21C1
:1012000041703968FF20887361490C220C396248AB
:101210000BF0A4FB60490F22891E00200BF0A9FAF5
:101220007CE1FF29FCD11920E96A00F091FD75E10C
:101230004A48C079FF28F3D14A4901204860C86074
:101240004A4E0C9807F003FE306842790179120289
:1012500011430A2251438079286000282AD00128AE
:101260000FD0022826D11AE04CE144E13BE133E102
:101270002BE123E115E10CE102E1FBE0F8E0E1E024
:10128000CAE021637D2292014648914200D9206341
:101290007D22216B520191420CD220630AE06163EE
:1012A000414A4248914200D960634149626B8A4297
:1012B00000D2606303F0F2FEFFF7CDFD00211120A4
:1012C00000F046FD0021122000F042FD0021132015
:1012D00000F03EFD0021142000F03AFD1EE10D98C3
:1012E000FF289DD1216003F0D9FE17E1FF2915E108
:1012F0000D98FF2894D10B98A0612E4A2E49904258
:1013000000D9A161A069884200D2A16103F0C6FEA4
:1013100004E10D98FF2804D121484143E96203F01C
:10132000BDFEFBE0FF2B51D10E4B01215960002186
:10133000D960174B203311460E9C521C615C195426
:10134000401C0C28F7D3FFF786FD0021112000F088
:10135000FFFC0021122000F0FBFC2FE078030020AE
:10136000700100203C0B0020A00300206801002039
:1013700018AA000009AA000002AA0000FF77FFFFD8
:1013800001DEFFFFC7EB0000D0070000C4EB000048
:10139000BC0700206C0100208E03002028030020E1
:1013A00060EA0000701700007C150000AC0D000022
:1013B000DC050000400D0300007102000021132035
:1013C00000F0C6FC0021142000F0C2FCA6E0FF2BB8
:1013D0000DD1F94901234B600023CB60F74B114637
:1013E0000E9C521C615C1954401C0C28F7D395E0EC
:1013F0006046FF2805D1F249012048718871FFF746
:10140000D6FD8BE06046FF2802D1ED4901208871AE
:1014100084E06046FF2881E0FF2F7FD1E64C012366
:10142000A360E64B163B19700D99597005219A700F
:101430000A460E9C491CA25C1C18E270401C07283E
:10144000F6D36BE0FF2F69D1DB4C0123A360DB4BAC
:10145000203B19700D99597005219A700A460E9C0F
:10146000491CA25C1C18E270401C0728F6D355E00A
:10147000FF2953E0FF2A51D10C9804F048FF4DE0BA
:10148000FF294BD10020FFF771FDCB4900204860B8
:1014900044E00D98FF2841D10B98606203F0FEFDF7
:1014A0003CE0C8484079FF2838D129630D9868632B
:1014B000AA630020606003F0F1FD2FE00D98FF2883
:1014C0002CD1616003F0EAFD28E0FF2926D101203C
:1014D000E06103F0E3FD21E0FF291FD10020E0617E
:1014E00003F0DCFD1AE00D98FF2817D1B248016126
:1014F00003F0D4FD12E0FF2910D10120206203F097
:10150000CDFD0BE0FF2909D10020206203F0C6FDCC
:1015100004E0FF2902D10020FFF728FD1421A9488B
:101520000BF035FA00200FB0F0BDA5488078704769
:10153000F8B501F07DF905284DD0FFF7F6FF4D25F0
:10154000AD02A14E9E4C002810D00020FFF72FFDC9
:101550009A48012149020C300BF019FAA069802247
:1015600040024119304600F052FE266160790028A1
:1015700061D0A0790027002853D0A77193491A2081
:1015800000F0E6FB00F0F8FD2169C87B962825D025
:101590008A485838814241D32661606900280CD0BE
:1015A000A06904214002401900F052FEA069802287
:1015B00040024119844800F009FEA069401CA06166
:1015C0005A2822D3A76167710322814900200BF0BA
:1015D000D0F80020F8BD0020C043F8BD2069C773D3
:1015E000012060617B48AB220068027008224270D3
:1015F000FF2242740F2278480BF0B0F9764912228C
:10160000891E00200BF0B5F815E040024119802238
:101610006D4800F0FCFD26616761B3E71031216180
:10162000B0E71A2000F098FB002804D1677103226C
:101630006A490BF09EF80020F8BD61484079704778
:101640005F4800797047F0B589B0074601F085F929
:101650000024E443012806D003F09EF8002804D0BB
:10166000204609B0F0BD2046FBE7FFF7E9FF002860
:1016700003D0FFF7E2FF002845D04F4E504C3046D4
:10168000F1688030012940D081690A0AA16A0A7094
:1016900082694A70F16AA56A090AA970F16AE9705B
:1016A000406A64210BF032F928710E2000F054FBDF
:1016B0004B497D25081AED0029460BF027F9A16A50
:1016C000487148480021406A08F09AFAA16A887176
:1016D000694600200AF015F80798D021411AA06A3F
:1016E000C17106990172059941720399817202993B
:1016F000C172019901739621C173F06F00280BD05C
:10170000012821D029E02046ABE7C1690A0AA16A75
:101710000A70C2694A70BDE701F01CF9E121C900F5
:10172000484329460BF0F2F8A16A2030487301F0D3
:1017300011F9E121C900484329460BF0E7F82030B0
:10174000A16A000A887308E001F004F9A16A4873ED
:1017500001F000F9A16A000A88734D25AD02002F3F
:1017600002D0012F52D144E01022A16AA0680BF0F0
:10177000F5F81D49A068884238D310480C30A060A5
:10178000E06A04214002401900F062FDE06A802214
:101790004002411909480C3000F018FD07480121AA
:1017A00049020C300BF0F3F8E06A401CE0625A2862
:1017B0002CD30020E06229E03C0B0020E807002049
:1017C0007001002078030020A0050020983A000056
:1017D000B8EB00006C0100208E030020BBEB000082
:1017E000A82F000028030020E40900201030A0608A
:1017F0000CE0E06A04214002401900F029FDE06A93
:10180000802240024119D84800F0E0FC002028E77F
:10181000F0B589B001F0A1F80024E443012805D017
:1018200002F0BAFF002803D020461AE7204618E746
:1018300000F0FEFFCD4C052803D0CD4820620020EB
:101840000FE70E2000F088FACA4F7D21381AC90030
:101850000BF05CF86062216A8142F0D02062C64DD4
:101860002846E968803001291CD081690A0AE169AB
:101870000A7082694A70E96AE669090AB170E96A20
:10188000F170406A64210BF041F830710E2000F0D5
:1018900063FA7D26381AF600B0420AD2E1690020C8
:1018A00048710FE0C1690A0AE1690A70C2694A70A9
:1018B000E1E70E2000F050FA381A31460BF026F816
:1018C000E1694871AD480021406A08F099F9E16981
:1018D00088716946002009F014FF0798D021411A49
:1018E000E069C1710699017205994172039981728B
:1018F0000299C172019901730021C173E86F002838
:1019000002D0012818D020E001F024F8E121C9001C
:10191000484331460AF0FAFFE1692030487301F08C
:1019200019F8E121C900484331460AF0EFFF2030A1
:10193000E169000A887308E001F00CF8E169487376
:1019400001F008F8E169000A88738D48AB2100684E
:10195000017001214170FF21417483490F225439E4
:1019600088480AF0FBFF87491222891E00200AF0EE
:1019700000FF606A002800D161E70020FFF763FEE6
:101980005DE77A494870704770B5062804D9012090
:10199000FFF7F7FF002070BD7349734A2C390D180B
:1019A000E978223A09021418E07801430BD000F0DC
:1019B00042FFE978E27809021143884208D3012006
:1019C000FFF7DFFF07E00020FFF7DBFF002070BD1F
:1019D0000020FFF7D6FF002070BD6749C031C86204
:1019E00070476548C030C06AC0B27047F0B589B072
:1019F0006946002009F085FE0698C6B20598C4B273
:101A0000FFF7EFFF00275C4DA04206D02046FFF70E
:101A1000E4FF2F62002004F07AFCA868002804D0BC
:101A2000012816D0AF6000201BE6E86900280CD022
:101A300000F001FFE969884203D30120FFF7A1FF0D
:101A4000F1E70020FFF79DFFEDE70020FFF799FF8A
:101A5000E9E7454D2C3D6978B14205D1A878201AB7
:101A6000C0B2FFF791FFDEE71F201E220B000AF035
:101A7000D8FF0D08091030373E454C535A61686F46
:101A80000800D0E7A978401A0019C0B2FFF77CFF20
:101A9000C9E72E78B00705D1642130460AF036FF39
:101AA00000290ED1FF21913130460AF02FFF002985
:101AB00007D0A8781C21081A0019C0B2FFF764FFEC
:101AC000B1E7A8781D21081A0019C0B2FFF75CFF22
:101AD000A9E7A978401A0019C0B2FFF755FFA2E79D
:101AE000A878101A0019C0B2FFF74EFF9BE7A9783B
:101AF000401A0019C0B2FFF747FF94E7A878101A00
:101B00000019C0B2FFF740FF8DE7A978401A00190D
:101B1000C0B2FFF739FF86E7A978401A0019C0B2B2
:101B2000FFF732FF7FE7A878101A0019C0B2FFF75D
:101B30002BFF78E7A978401A0019C0B2FFF724FFFD
:101B400071E7A878101A0019C0B2FFF71DFF6AE705
:101B5000A978401A0019C0B2FFF716FF63E700200A
:101B60007047024840787047F40700207001002059
:101B7000FF0F0000A82F00003C0B002028030020CE
:101B80006C0100208E03002010B556490878C04330
:101B9000C0B20870002804D00821012008F04EFBD4
:101BA00010BD0821012008F064FB10BD10B500F045
:101BB000F1F8FEF755FE00F09DF8FFF728F907F061
:101BC0005AF900F045F900F071F9FFF797F9FFF7BE
:101BD000C6FF00F093F900F0D3F900F00AFA00F024
:101BE00041FAFEF7FBFA10BDFFF7E0FF00F04DFBF6
:101BF00000F062FB06F003FD00F070FA06F041FD14
:101C000008F040F800F097FA0020FFF7ACF93649E9
:101C1000102000F09DF8FF212D310120FEF72BFE52
:101C2000022000F099F8002805D10121022000F0DF
:101C30008FF8FEF796FB012000F08EF800280AD1FD
:101C40001421012000F084F807F069FB00F094FAF9
:101C500026480121C161002000F07EF8002804D14F
:101C6000022100F075F806F011FE1B2000F074F858
:101C7000002805D132211B2000F06AF8FFF7BBF9DC
:101C80001D2000F069F8002805D132211D2000F048
:101C90005FF8FFF7BDFD1C2000F05EF8002805D1BD
:101CA00032211C2000F054F8FFF742FC042000F021
:101CB00053F8002806D17D21C900042000F048F81F
:101CC000FFF794FE232000F047F8002806D10521F5
:101CD000232000F03DF80648FEF774FBFFF754FFA1
:101CE0009EE70000A6010020DC050000FC0B0020A0
:101CF0005803002010B50A4C59202060162020609F
:101D0000882020600121002008F0B6F8054808F07E
:101D1000E6F9054808F0A5F90020206010BD000094
:101D2000000100508813000080F0FA0210B5174936
:101D30000878C043C0B20870002804D009210020F0
:101D400008F07CFA10BD0921002008F092FA10BDBD
:101D50000F4A8000115070470D49800008587047A5
:101D600000210A4A5078401CC0B250700A280CD397
:101D70000020507006480268002A01D0521E0260FE
:101D8000001D491C4529F6D3D0E77047A701002064
:101D9000040A002010B5284C59202060162020602D
:101DA0008820206001220421022008F01DFA234827
:101DB000816810229143816001221146022008F0BF
:101DC00013FA0121022008F054FA01220321022013
:101DD00008F00AFA0321022008F04BFA012202213E
:101DE000104608F001FA0221012008F042FA01220F
:101DF0000721022008F0F8F90721022008F039FA3B
:101E000002210122084608F0EFF90221084608F0F5
:101E100030FA03220921002008F0E6F90322082104
:101E2000012008F0E1F903220821012008F0DCF983
:101E30000020206010BD00000001005080400050D4
:101E400010B5FFF78DFF13480168491C016010BDF4
:101E500010B5114C59202060162020608820206089
:101E600009F088FF0721022007F092FF01220B49A9
:101E7000002009F086FF0123094A022100200AF010
:101E8000F6F800200AF085F900200AF0A7F90020F2
:101E9000206010BD1C00002000010050204E0000FA
:101EA000411E000010B5FEF743FA10BD10B5104CEE
:101EB00059202060162020608820206009F05AFFF9
:101EC0000721042007F064FF01220A49022009F0DB
:101ED00058FF02210123084A08460AF0C8F80220E8
:101EE0000AF057F902200AF079F90020206010BDAD
:101EF00000010050204E0000A51E00007FB51E4CC2
:101F000059202060162020608820206008F09AFE6A
:101F1000342008F055FA0221002009F0A2FA01202D
:101F20006A4610706421517000259570D570134970
:101F30000191029503906946002008F058FF0121A5
:101F4000002009F048FA0121002008F0A9FE2560D0
:101F50007FBD1FB55F2800D95F2001216A4611703F
:101F60006422101A6A465070044801900391694631
:101F7000002008F03CFF1FBD00010050400D030091
:101F80007FB5544C592020601620206088202060A6
:101F9000362008F015FA0221084609F062FA0120FD
:101FA0006A4610706421517000259570D5704A49B9
:101FB0000191029503906946022008F018FF012163
:101FC000022009F008FA0121022008F069FE2560CC
:101FD0007FBD1FB501216A4611706422101A6A463E
:101FE00050703D48019003916946022008F0FFFEC1
:101FF0001FBD7FB5374C59202060162020608820F7
:102000002060372008F0DCF90221032009F029FACA
:1020100001206A4610706421517000259570D570BA
:102020002D490191029503906946032008F0DFFED7
:102030000121032009F0CFF90121032008F030FE2F
:1020400025607FBD1FB501216A4611706422101AF8
:102050006A4650702048019003916946032008F0B9
:10206000C6FE1FBD7FB51B4C592020601620206086
:1020700088202060352008F0A3F90221012009F012
:10208000F0F901206A4610706421517000259570A6
:10209000D5701149019102950390694608F0A7FE99
:1020A0000121084609F097F90121084608F0F8FDDA
:1020B00025607FBD1FB501216A4611706422101A88
:1020C0006A4650700448019003916946012008F067
:1020D0008EFE1FBD00010050D007000010B58AB071
:1020E0000B4C59202060162020608820206009F0C9
:1020F00022FA01A809F046FA002009F004FD05487B
:10210000016B082291430163002020600AB010BDDA
:1021100000010050008000401F4859210160162135
:102120000160882101601D490A6808231A430A607A
:1021300000210160704710B5174C5920206016200F
:102140002060882020600221002007F021FE072067
:102150000AF0B4F812480AF0CEF8002108460AF056
:1021600062F8002102200AF05EF8002107200AF040
:102170005AF80020206010BD10B5074C592020608F
:102180001620206088202060002106200AF04BF8ED
:102190000020206010BD0000000100500040004001
:1021A0001921000003E00221491E0029FCD1401E34
:1021B000F9D27047044A03E01146491E0029FCD1B8
:1021C000401EF9D2704700009D170000F8B5054683
:1021D0000F461646002472B6592135480160162173
:1021E0000160882101600AF069FB07E02046800059
:1021F000641CC01929680AF0E3FA2D1D761EF5D279
:102200000AF072FB2A480021016062B6F8BDF8B5F9
:1022100006460F461546002472B65921244801602F
:1022200016210160882101600AF048FB07E0204682
:102230008000641CC01931460AF0ECFA361D6D1E90
:10224000F5D20AF051FB1A480021016062B6F8BDD0
:10225000F8B506460D46002472B65920144F386072
:1022600016203860882038600AF028FB05E02046F8
:102270008000641C80190AF0F9FA6D1EF7D20AF08A
:1022800033FB0020386062B6F8BD10B5084C592009
:10229000206016202060882020600AF02BFB13218C
:1022A0003E2209030348FFF7B2FF0020206010BD63
:1022B000000100503C0B0020F8B5D54B7D22986AF8
:1022C0005201904200D29A62D249986A884200D95B
:1022D0009A62D149186B884200D21963CF481C6BAF
:1022E000844200D91963D86F0126012800D9DE671E
:1022F000C748C82480304568C82D00D244604B27A9
:102300004568FF00BD4200D944608468642C01D256
:1023100064248460FF2584683C35AC4201D9642480
:1023200084600468022C00D206600468022C00D984
:102330000660C4680025012C00D9C5605C68002CCB
:1023400000D05D60DC68022C00D9DD60B44C1F69F0
:10235000A74201D903241C61B24CC76AA74200D32B
:10236000C462B14CC76AA74201D8AE4CC4629C6932
:10237000012C00D99D61AA4CDF69A74200D9DD611B
:10238000A34B1B6A5B1C01D1A14B1D62A04CA74F44
:10239000C034636ABB4201D2A54B6362A54F636A36
:1023A000BB4201D9A24B6362A36A012B00D9A5628B
:1023B000076BFF23FF2F00D90363476BFF2F00D963
:1023C0004363876BFF2F00D98363C36B0F2B00D947
:1023D000C5632368012B00D926606368032B00D9ED
:1023E0006560A3680F2B00D9A560E3680F2B00D9A7
:1023F000E560874B9B6B102B01D3854B9D63836AF4
:10240000642B01D964238362874B07695B1E9F425B
:1024100000D3056187699F4200D38561C7699F42E8
:1024200000D3C561E069012800D9E561206A01286F
:1024300000D92562794BA7697F489F4200D9A061E6
:102440007D48A369834200D2A0617D23206B9B015C
:10245000984200D92163206B904200D22163774BD0
:10246000626B77489A4200D96063764B626B9A42FE
:1024700000D26063664FF86B884202D3A269904233
:1024800001D96948F863386C884202D3A269904246
:1024900001D96D483864786C884202D3A2699042B1
:1024A00001D96A487864B86C884202D3A269904224
:1024B00001D96748B864F86C884202D3A269904297
:1024C00001D96448F864386D884202D3A269904209
:1024D00001D957483865786D884202D3A269904285
:1024E00001D95D487865B86D884202D3A2699042EF
:1024F00001D95A48B865F86D884202D3A269904262
:1025000001D95748F865386E884202D3A2699042D3
:1025100001D954483866786E884202D3A269904245
:1025200001D951487866B86E884202D3A2699042B8
:1025300001D94E48B866F86E884202D3A26990422B
:1025400001D94B48F866386F884202D3A26990429D
:1025500001D948483867786F884202D3A26990420F
:1025600001D945487867B86F884202D3A16988428B
:1025700001D93148B867FF21153140480AF007FA00
:1025800014213F480AF003FA14213E480AF0FFF9EB
:10259000002002F07AFD0020FFF7DBFC3A4881685A
:1025A0001022914381600121022007F062FE032185
:1025B000022007F05EFE0721022007F03FFE022105
:1025C000084607F056FE002002F0BAF8012001F09C
:1025D000E8FD082000F05AF8002006F034FC7D6089
:1025E0007E6206F0A9FC002811D006F073FC0028DA
:1025F0000DD106F088FC002809D11620616AFFF78A
:10260000A7FB012000F042F80020FEF77FFBF8BD99
:102610003C0B0020E02E000070170000400D03006E
:10262000FF0F0000C027090010270000983A0000A3
:1026300060EA000080A90300007102007C15000020
:10264000AC0D0000DC050000204E000030750000DD
:10265000409C000050C30000701101008038010050
:10266000905F0100A0860100B0AD0100C0D4010060
:10267000D0FB0100E0220200F0490200040A002021
:10268000780300208C03002080400050FF494870F0
:102690007047FE480078704770B50021084607F083
:1026A000F6FD0021012007F0F2FD0021022007F0D5
:1026B000EEFD0621022007F0C1FD0F21012007F0E9
:1026C000BDFD0321002007F0B9FDF149012048625A
:1026D0000020FFF77EFC0020FFF7B4FC0020FFF78E
:1026E000E9FCFEF77FFBFEF7B6FB0020FFF731FCAD
:1026F0000121022007F0BDFD0321022007F0B9FDF2
:102700000221012007F0B5FD0721022007F0B1FDED
:10271000E04CA0681026B043A0600221084607F0F4
:10272000A8FD0021022007F089FD0020FEF71EFC15
:10273000D94D59202860162028608820286008F08C
:10274000EEF808F090FA002009F03DFF280309F0A8
:102750003AFF012009F055FC032009F052FC00204B
:1027600007F02EFE00221146012007F03DFD012159
:102770000022084607F038FD002007F0B4FB0020D7
:102780002860FFF713FA0020FFF7E3FB0121022086
:1027900007F06FFD0321022007F06BFD02210120ED
:1027A00007F067FD0721022007F048FDA068B0434D
:1027B000A0600221084607F05CFDB548C030416AC0
:1027C0001620FFF7C5FAFF21F5312820FFF7C0FAE0
:1027D000FF2191310F20FFF7BBFAFFF75AFF0128C5
:1027E00002D10720FFF752FF70BDA8494872704719
:1027F000A64988717047A5494871704700B5A74A36
:10280000A749D068884203D90120FFF7F4FF02E00E
:102810000020FFF7F0FF1921D0680902884203D297
:102820000120FFF7E5FF00BD0020FFF7E1FF00BD3D
:102830009648407870479648C0300069704708B5A0
:10284000934919228031496A0020120291420BD922
:102850007D20944BC000994206D2881A7D21C90080
:10286000484391490AF052F80A210AF04FF80A2128
:102870000AF04CF803000AF0D4F80A060F18212ACF
:10288000333C454E57608948009003230022402185
:102890003820FEF7CBF908BD8548009003230022BD
:1028A00040213820FEF7C2F908BD8248009003237A
:1028B000002240213820FEF7B9F908BD7E4800907B
:1028C0000323002240213820FEF7B0F908BD7B48E1
:1028D00000900323002240213820FEF7A7F908BD0D
:1028E000774800900323002240213820FEF79EF90C
:1028F00008BD744800900323002240213820FEF7D1
:1029000095F908BD7048009003230022402138202B
:10291000FEF78CF908BD6D4800900323002240218A
:102920003820FEF783F908BD694800900323002290
:1029300040213820FEF77AF908BD6648009003234D
:10294000002240213820FEF771F908BD5048C03000
:10295000406970474D48C06A70474D484069C0B2F1
:1029600070474B48C0300068C0B27047F0B585B0C2
:10297000002001903D20FFF7EFF9444D444E7D24A7
:1029800000272035C036E400002860D028780028D1
:1029900002D02F70FEF75FFA4320FFF7DDF9002821
:1029A0004FD1FF21F5314320FFF7D2F90120FEF787
:1029B0009BFA3D20FFF7D0F9474909F0A7FF474DA3
:1029C0000846294609F0A2FF2A214843444F012125
:1029D000C2190E20FEF70CF93D20FFF7BDF929467C
:1029E00009F094FF0846214609F090FF2A21484348
:1029F000C21901211C20FEF7FBF83A48009004237D
:102A0000032232212A20FEF711F9012336A20421E4
:102A10000A20FEF72CF900211120FFF799F9002177
:102A20001220FFF795F900211320FFF791F90021FB
:102A30001420FFF78DF9AF20FEF752FA0020FEF7C1
:102A400053FA1620716AFFF783F905B0F0BD2878B4
:102A5000002803D101202870FEF7FDF93B20FFF785
:102A60007BF90A4900287DD0C87D002802D0CF75A7
:102A7000FEF7F1F90120FEF737FA0549C86800288A
:102A800040D001285BD0022879D033E0AC0100208F
:102A90003C0B002080400050000100502803002023
:102AA000282300006C2000006C0700005AD70000AB
:102AB00042D700002AD7000012D70000FAD6000043
:102AC000E2D60000CAD60000B2D600009AD60000B6
:102AD00082D600006AD60000A08601001027000000
:102AE0000BEA00007AD700004C4F41442E2E2E0AEC
:102AF00000000000CF60AF20FEF7F2F90020FEF7E3
:102B0000F3F9A2E70523FFA201210D20FEF7AFF89C
:102B10000523FEA203210D20FEF7A9F8FD48009031
:102B20000323012206210020FEF780F8FA480090D6
:102B30000323012240213A20FEF778F8DBE7052342
:102B4000F6A201210D20FEF792F80523EFA2032142
:102B50000D20FEF78CF8EF48032301220621009098
:102B6000002001E018E00AE0FEF760F8EA48009073
:102B70000323012240213A20FEF758F8BBE7052342
:102B8000E8A201210320FEF772F803210523E7A242
:102B90000846FEF76CF8AEE7E648C07D002804D191
:102BA000E4490120C875FEF756F93C20FFF7D4F838
:102BB000002854D0DF48017E002902D00776FEF7B6
:102BC0004AF90120FEF790F90123DBA219460520FE
:102BD000FEF74DF8DB490869030009F022FF0627DC
:102BE000040B121920270523D7A203210720FEF783
:102BF0003EF81DE00523D6A203210D20FEF737F88D
:102C000016E00523D4A203210D20FEF730F80FE0D3
:102C10000523D3A203210D20FEF729F808E00523A0
:102C2000D1A203210720FEF722F801E0032008616A
:102C3000B84800900523032206210020FDF7F6FF87
:102C4000B54800900523032240213A20FDF7EEFF0E
:102C5000AF20FEF745F90020FEF746F9F5E6B54846
:102C6000007E002804D1B34901200876FEF7F3F86E
:102C70001E20FFF771F8002841D0AE48417E0029A0
:102C800002D04776FEF7E7F80120FEF72DF9FEF7B0
:102C900070F9B74C012804D0FEF76BF9002814D066
:102CA00026E004230022302110200094FDF7BEFF0F
:102CB0000023B0A204210120FDF7D9FF0023B0A218
:102CC00005210420FDF7D3FF12E004230022302168
:102CD00010200094FDF7AAFF0023A6A204210120E2
:102CE000FDF7C5FF0023A9A205210120FDF7BFFFC5
:102CF000AF20FEF7F5F80020FEF7F6F8A5E68D48C0
:102D0000407E002804D18B4901204876FEF7A3F8C5
:102D10002720FFF721F8002842D08648817E00292D
:102D200002D08776FEF797F80120FEF7DDF8FFF76F
:102D300018FE012804D0FFF714FE002815D028E063
:102D4000954800900423002230211020FDF76EFFEB
:102D5000002392A204210120FDF789FF0521002311
:102D600087A20846FDF783FF13E08F4800900423F5
:102D7000002230211020FDF759FF002387A20421F3
:102D80000120FDF774FF002380A205210120FDF73B
:102D90006EFFAF20FEF7A4F80020FEF7A5F854E67A
:102DA0006448807E002804D1624901208876FEF7BD
:102DB00052F83E20FEF7D0FF002830D05D48C17E9B
:102DC000002902D0C776FEF746F80120FEF78CF8FE
:102DD000B06A002809D0012814D0B762AF20FEF7EE
:102DE0007FF80020FEF780F82FE600236FA2012174
:102DF0000820FDF73CFF05236FA203210720FDF704
:102E000036FFEBE7002369A201210820FDF72FFF21
:102E100005236BA203210220FDF729FFDEE74548C9
:102E2000C07E002804D143490120C876FEF713F87C
:102E30003F20FEF791FF002862D03E48017F002925
:102E400002D00777FEF707F80120FEF74DF80023C0
:102E50005DA219460220FDF70AFF3A4F5D49386A24
:102E60005D4E5E4D88424CD3214609F04FFD5C49D2
:102E700009F04CFD08465B4909F048FD103014216B
:102E80004843421901210720FDF794FE2146386A84
:102E900009F03CFD534909F039FD0846214609F087
:102EA00035FD103014214843421901211120FDF74E
:102EB00081FE2146386A09F029FD214609F026FDE8
:102EC0000846642109F022FD1030142148434219BC
:102ED00001211B20FDF76EFE2146386A09F016FD20
:102EE000642109F013FD08460A2109F00FFD103096
:102EF00014214843421901212520FDF75BFE73E0B0
:102F000068E288E0574154540A0000004D4F4445A0
:102F10000A0000007CDB000088DB000054454D50B7
:102F20000A0000004D454D4F52590A00204D4F44B4
:102F300045200A00AC010020535452454E475448E6
:102F40000A0000003C0B0020204D494E200A0000E2
:102F5000534F46540A0000004E4F524D0A000000E5
:102F6000484152440A000000204D4158200A000008
:102F7000EACF0000424C5545544F4F54480A0000D8
:102F80002020204F4E202020200A00002020204F0B
:102F900046462020200A0000EAD000002020204CD5
:102FA00045442020200A00006AD1000053544541C6
:102FB0004C54480A00000000204F464620200A00DA
:102FC00020204F4E20200A002020544F44415920F9
:102FD000200A000080969800F6E1000083E50000DA
:102FE000A0860100102700002146386A09F08EFCF7
:102FF0000A2109F08BFC1031142041434A190121A8
:103000002F20FDF7D7FD032301224321392000960D
:10301000FDF70CFED1E0FF4988424ED3214609F06E
:1030200075FCFD4909F072FC0846214609F06EFC6A
:10303000103014214843421901210C20FDF7BAFD3C
:103040002146386A09F062FC214609F05FFC084617
:10305000642109F05BFC103014214843421901211E
:103060001620FDF7A7FD2146386A09F04FFC6421C0
:1030700009F04CFC08460A2109F048FC10301421E4
:103080004843421901212020FDF794FD2146386A6A
:1030900009F03CFC0A2109F039FC103114204143AD
:1030A0004A1901212A20FDF785FD032301223E2133
:1030B00034200096FDF7BAFD7FE0D84988423BD323
:1030C000214609F023FC214609F020FC0846642132
:1030D00009F01CFC10301421484342190121112031
:1030E000FDF768FD2146386A09F010FC642109F0FB
:1030F0000DFC08460A2109F009FC10301421484350
:10310000421901211B20FDF755FD2146386A09F0BF
:10311000FDFB0A2109F0FAFB1031142041434A1942
:1031200001212520FDF746FD0323012239212F200F
:103130000096FDF77BFD40E0B749884228D3214641
:1031400009F0E4FB642109F0E1FB08460A2109F0DB
:10315000DDFB103014214843421901211620FDF7F0
:1031600029FD2146386A09F0D1FB0A2109F0CEFB7E
:103170001031142041434A1901212020FDF71AFD86
:103180000323012234212A200096FDF74FFD14E08D
:10319000214609F0BBFB0A2109F0B8FB10311420CD
:1031A00041434A1901211B20FDF704FD032301229D
:1031B0002F2125200096FDF739FD002398A2032139
:1031C0000220FDF754FDFFF736FB934EB04251D37A
:1031D000FFF731FB914909F099FB0846314609F0A8
:1031E00095FB103014214843421904210720FDF7B4
:1031F000E1FCFFF720FB314609F088FB0846214639
:1032000009F084FB10301421484342190421112095
:10321000FDF7D0FCFFF70FFB214609F077FB0846CE
:10322000642109F073FB1030142148434219042132
:103230001B20FDF7BFFCFFF7FEFA642109F066FBD7
:1032400008460A2109F062FB103014214843421954
:1032500004212520FDF7AEFCFFF7EDFA0A2109F065
:1032600055FB1031142041434A1904212F20FDF74A
:10327000A1FCA8E0FFF7DFFAA04240D3FFF7DBFA9A
:10328000314609F043FB0846214609F03FFB103068
:1032900014214843421904210C20FDF78BFCFFF751
:1032A000CAFA214609F032FB0846642109F02EFBD8
:1032B000103014214843421904211620FDF77AFCEE
:1032C000FFF7B9FA642109F021FB08460A2109F049
:1032D0001DFB103014214843421904212020FDF722
:1032E00069FCFFF7A8FA0A2109F010FB103114203D
:1032F00041434A1904212A20FDF75CFC63E0FFF7F3
:103300009AFA64282FD3FFF796FA214609F0FEFABD
:103310000846642109F0FAFA103014214843421992
:1033200004211120FDF746FCFFF785FA642109F01E
:10333000EDFA08460A2109F0E9FA10301421484351
:10334000421904211B20FDF735FCFFF774FA0A210E
:1033500009F0DCFA1031142041434A1904212520D8
:10336000FDF728FC2FE0FFF766FA0A281ED3FFF7C7
:1033700062FA642109F0CAFA08460A2109F0C6FA7D
:10338000103014214843421904211620FDF712FC85
:10339000FFF751FA0A2109F0B9FA1031142041431C
:1033A0004A1904212020FDF705FC0CE0FFF743FA41
:1033B0000A2109F0ABFA1031142041434A190421C3
:1033C0001B20FDF7F7FBAF20FDF78AFD0020FDF77E
:1033D0008BFD43E41548007F002804D113490120E8
:1033E0000877FDF738FD3A20FEF7B6FC00287ED0BE
:1033F0000E48417F002902D04777FDF72CFD0120C0
:10340000FDF772FD0A49002008F07BF90423094DFD
:10341000022211E040420F0010270000A0860100A8
:103420002020505546465320200A0000AC010020C1
:10343000180B00205FDB000020211E200095FDF707
:10344000F5FB0423022231212F200095FDF7EEFB2E
:10345000FE4DFF49E86909F059FA0846264631460B
:1034600009F054FAFB4C00010019009004230222D9
:1034700009210120FDF7DAFB3146E86909F046FA37
:103480000846642109F042FA000100190090042363
:10349000022210210820FDF7C9FB6421E86909F028
:1034A00035FA08460A2109F031FA000100190090A6
:1034B0000423022217210F20FDF7B8FB0A21E86937
:1034C00009F024FA080100190090042302221E21A9
:1034D0001620FDF7ABFB6421A86909F017FA08462E
:1034E0000A2109F013FA00010019042300E037E073
:1034F0000090022228212020FDF798FB0A21A869CC
:1035000009F004FA080100190090042302222F2177
:103510002720FDF78BFB6421686909F0F7F908465D
:103520000A2109F0F3F90001001900900423022296
:1035300039213120FDF77AFB0A21686909F0E6F9A3
:103540000801001900900423022240213820FDF7D1
:103550006DFBAF20FDF7C4FC0020FDF7C5FC1EE4A9
:10356000BD48407F002804D1BB4901204877FDF7C2
:1035700072FC3920FEF7F0FB00285ED0B648817F50
:10358000002902D08777FDF766FC0120FDF7ACFC2F
:10359000AE49002008F0B5F8AC4C6421E06809F0B1
:1035A000B5F908460A2109F0B1F938214843AB4D75
:1035B00005234019009001220E210020FDF736FB63
:1035C0000A21E06809F0A2F9382041434819009027
:1035D000052301221C210E20FDF728FBA0480090A6
:1035E0000523012223211D20FDF720FB6421A06873
:1035F00009F08CF908460A2109F088F93821484376
:10360000401900900523012232212420FDF70EFBF2
:103610000A21A06809F07AF938204143481900903E
:103620000523012240213220FDF700FBAF20FDF7EA
:1036300057FC0020FDF758FCCBE68748807F002828
:1036400004D1854901208877FDF705FC0F20FEF79E
:1036500083FB00282CD08048C17F002902D0C77787
:10366000FDF7F9FB0120FDF73FFC042302220921AD
:103670000020FDF707FC0423022240213620FDF73D
:1036800001FC784800220090042340211046FDF7F9
:10369000CDFA754800900623042240210020FDF752
:1036A000C5FAAF20FDF71CFC0020FDF71DFC90E6DD
:1036B0006948C07F002804D167490120C877FDF719
:1036C000CAFB2D20FEF748FB002838D02D20FEF73E
:1036D00043FBA04233D26878002812D06F70FDF708
:1036E000BAFB00211120FEF733FB00211220FEF768
:1036F0002FFB00211320FEF72BFB00211420FEF7E7
:1037000027FB0120FDF7F0FB58480090042300221E
:1037100038210820FDF78AFA002355A2042105204C
:10372000FDF7A5FA002355A205210220FDF79FFA17
:10373000AF20FDF7D5FB0020FDF7D6FB49E6687802
:10374000002803D101206870FDF785FB1720FEF7E4
:1037500003FB002833D04048417D002905D0477540
:10376000AE20FDF7BDFBFDF776FBFFF7F6F800286E
:1037700010D10120FDF7B8FB43480090062300223A
:1037800038210820FDF752FAAF20FDF7A9FB0020F1
:10379000FDF7AAFBFFF7E1F8012888D1FDF7A4FBAC
:1037A0003A4800900623002230211020FDF73EFA0F
:1037B000AF20FDF795FB0020FDF796FB09E62648B4
:1037C000407D002804D1244901204875FDF743FBC2
:1037D0001820FEF7C1FA002818D01F48817D002963
:1037E00002D08775FDF737FB0120FDF77DFB2748E9
:1037F00000900623002230211020FDF717FAAF2099
:10380000FDF76EFB0020FDF76FFBE2E51248807DBF
:10381000002804D1104901208875FDF71CFB1220F7
:10382000FEF79AFA0949A431039100283BD1FF2100
:103830005F311220FEF78CFAB06A012830D00120E7
:10384000FDF752FB01482430C06821E0180B00202E
:1038500010270000EFD70000AC0100202FD9000096
:10386000AAD70000DACB0000DACC0000ACDB000005
:10387000202054454D502020200A000050524F5423
:1038800045435445440A0000DACD0000FACE00005A
:10389000002809D0FE49012852D002283DD04FE02F
:1038A000AE20FDF71DFBCBE1F9494868002802D0A6
:1038B000012804D044E0F748096B416340E0FEF77B
:1038C000B7FF05280AD0F448F24A00780102F3480D
:1038D0000078084364214843506331E00E20FEF72E
:1038E0003BFAEF49081A214609F010F8EA49085C4A
:1038F0000102E84841630E20FEF72EFAE849081A53
:10390000214609F003F8E549085CE249496B0843A0
:1039100064214843DF49486312E04868002802D028
:10392000012807D00CE0886B80004018C16BD94893
:10393000416305E0886B80004018C16BD548416346
:10394000D349C868002803D001287ED002284BD173
:10395000D048416BD348814247D3022300222F2114
:103960002A20FDF78FFA0323022238213220FDF7A7
:1039700089FAC848CC49406B08F0C8FF0846C949D5
:1039800008F0C4FF2A214843C849421800210846CC
:10399000FDF72EF9BF48C349406B08F0B7FF084652
:1039A000C34908F0B3FF2A214843C0494218002107
:1039B0000E20FDF71DF9B748BD49406B08F0A6FF82
:1039C0000846214608F0A2FF2A214843B749421879
:1039D00000211C20FDF70CF9B648009003230222B9
:1039E00032212A20FDF722F924E1032300221C21A1
:1039F0001A20FDF747FA0323002221211F20FDF79B
:103A000041FAAD480090032300221F211C20FDF73E
:103A10000DF9A048A649406B884206D20022032334
:103A20000E211046FDF72EFA0EE09E4908F06EFFBB
:103A300008469F4908F06AFF2A2148439B494218DB
:103A400000210846FDF7D4F800E02AE091489849A3
:103A5000406B08F05BFF0846214608F057FF2A211B
:103A600048439249421800210E20FDF7C1F88948C9
:103A70002146406B08F04AFF0846642108F046FFE3
:103A80002A2148438949421800212120FDF7B0F836
:103A9000884800900323022237212F20FDF7C6F823
:103AA000C8E04868002802D001287ED0C2E0C86F74
:103AB000002802D0012840D0BCE0FEF7B9FE05285E
:103AC00037D00398806802902146029808F01EFFC4
:103AD0000846642108F01AFF2A2148437349421816
:103AE00000210846FDF784F86421029808F00EFFD3
:103AF00008460A2108F00AFF2A2148436B49421868
:103B000000210E20FDF774F80A21029808F0FEFE4D
:103B10002A20414365480A1800211C20FDF768F857
:103B2000664800900323022236212A20FDF77EF802
:103B300080E0FEF70FFF0290C6E7FEF779FE05284A
:103B400039D00398406802902146029808F0DEFEC2
:103B50000846642108F0DAFE2A21484353494218F6
:103B600000210846FDF744F86421029808F0CEFED3
:103B700008460A2108F0CAFE2A2148434B49421848
:103B800000210E20FDF734F80A21029808F0BEFE4D
:103B90002A20414345480A1800211C20FDF728F837
:103BA000032302224648362100E008E000902A2044
:103BB000FDF73CF83EE0FEF7CDFE0290C4E7FEF7CD
:103BC00037FE052842D0FEF7C1FE0290214602983A
:103BD00008F09CFE0846642108F098FE2A2148431C
:103BE0003249421800210846FDF702F86421029884
:103BF00008F08CFE08460A2108F088FE2A21484376
:103C00002A49421800210E20FCF7F2FF0A210298EF
:103C100008F07CFE2A20414324480A1800211C2079
:103C2000FCF7E6FF264800900323022236212A20D3
:103C3000FCF7FCFFAF20FDF753F90020FDF754F926
:103C40001120FEF789F8002804D0C6E0FEF782FEB6
:103C50000290BBE764211120FEF77AF8B06A0128D0
:103C600030D00120FDF740F94220FEF775F800281A
:103C700073D0A878002806D0AF70052303221D2139
:103C80000020FDF7FFF8FEF7D3FD05281ED024E045
:103C90003C0B0020AC010020E8070020DC070020DE
:103CA000442F0000A086010040420F000BEA0000F4
:103CB0001027000072D7000063DB00008ED70000E1
:103CC00082D70000AE20FDF70BF986E00E20FEF74C
:103CD00043F8FF49091AFF4881630123FEA203212B
:103CE0000B20FCF7C4FFFB4DFC49A86B08F00EFE4F
:103CF0000846FB4908F00AFE10300A214843F94FF4
:103D00000321C2190020FCF737FFF549A86B08F022
:103D1000FDFD0846214608F0F9FD10300A21484310
:103D2000C21903210720FCF727FF2146A86B08F0E2
:103D3000EDFD0846642108F0E9FD10300A214843F2
:103D4000C21903210F20FCF717FF0123E6A203216C
:103D50001720FCF78CFF3AE0FFE7E44801690B000D
:103D600008F05FFE0631040D161F2831E048009070
:103D7000052303221D210020FCF758FF25E0DD4824
:103D80000090052303221D210020FCF74FFF1CE0BB
:103D9000D9480090052303221D210020FCF746FF8F
:103DA00013E0D6480090052303221D210020FCF7D4
:103DB0003DFF0AE0D2480090052303221D21002088
:103DC000FCF734FF01E0032101610120A870AF205E
:103DD000FDF786F80020FDF787F81320FDF7BCFFFC
:103DE000002822D1FF212D311320FDF7B1FFB06A49
:103DF000012817D00120FDF777F8FDF7BAF8012860
:103E000014D00223002236212E20FDF73BF8FEF7C6
:103E100016FDB64DE868002811D0012854D00228BC
:103E200043D143E0AE20FDF75BF8DEE0B5480090FB
:103E30000223002236212E20FCF7F8FEE7E7FEF7EA
:103E4000FAFC214608F062FD0846642108F05EFD98
:103E500010300A214843A34D032142192620FCF7C4
:103E60008BFEFEF7E8FC642108F050FD08460A21AD
:103E700008F04CFD10300A214843421903212D203F
:103E8000FCF77AFEFEF7D7FC0A2108F03FFD10315F
:103E90000A2041434A1903213420FCF76DFE012317
:103EA00099A203213B20FCF7E2FE98E0A86B2C21AD
:103EB000401C4843954905234018009003224021A7
:103EC0002A20FCF7B3FE8AE0854F686BB84243D3E3
:103ED00001238FA203212920FCF7C9FE01237EA222
:103EE00003213020FCF7C3FE7C49686B08F00EFD0F
:103EF0000846394608F00AFD10300A214843794F38
:103F00000321C2192520FCF737FE7549686B08F0BC
:103F1000FDFC0846214608F0F9FC10300A21484310
:103F2000C21903212C20FCF727FE2146686B08F0FC
:103F3000EDFC0846642108F0E9FC10300A214843F2
:103F4000C21903213420FCF717FE012371A20321BB
:103F50003B20FCF78CFE42E001235FA203212920D5
:103F6000FCF785FE01236AA203213020FCF77FFEC7
:103F70003946686B08F0CAFC0846214608F0C6FCC2
:103F800010300A214843574F0321C2192520FCF75E
:103F9000F3FD2146686B08F0B9FC0846642108F07F
:103FA000B5FC10300A214843C21903212D20FCF72B
:103FB000E3FD6421686B08F0A9FC08460A2108F0BB
:103FC000A5FC10300A214843C21903213420FCF714
:103FD000D3FD01234FA203213B20FCF748FEAF2075
:103FE000FCF77EFF0020FCF77FFF1420FDF7B4FEF6
:103FF000002800D009E4FA211420FDF7A9FEB06AD8
:1040000001280BD00120FCF76FFF384DE86800282D
:1040100009D001280BD0022810D104E0AE20FCF713
:104020005FFF05B0F0BD03988069019006E0FEF7E0
:10403000FFFB052874D0039880690190002326A215
:1040400005210420FCF713FE254E0198314608F0A7
:104050005DFC08462746394608F058FC10308100C0
:1040600040182D4C052102190020FCF767FD394648
:10407000019808F04BFC0846642108F047FC10301A
:1040800081004018021905210820FCF757FD642122
:10409000019808F03BFC08460A2108F037FC103074
:1040A00081004018021905210F20FCF747FD1B482D
:1040B0000090062305221D211620FCF7B7FDED6AAE
:1040C000002305A205212920FCF7D1FD314628E077
:1040D000442F0000AC0100202E0A0000A086010041
:1040E0001027000035E30000530A00003C0B0020BD
:1040F00058DF000092DF0000CCDF000006E0000087
:1041000040E000009AD70000500A00006CDC00007C
:10411000200A0000570A00000EE20000D4D7000079
:104120003BE0284608F0F2FB0846394608F0EEFB73
:10413000103081004018021905212520FCF7FEFCF3
:104140003946284608F0E2FB0846642108F0DEFB09
:10415000103081004018021905212D20FCF7EEFCDB
:104160006421284608F0D2FB08460A2108F0CEFB5D
:10417000103081004018021905213420FCF7DEFCC4
:104180000023FFA205213B20FCF771FDAF20FCF7C7
:10419000A7FE0020FCF7A8FE43E70398C069019042
:1041A0004CE7F849C8727047F648407A704770B5D6
:1041B0000024FFF7F9FF00285FD00221084606F02F
:1041C0003DF8FCF75CF8FCF771F8641C822CF8D31E
:1041D000ED480A21C569406906462C1A204608F0B8
:1041E00095FB0146E948704308F090FB1E2801D971
:1041F0001E3800E00020E34AD16E0B460F33984290
:1042000002D80F39884200D2D066E148D16E0161F0
:10421000002E01D100210161C82C02D3711BC829D5
:1042200001D2DC4901610020FEF7DFFA02210846D5
:1042300006F01FF80920FDF7B5FF1E211120FDF73C
:1042400087FD1E211220FDF783FD1E211320FDF79F
:104250007FFD1E211420FDF77BFD1E211F20FDF791
:1042600077FD1E212020FDF773FD96212120FDF70B
:104270006FFDC6492220FDF76BFD70BD10B52F20E4
:10428000FDF76AFD00280ED1C0492F20FDF760FD23
:10429000FFF78DFFBE48C04900693738884202D316
:1042A0000120FFF77EFF10BDB64908707047B54981
:1042B00088627047B349C8627047B248806A7047E5
:1042C000F0B589B0B14C2A202146FDF741FD2146C9
:1042D0004220FDF73DFDAE4DA86968612E4640368F
:1042E000AE4AB169AE48914200D9B061B16981422C
:1042F00000D2B061A64FA34C803FF868002807D0D9
:1043000001287ED002287DD00020F86009B0F0BDE1
:104310000121022005F092FF7868002810D00128C2
:1043200011D0002078603420FDF716FD002854D00D
:104330003869030008F075FB064F232E5139444FAE
:10434000386B6065EFE70E20FDF706FD9549081A0A
:104350008E4908F0DBFA9449085C000260650E2083
:10436000FDF7FAFC8F49081A884908F0CFFA8F49FF
:10437000085C616D0843642148436065D3E7616D63
:1043800008910801401A642108F0C0FA0899081A37
:10439000606522E0626D0A2050436421079208F0B4
:1043A000B5FA079A101A606517E0626D0A2050434B
:1043B0006421069208F0AAFA069A801860650CE05B
:1043C000616D05910801401A642108F09FFA059972
:1043D0004018606501E003203861B069616D884272
:1043E00000D2606568484068F8624043696908F037
:1043F0008DFA7863616D0A46FF3A2D3A904207D2F2
:1044000001E015E022E1226B5F2A01D2521C2263F7
:10441000FF312D31884204D9206B002801D0401E85
:1044200020632020FFF746FF206BFDF792FD6DE72C
:104430000121022005F002FF7868002816D001282B
:1044400029D0002078605048514F4068803FF86282
:10445000E9694043049108F059FA786339690B001F
:1044600008F0DFFA062E1F2225282B2EF86F0028D1
:1044700009D00128E7D16868A0654B21C9008842AE
:10448000E1D9A165DFE7A868A065FF213C3188423A
:10449000D9D9A165D7E7FEF759FAA0650120F867D9
:1044A000D1E7434921660FE0424921660CE04249C9
:1044B000216609E04149216606E04149216603E0A1
:1044C000334A0321803A1161E968012906D1304954
:1044D000803940004863206E400020660498AF6930
:1044E000B84201D2E76501E00498E0652868012838
:1044F0001AD002281BD001202860E06D2349C01B80
:104500004843216D08F002FA20494843394608F033
:10451000FDF91930FFF7CBFE1D4D803DE86F0028F7
:104520000AD001280CD015E0306B2065E5E7706BF0
:10453000FF30F5302065E0E7FFF7BFFE606609E079
:10454000FFF7BBFEE121C9004843104908F0DEF93E
:1045500020306066A26D616E91420CD2686B236E52
:10456000984208D2206B5F2801D2401C2063206B48
:10457000062800D9E064914249D92C2022E00000AD
:10458000560A0000AC01002028030020E8030000C8
:10459000BC0B00200F270000810B0000400D030022
:1045A00000710200442F0000E8070020DC07002013
:1045B00030750000409C000050C3000060EA00001D
:1045C00070110100FDF7C8FB002813D1A16D606ECA
:1045D000401A322804D900212C20FDF7B9FB04E051
:1045E0003221091A2C20FDF7B3FBE06C062801D913
:1045F000401EE064E16CA06C884201D2401CA064C3
:10460000A06C884201D9401EA064A06C2063A16DFB
:10461000606E884212D9A06E401CA066052811D990
:104620000846FFF747FE2D20FDF796FB002809D12D
:104630007D2109012D20FDF78BFB03E0FFF73AFEFA
:104640000020A066206BFDF784FC5FE601210220BC
:1046500005F0F4FD7868002810D0012814D000205F
:1046600078603420FDF778FB002841D038690300DA
:1046700008F0D7F9063C101B3E26313CB86B800091
:10468000C019C06B6065ECE7B86B8000C019C06BE7
:104690006065E6E7616D03910801401A642108F046
:1046A00035F90399081A606522E0626D0A205043CB
:1046B0006421029208F02AF9029A101A606517E044
:1046C000626D0A2050436421019208F01FF9019A9B
:1046D000801860650CE0616D00910801401A64214A
:1046E00008F014F900994018606501E00320386172
:1046F000B069616D884200D26065FD484068F8622B
:104700004043696908F002F97863616D0A46FF3A2F
:104710002D3A904204D2226B5F2A01D2521C2263AE
:10472000FF312D31884204D9206B002801D0401E72
:1047300020632020FFF7BEFD206BFDF70AFCE5E5B6
:10474000EC49C870704770B5E94D0A21E86A4843E2
:104750006A2108F0DBF87D210446C90048430A219C
:1047600008F0D4F86A680146101B8722D200504333
:1047700008F0CCF80028DF4A116F0B460F3398423F
:1047800002D80F39884200D21067DB48116FC1612F
:1047900070BDD84880797047D648C0787047FEB55C
:1047A0000027D548D44C4030C069803C002804D153
:1047B000E068012801D10020E060FEF7CEF8CF4D7F
:1047C000102601280ED0FFF7E7FF002817D00020A1
:1047D000FDF7BFFBA868B043A8600121022005F0E7
:1047E00048FDFEBD0020FDF7B4FBA868B043A860FB
:1047F0000121022005F03DFDFEF7B8F8FEBDFFF7F0
:10480000C8FF00282CD0A868B043A8600120FCF79E
:104810006BFBFCF724F9FCF71EFBB948009003235F
:10482000012230211020FCF701FA0023B5A2032158
:104830000220FCF71CFA0023B5A204210220FCF799
:1048400016FA0322B549002007F093FFAF20FCF7CA
:1048500047FB0120FFF774FF0020FCF784FBFEBD3F
:10486000A348C168AE48814231D2A249C86B401CFE
:10487000C863FF21F53188422CD9A868B043A860ED
:104880000120FCF731FBFCF7EAF8FCF7E4FA9C485E
:1048900000900323012230211020FCF7C7F90023E8
:1048A00098A203210220FCF7E2F9002398A2042138
:1048B0000220FCF7DCF903229A49002007F059FF97
:1048C000AF20FCF70DFB0120FFF73AFFFEBD894941
:1048D0000020C86386480021406A05F091F95528F8
:1048E0002DD9A868B043A8600120FCF7FDFAFCF7B9
:1048F000B6F8FCF7B0FA8C480090042302223A2163
:104900002220FCF793F9002388A202210820FCF75B
:10491000AEF9002387A203210820FCF7A8F903229F
:104920008649002007F025FFAF20FCF7D9FA0120C7
:10493000FFF706FF82493D20FDF70AFAFEBDFDF7AD
:1049400010F9002829D0A868B043A8600120FCF71E
:10495000CBFAFCF784F8FCF77EFA7A48009005233E
:10496000022214210020FCF761F90023764A02217B
:104970001C20FCF77CF9002374A203211C20FCF707
:1049800076F903227349002007F0F3FEAF20FCF70D
:10499000A7FA0120FFF7D4FEFEBDE068564C0028C0
:1049A00001D0022834D12169642931D2A868B043EA
:1049B000A8600120FCF798FAFCF751F80120FFF7F6
:1049C000F0FB0020A061FCF746FA63480090022348
:1049D000002230211020FCF729F95A4800900623C4
:1049E000032214210020FCF721F900235BA20321FC
:1049F0001820FCF73CF900235BA204211820FCF7E7
:104A000036F9AF20FCF76CFA0120FFF799FEFEBDE6
:104A1000012834D12069372831D2A868B043A86072
:104A20000120FCF761FAFCF71AF80120FFF7B9FB47
:104A30000020A061FCF70FFA4748009002230022F3
:104A400030211020FCF7F2F83E48009006230322A4
:104A500014210020FCF7EAF8002340A203211820CB
:104A6000FCF705F9002340A204211820FCF7FFF809
:104A7000AF20FCF735FA0120FFF762FEFEBD3C498E
:104A8000206988427DD23B4A90427AD9A868B043D7
:104A9000A8600120FCF728FAFBF7E1FF0120FFF7EF
:104AA00080FB0020A061FCF7D6F92B480090022380
:104AB000002230211020FCF7B9F82248009006238C
:104AC000032214210020FCF7B1F8002323A20321C4
:104AD0001820FCF7CCF8002327A204211820FCF7AB
:104AE000C6F8AF20FCF7FCF90120FFF729FEFEBD58
:104AF00028030020AC010020BC0B002080400050A7
:104B000076E100002020204C4F572020200A000092
:104B10002042415454455259200A0000AFEB000096
:104B200088130000B5EB0000BACF0000544F4F0AC5
:104B300000000000484F540A00000000C1EB0000D4
:104B400030750000BAE00000682F0000505546465E
:104B5000530A0000BEEB0000F6E000004F484D2075
:104B6000544F4F0A000000004C4F570A000000004D
:104B70000F270000B80B0000484947480A00000012
:104B8000FFE788422DD3A868B043A8600120FCF756
:104B9000ABF9FBF764FF0120FFF703FB0020A061E6
:104BA000FCF759F90023FFA203210820FCF75FF866
:104BB0000023FFA204210520FCF759F8FF480090CC
:104BC0000223002230211020FCF730F8AF20FCF740
:104BD00087F90120FFF7B4FDFF209130FDF7EAFAD5
:104BE000FEBD17213838C90188420BD2A069372889
:104BF00008D2A868B043A8600120FFF7D2FA0020CD
:104C0000A061FEBDFFF7C5FD002835D1EC487D2130
:104C1000C068490188422CD2EA49086C401C0864EB
:104C2000FF21F531884227D9A868B043A860012048
:104C3000FCF75AF9FBF713FFFCF70DF9E248009077
:104C40000323012230211020FBF7F0FF0023DFA215
:104C500004210220FCF70BF80023DF4A0521022083
:104C6000FCF705F8AF20FCF73BF90120FFF768FDE2
:104C7000FEBDD449002008642220FDF76DF800280D
:104C800032D0D049002048643320FDF765F8002871
:104C900071D0A868B043A8600120FCF725F9FBF7A4
:104CA000DEFEFCF7D8F8CD48009004230122402115
:104CB0002C20FBF7BBFF0023C9A202211846FBF7FB
:104CC000D6FF0023C8A203211846FBF7D0FF00231C
:104CD000C7A204211846FBF7CAFFAF20FCF700F972
:104CE0000120FFF72DFDFEBDE069029032283DD97D
:104CF000A16901910521019807F008FE0199411869
:104D0000029881422ED9BD48C0680128BCD1AD4966
:104D1000486C401C4864FF21F5318842B4D9A8682A
:104D2000B043A8600120FCF7DFF8FBF798FEFCF722
:104D300092F80523B2A201210320FBF798FF03217B
:104D40000523B14A0846FBF792FFAF20FCF7C8F8ED
:104D50000120FFF7F5FC0720FDF798FCA74900208C
:104D6000C860FEBD9749002048648DE79549002042
:104D7000486489E7FFE72020FCF7EEFF002840D1D8
:104D80009E48C16801293CD0406BA049884238D96F
:104D9000FBF775FA7F1C052FFAD38948E12140699A
:104DA000C90088422DD2A868B043A8600120FCF752
:104DB0009BF8FBF754FEFCF74EF895480090022351
:104DC000002230211020FBF731FF002391A20321A4
:104DD0000920FBF74CFF002375A204210520FBF7F7
:104DE00046FF03228E49002007F0C3FCAF20FCF7EA
:104DF00077F80120FFF7A4FC8A493320FCF7A8FFCD
:104E0000FEBD2120FCF7A8FF002832D1FFF79BFC54
:104E1000E06932282DD2A868B043A8600120FCF7D1
:104E200063F8FBF71CFEFCF716F8794800900223A4
:104E3000002230211020FBF7F9FE00237AA2032183
:104E40000920FBF714FF002359A204210520FBF7DA
:104E50000EFF03227249002007F08BFCAF20FCF705
:104E60003FF80120FFF76CFC6E493320FCF770FF20
:104E7000FEBDFFF725FAFDF779FDFEBD5148C07A6A
:104E8000704710B55D4A6B498032106937388842E7
:104E900017D2FFF7F3FF002813D00020FFF781F9A6
:104EA0009069116902461E32914202D81E38814231
:104EB00007D20420FDF7EAFBFBF7CDFF41490120B3
:104EC000087310BD3F488078704738B53D480024CE
:104ED000017B002902D00473FBF7BDFF0120FCF722
:104EE00003F80021052354A20846FBF7C0FE052362
:104EF00053A202210020FBF7BAFE052352A204218F
:104F00000A20FBF7B4FE052350A204212C20FBF756
:104F1000AEFE4F4806230090042219460020FBF7FE
:104F200085FE4C4800900623042240213A20FBF7DE
:104F30007DFEFFF7C7FF484D002802D0012817D19A
:104F400017E004F058FE002812D0002004F004F806
:104F5000424800900623042240213A20FBF766FED7
:104F60002846FDF727F9FBF776FF0720FDF78EFBB4
:104F700084E004F040FE002813D0002003F0ECFF92
:104F80001E49803108698861354A904200D38C619E
:104F900088690862334806230422009019460020DD
:104FA00062E06BE020434845434B20200A000000AC
:104FB00041544F4D495A45520A000000F6E00000A6
:104FC00028030020AC0100207AE0000020204348A4
:104FD00045434B20200A0000104B0000BAE00000BF
:104FE000444F4E27540A000041425553450A0000E1
:104FF00050524F5445435453210A00003C0B0020AB
:105000002057415454200A002C2F000060EA000071
:1050100036E100002D53484F52542D200A00000065
:10502000B2EB0000881300002053484F5254202058
:105030000A000000810B00004953204E45570A002A
:10504000434F494C3F200A00590A00004E0A000015
:105050007CDB000088DB0000DC050000A0DB00003A
:105060000F27000094DB0000FBF7E0FD2846FDF76A
:10507000A1F8FBF7F0FE0720FDF708FBAF20FBF7D8
:105080002FFF0020FBF730FF38BDFF490860704755
:10509000FE4988727047FD48807A704710B5132426
:1050A000240304212046FDF7D3F83E222146F6488A
:1050B000FDF78CF810BDF5498870704710B58AB0BF
:1050C000F248002444738473C4730474447401204C
:1050D000FBF70AFFFBF7BFFEEB48C030416A162022
:1050E000FCF736FEEA490D20FCF732FE002004F002
:1050F0000AF9002004F00AF90020FFF7C6FF00209B
:10510000FFF7D9FFFBF73DFCFFF7C8FFAE20FBF729
:10511000E7FE0720FDF7BAFAFFF7BDFF002820D011
:105120000020FFF7B5FF0120694608714C71D9488E
:105130004169029101690391C168049105948168F4
:105140000691416807910068089008A90C7101A9AF
:10515000002006F0CBFB002803D001A9002006F0B8
:10516000C5FB0AB010BDF8B504460D4616461F46ED
:105170003520FCF7F1FD64280BD90120FBF7B4FEC4
:10518000C54800903B46324629462046FBF74EFD77
:10519000F8BD0120FBF7A8FEC04800903B46324610
:1051A00029462046FBF742FDF8BDF8B504460D46FA
:1051B00016461F463620FCF7CFFD64280BD9012088
:1051C000FBF792FEB64800903B4632462946204601
:1051D000FBF72CFDF8BD0120FBF786FEB1480090DF
:1051E0003B46324629462046FBF720FDF8BD38B540
:1051F00003F0B5FE002809D003F0B1FE01282CD041
:10520000FFF75CFFAF20FBF76BFE38BD04F0EAFC54
:105210000028F7D0002003F09CFE0120FBF764FE7D
:10522000FBF719FEA0480090042300223021102033
:10523000FBF7FCFC00239DA205210A20FBF717FDCC
:1052400000239BA205210F20FBF711FD002399A24B
:1052500005211420FBF70BFDD4E704F0C6FC002861
:1052600032D0002003F07EFE0120FBF73DFE192422
:10527000640121460720FCF76BFD21460820FCF75E
:1052800067FDFF242D34204603F060FE204603F026
:105290005AFE04F0ADFC00257B4C002803D104F03D
:1052A000AAFC00280AD0002004F036F8002003F001
:1052B00053FE606A012814D001206062606A0028F1
:1052C00011D0012822D06562052303220621002087
:1052D000FFF76BFF0523032240213A20FFF743FF2E
:1052E00090E76562EAE7062303223A211846FBF7B6
:1052F000C9FD05236FA201210720FBF7B8FC052398
:105300006EA203210720FBF7B2FCDDE70623032290
:105310003A211846FBF7B6FD052366A201210720B6
:10532000FBF7A5FC052367A203210220FBF79FFCE6
:10533000CAE770B50C4611461A46049B092814D0DA
:105340000A2812D0632810D064280ED05F4DA842DE
:105350000BD06D1CA84208D05D4DA84205D06D1C35
:10536000A84202D05B4DA84202D12046FBF78AFD3D
:1053700070BDF8B504F03CFC0026444D002809D06F
:10538000002003F0C9FF687C401CC0B26874042888
:1053900000D96E7404F02FFC3E4C00285DD0002034
:1053A00003F0DAFDFFF78EFD002802D0012854D16A
:1053B00029E00120FFF76CFE687C030007F031FB59
:1053C00005040B11171D4D0043492068884244D243
:1053D000401C206041E060680C283ED2401C6060A8
:1053E0003BE0A0681F2838D2401CA06035E0E06890
:1053F000172832D2401CE0602FE020693B282CD2D5
:10540000401C206129E00120FFF742FE687C030078
:1054100007F007FB05040C12181E23007D212068ED
:105420000901884219D9401E206016E060680128F1
:1054300013D9401E606010E0A06801280DD9401EFD
:10544000A0600AE0E068002807D0401EE06004E0A9
:105450002069012801D9401E206104F0C6FB002804
:105460007ED0002003F07EFD66611C4E03230122E6
:1054700020211E200096FBF7D9FB032301223121B6
:105480002F2000962CE000003C0B0020AC010020F7
:10549000442F0000340C0020A0DB000088DB00005B
:1054A00094DB00007CDB0000EAD50000360A000037
:1054B0002E0A0000504F5745520A0000204F464622
:1054C000200A000020204F4E200A0000E7030000C1
:1054D0000F2700009F860100330800005FDB0000FB
:1054E000FBF7A4FBFD49206807F010FA7D2708466A
:1054F000FF00394607F00AFAF94E0001801901222F
:105500000090032309211046FBF790FB39462068E1
:1055100007F0FCF90846642107F0F8F9000180194A
:1055200000900323012210210820FBF77FFB642158
:10553000206807F0EBF908460A2107F0E7F90001B7
:10554000801900900323012217210F20FBF76EFB27
:105550000A21206807F0DAF908018019032300E026
:10556000ACE0009001221E211620FBF75FFB6421B6
:10557000606807F0CBF908460A2107F0C7F9000177
:10558000801900900323012228212020FBF74EFBE5
:105590000A21606807F0BAF9080180190090032316
:1055A00001222F212720FBF741FB6421A06807F08F
:1055B000ADF908460A2107F0A9F900018019009009
:1055C0000323012239213120FBF730FB0A21A06897
:1055D00007F09CF908018019009003230122402163
:1055E0003820FBF723FB6421E06807F08FF90846B9
:1055F0000A2107F08BF9000180190090052303228E
:1056000015210D20FBF712FB0A21E06807F07EF957
:10561000080180190090052303221D211520FBF7A6
:1056200005FBB04800900523032225211D20FBF730
:10563000FDFA6421206907F069F908460A2107F09C
:1056400065F9000180190090052303222D212520F2
:10565000FBF7ECFA0A21206907F058F908018019D4
:1056600000900523032235212D20FBF7DFFA687C0B
:105670009D4D030007F0D5F9050423426180220007
:105680006421206807F042F908460A2107F03EF934
:105690000001401900900323012217210F20FBF77E
:1056A000C5FA0A21206807F031F908014019009075
:1056B000032301221E211620FBF7B8FAF8BD64214E
:1056C000606807F023F908460A2107F01FF9000176
:1056D000401900900323012228212020FBF7A6FA7D
:1056E0000A21606807F012F90801401900900323AD
:1056F00001222F212720FBF799FAF8BD6421A06829
:1057000007F004F908460A2107F000F900014019E2
:1057100000900323012239213120FBF787FA0A2167
:10572000A06807F0F3F80801401900900323012254
:1057300040213820FBF77AFAF8BD6421E06807F0D1
:10574000E5F808460A2107F0E1F800014019009049
:105750000523032215210D20FBF768FA0A21E068D2
:1057600007F0D4F8080140190090052303221D21F9
:105770001520FBF75BFAF8BD6421206907F0C6F835
:1057800008460A2107F0C2F80001401900900523DD
:1057900003222D212520FBF749FA0A21206907F071
:1057A000B5F80801401900900523032235212D206A
:1057B000FBF73CFAF8BDF0B58BB003F0D0FB002648
:1057C0004A4C002814D003F0CAFB012838D003F05B
:1057D000C6FB474F474D02287ED003F0C0FB03288D
:1057E0007BD0FFF76BFCAF20FBF77AFB0BB0F0BD73
:1057F00004F0F8F9002821D0002003F0AAFB0120D2
:10580000FBF772FBFBF727FB3B48009004230022C9
:1058100030211020FBF70AFA002338A205210320CB
:10582000FBF725FA002336A205210820FBF71FFA13
:10583000002334A205210D20FBF719FAA673D2E745
:10584000FFF740FB002802D001282CD115E004F01E
:10585000CFF9002803D104F0CEF9002823D000208E
:1058600003F05AFD002003F077FBA07B052802D24D
:10587000401CA07317E0A67315E004F0B9F90028E6
:1058800003D104F0B8F900280DD0002003F044FD46
:10589000002003F061FBA07B002802D0401EA07313
:1058A00001E00520A07304F0A0F900289BD000209F
:1058B00003F058FB0120FBF717FBFBF7CCFA192587
:1058C0006D0129460720FCF743FA29460820FCF71A
:1058D0003FFAFF252D351BE0DCE0E5E31027000053
:1058E000EFD700006CDB00008FD80000AC01002077
:1058F00083E50000FC0B0020EAD20000350A00001E
:105900002E0A000053455454494E470A0000000037
:10591000284603F01BFB284603F015FBA07B030081
:1059200007F07FF80605203B56829D045BE7FD48A3
:1059300000900423002230211020FBF777F9002388
:10594000F9A205211846FBF792F905210023F7A2D9
:105950000846FBF78CF90023F5A205210A20FBF786
:1059600086F940E7F54800900423002230211020FA
:10597000FBF75CF90023F2A205211846FBF777F943
:1059800005210023E9A20846FBF771F90023EDA2E7
:1059900005210A20FBF76BF925E7ED480090042369
:1059A000002230211020FBF741F90023E9A2052154
:1059B0000420FBF75CF90023DCA205210920FBF79A
:1059C00056F90023E4A205210E20FBF750F90AE75F
:1059D000E44800900423002230211020FBF726F930
:1059E0000023E1A205210E20FBF741F90023CFA2FD
:1059F00005211320FBF73BF90023CEA20521182037
:105A0000FBF735F902A9002005F07BFED74809997C
:105A1000016008994160079981600599C160049906
:105A2000016103994161DEE6D14800900423002220
:105A300030211020FBF7FAF80023CEA20521042024
:105A4000FBF715F90023B9A205210920FBF70FF98F
:105A50000023C9A205210E20FBF709F9C3E6C948B6
:105A600000900423002230211020FBF7DFF80023F0
:105A7000C5A205211846FBF7FAF805210023ABA2C1
:105A80000846FBF7F4F80023C0A205210A20FBF723
:105A9000EEF8A8E6C048B54C807B783C030006F0E1
:105AA000C0FF060565FDFCFBFA049CE604F0A0F8C7
:105AB000002803D104F09FF8002809D0002003F04B
:105AC0002BFC002003F048FAA86A00282FD0AE6211
:105AD00004F08BF800281DD0002003F043FA0120C9
:105AE000FBF702FAA86A002824D0012830D0AE6261
:105AF0001924640121460720FCF72AF921460820D1
:105B0000FCF726F9FF242D34204603F01FFA204627
:105B100003F019FA0523032206210020FFF745FBB5
:105B20000523032240213A20FFF71DFB5BE60120FD
:105B3000A862CDE70023994A01210820FBF797F8D6
:105B4000964A05230C3203210720FBF790F8CFE794
:105B50000023924A01210820FBF789F88F4A052388
:105B6000143203210220FBF782F8C1E704F043F866
:105B700000281AD0002003F0EFF9FFF7A3F900285E
:105B800002D0012811D108E0A06A642802D2401C8A
:105B9000A0620AE06420A06207E0A06A0A2802D995
:105BA000401EA06201E00A20A06204F01EF8002856
:105BB00055D0002003F0D6F90120FBF795F900231A
:105BC00077A201210520FBF752F800235DA20221F4
:105BD0000520FBF74CF80620009003233A2206210B
:105BE000A06AFFF7A6FBA06A642839D305236FA239
:105BF00003210220FBF73BF87D21C900A06A06F0D3
:105C000085FE0846642106F081FE103014214843C9
:105C1000C21903210C20FAF7CDFF6421A06A06F017
:105C200075FE08460A2106F071FE10301421484323
:105C3000C21903211620FAF7BDFF0A21A06A06F057
:105C400065FE103114204143CA1903212020FAF7C0
:105C5000B1FF052356A203212A20FBF708F853E0E1
:105C60000A282DD3052351A203210720FAF7FFFFAD
:105C70006421A06A06F04AFE08460A2106F046FEA4
:105C8000103014214843C21903211120FAF792FF62
:105C90000A21A06A03E08FE1F2E0EEE08AE006F07C
:105CA00035FE103114204143CA1903211B20FAF795
:105CB00081FF05233EA203212520FAF7D8FF23E028
:105CC00005233AA203210220FAF7D1FF052337A2C8
:105CD00003210C20FAF7CBFF0A21A06A06F016FE7A
:105CE000103114204143CA1903211620FAF762FF2C
:105CF00005232FA203211620FAF7B9FF05232BA2B3
:105D000003212A20FAF7B3FF0523032206210020EE
:105D1000FFF74BFA0523032240213A20FFF723FA2D
:105D200061E500006AD30000410A00002E0A00006D
:105D30005343522054494D450A000000EAD3000065
:105D4000420A0000434F4E54524153540A0000008F
:105D50006AD40000430A0000534352204449520AC7
:105D6000000000006AD20000440A0000340C002049
:105D7000EAD40000450A000041444A204F484D0A39
:105D8000000000006AD50000460A0000444F574E4C
:105D90004C4F41440A000000AC010020AC2F000031
:105DA0002053435245454E200A000000200A0000BF
:105DB000250A000003F01CFFFF4C002803D103F06C
:105DC0001AFF00280DD0002003F0A6FA002003F0EF
:105DD000C3F8A069002827D0A661A069C0B2FAF76D
:105DE00095FF03F002FF00289AD0002003F0BAF8D4
:105DF0000120FBF779F8A069002818D0012829D0E4
:105E0000A6611924640121460720FBF7A1FF214662
:105E10000820FBF79DFFFF242D34204603F096F861
:105E2000204603F090F8DEE40120A061D5E70623C8
:105E3000032240210020FBF725F80523DFA20121E2
:105E40000220FAF714FF0523DEA203210220FAF74D
:105E50000EFFD6E70623032240210020FBF712F8AD
:105E60000523D6A201210220FAF701FF0523D7A2BC
:105E700003210220FAF7FBFEC3E7FFF77AFAB2E448
:105E800003F0B9FE002818D0002003F065F8FFF7F2
:105E900019F8002802D001280FD107E0216AA06973
:105EA0003231884209D2401CA06106E0216AA06913
:105EB0003239884201D9401EA06103F096FE0028C5
:105EC0006DD0002003F04EF80120FBF70DF8002301
:105ED000C0A219460520FAF7CAFE0023C0A201217C
:105EE0000820FAF7C4FE0023C0A202210820FAF716
:105EF000BEFE0620009003233A220621A069FFF788
:105F000018FABD49A06906F001FD7D250846ED009F
:105F1000294606F0FBFC103014214843C219042125
:105F20000620FAF747FEB548009006230422122106
:105F30001020FAF77BFE2946A06906F0E7FC084628
:105F4000642106F0E3FC103014214843C2190421F7
:105F50001220FAF72FFE6421A06906F0D7FC08464C
:105F60000A2106F0D3FC103014214843C219042141
:105F70001A20FAF71FFE0A21A06906F0C7FC1031AB
:105F800014204143CA1904212220FAF713FE9C4829
:105F900000900623042238212E20FAF747FE06231C
:105FA000042219460020FFF700F9062304224021AD
:105FB0003A20FFF7D8F816E403F01AFE002803D1C0
:105FC00003F019FE00280AD0002003F0A5F90020F4
:105FD00002F0C2FF8B480179002930D0067103F02E
:105FE00004FE00281ED0002002F0BCFF0120FAF7BA
:105FF0007BFF84490879002824D001283BD00E710A
:106000007D24E40021460720FBF7A2FE214608205C
:10601000FBF79EFEFF242D34204602F097FF20461A
:1060200002F091FF0022022306211046FFF7BDF87F
:106030000223002240213A20FFF795F876E401215F
:106040000171CCE7022300223A210620FAF71AFF59
:1060500005236DA200210C20FAF709FE05236CA28E
:1060600002210C20FAF703FE05236B4A04210C20C1
:10607000FAF7FDFDC4E7022300223A210620FAF7D1
:1060800001FF052365A200210720FAF7F0FD052393
:106090005FA202210C20FAF7EAFD05235E4A0421E3
:1060A0000C20FAF7E4FDABE7A07B030006F0B9FC97
:1060B0000605FDFCFBFAF90438E4A86A012806D0BD
:1060C000FEF700FF002805D0012826D114E0FEF7D6
:1060D000F5FF2BE403F08FFD00281ED0002002F016
:1060E0003BFF5049686A884204D27D21C9004018AC
:1060F000686212E0696210E003F07DFD00280CD0B8
:10610000002002F029FF4849686A884204D97D21AD
:10611000C900401A686200E0696203F066FD002869
:1061200049D0002002F01EFF0120FAF7DDFE052312
:1061300022A200210220FAF79AFD022105233BA2A8
:106140000846FAF794FD7D26F6003146686A06F0A7
:10615000DDFB062104233A220091FFF7EAF83549D6
:10616000686A884275D30C4606F0D0FB10301421C3
:106170004843C21904210C20FAF71CFD2146686A25
:1061800006F0C4FB1C4C0846214606F0BFFB10304D
:1061900014214843C21904211620FAF70BFD2146A9
:1061A000686A06F0B3FB0846314606F0AFFB1030D4
:1061B0001421484341E08EE03C0B002053435245FC
:1061C000454E0A004E4F524D414C0A00524F544129
:1061D00054450A002041444A555354200A00000007
:1061E000494E495449414C0A0000000020204F48C4
:1061F0004D20200A00000000102700000AE20000E5
:10620000DBD70000AC010020455849540A000000CB
:10621000444F574E0A000000905D0000454E544523
:10622000520A000080A90300983A00002054494D0A
:1062300045200A00A08601000BE0C219042120209D
:10624000FAF7B8FC0523FFA204212A20FAF70FFD74
:1062500041E0FD4CA04229D306F058FB08462146F8
:1062600006F054FB103014214843C21904211120B8
:10627000FAF7A0FC2146686A06F048FB084631465A
:1062800006F044FB103014214843C21904211B209E
:10629000FAF790FC0523EBA204212520FAF7E7FC8E
:1062A00019E031E02DE029E025E021E0214606F06B
:1062B0002DFB0846314606F029FB103014214843D7
:1062C000C21904211620FAF775FC0523DDA204216A
:1062D0002020FAF7CCFC0623042219460020FEF702
:1062E00064FF0623042240213A20FEF73CFF1DE410
:1062F000FEF7E4FE1AE4FEF7E1FE17E4FEF7DEFE29
:1063000014E4FEF7DBFE11E4FEF7D8FE0EE4CF49FD
:1063100008617047F8B502F022FE002817D002F09D
:106320001EFECA4D7D260027C03DF600012835D04F
:1063300002F015FEC64C02287ED002F010FE0328A3
:106340007BD0FEF7BBFEAF20FAF7CAFDF8BD03F025
:1063500049FC0028F7D0002002F0FBFD0120FAF7ED
:10636000C3FDFAF778FDBB480090042300223021DA
:106370001020FAF75BFC0023B7A205210B20FAF7E7
:1063800076FC0023B5A205211020FAF770FC00234B
:10639000B34A05211520FAF76AFCD4E7FEF792FD0F
:1063A000002802D001281ED110E003F024FC0028B0
:1063B00019D0002002F0D0FDAF60AA49E8698842F8
:1063C00002D2401CE8610EE0E9610CE003F013FC2E
:1063D000002808D0002002F0BFFDAF60E869002867
:1063E00001D0401EE86103F000FC00287AD00020B4
:1063F00002F0B8FD0120FAF777FD00239AA21946B2
:106400000920FAF734FC0320009002233A220621E7
:10641000E869FEF78EFFE869964C002830D06428C2
:1064200035D3314606F072FA0846642106F06EFA5A
:1064300010301421484301E0B5E1C0E10219012107
:106440001120FAF7B7FB6421E86906F05FFA084605
:106450000A2106F05BFA1030142148430219012189
:106460001B20FAF7A7FB0A21E86906F04FFA103162
:10647000142041430A1901212520FAF79BFB56E01D
:1064800005237DA201210720FAF7F1FB4FE00A283E
:1064900029D305237AA201210C20FAF7E8FB642115
:1064A000E86906F033FA08460A2106F02FFA1030A0
:1064B00014214843021901211620FAF77BFB0A2117
:1064C000E86906F023FA1031142041430A1901212A
:1064D0002020FAF76FFB052369A201212A20FAF791
:1064E000C6FB24E052E1052365A201210720FAF74B
:1064F000BEFB052362A201211120FAF7B8FB0A2195
:10650000E86906F003FA1031142041430A19012109
:106510001B20FAF74FFB052359A201212520FAF78A
:10652000A6FB052356A201212F20FAF7A0FB00238A
:1065300054A203210220FAF79AFBFCF77CF9424DA2
:10654000A84251D3FCF777F9514906F0DFF9084624
:10655000294606F0DBF910301421484302190421C2
:106560000720FAF727FBFCF766F9294606F0CEF973
:106570000846314606F0CAF9103014214843021982
:1065800004211120FAF716FBFCF755F9314606F005
:10659000BDF90846642106F0B9F9103014214843CA
:1065A000021904211B20FAF705FBFCF744F96421CA
:1065B00006F0ACF908460A2106F0A8F910301421BB
:1065C0004843021904212520FAF7F4FAFCF733F9BD
:1065D0000A2106F09BF91031142041430A190421C5
:1065E0002F20FAF7E7FAD1E0FCF725F9B04269D39A
:1065F000FCF721F9294606F089F90846314606F0EC
:1066000085F9103014214843021904210C20FAF7AF
:10661000D1FAFCF710F9314606F078F90846642102
:1066200006F074F910301421484302190421162091
:10663000FAF7C0FAFCF7FFF8642106F067F908469C
:106640000A2127E0530A000010270000FC0B00205D
:10665000CC010020EAD10000340A00002E0A00001C
:106660004C4B0000E703000020204D415820200A39
:106670000000000083E500004E455645520A000028
:10668000200A000020414C5245414459200A000094
:10669000A086010006F03AF910301421484302198F
:1066A00004212020FAF786FAFCF7C5F80A2106F043
:1066B0002DF91031142041430A1904212A20FAF738
:1066C00079FA63E0FCF7B7F864282FD3FCF7B3F846
:1066D000314606F01BF90846642106F017F9103020
:1066E00014214843021904211120FAF763FAFCF738
:1066F000A2F8642106F00AF908460A2106F006F914
:10670000103014214843021904211B20FAF752FAD1
:10671000FCF791F80A2106F0F9F8103114204143F2
:106720000A1904212520FAF745FA2FE0FCF783F82F
:106730000A281ED3FCF77FF8642106F0E7F8084624
:106740000A2106F0E3F8103014214843021904210D
:106750001620FAF72FFAFCF76EF80A2106F0D6F8A1
:106760001031142041430A1904212020FAF722FA9B
:106770000CE0FCF760F80A2106F0C8F8103114208C
:1067800041430A1904211B20FAF714FA03230122BA
:1067900006210020FEF709FD0323012240213A20B3
:1067A000FEF7E1FCCFE5FCF746F8002803D0032014
:1067B00002F0ACFD01E0FEF781FCE770C3E50120CB
:1067C000FAF792FB0523FA4A00210720FAF74FFA5D
:1067D0000523F8A202210720FAF749FA0523F7A2B8
:1067E00004210A20FAF743FA0523F5A204212C20FC
:1067F000FAF73DFAF34806230090042219460020D8
:10680000FAF714FAF04800900623042240213A20B7
:10681000FAF70CFA02F077FB00280DD10120E070A6
:106820002F620020FFF773FDE84806230090042242
:1068300019460020FAF7FAF902F04CFB002807D1BC
:10684000E34800900623042240213A20FAF7EEF9AB
:10685000E078002803D102F03DFB0028A2D13046A9
:10686000FBF7A8FCFAF7F7FAFEF728FC6BE5F8B59A
:1068700003F0BEF90025D74C002809D0002002F013
:106880004BFD207C401CC0B22074022800D9257426
:10689000207CFF25D04C002804D0012849D00228B4
:1068A00046D18DE0FEF70EFB002802D001281BD157
:1068B0000EE003F0A0F9002816D0002002F04CFBF7
:1068C000206BFF2802D2401C20630DE025630BE003
:1068D00003F091F9002807D0002002F03DFB206B67
:1068E000002801D0401E206300220223062110460A
:1068F000FEF75BFC0223002240213A20FEF733FC26
:106900000423022206210020FAF7BCFA0423022203
:1069100040213A20FAF7B6FA06230422194600204D
:10692000FAF7B0FA0623042240213A20FAF7AAFA2D
:106930008CE0FEF7C7FA002802D001281BD10EE038
:1069400003F059F9002816D0002002F005FB606B17
:10695000FF2802D2401C60630DE065630BE003F08A
:106960004AF9002807D0002002F0F6FA606B0028F0
:1069700001D0401E60630022022306211046FAF770
:1069800081FA0223002240213A20FAF77BFA0423FD
:10699000022206210020FEF708FC042302224021E7
:1069A0003A20FEF7E0FB0623042219460020FAF7FE
:1069B00069FA0623042240213A20FAF763FA45E0F7
:1069C000FEF780FA002802D001281BD10EE003F068
:1069D00012F9002816D0002002F0BEFAA06BFF28A2
:1069E00002D2401CA0630DE0A5630BE003F003F9A5
:1069F000002807D0002002F0AFFAA06B002801D0D9
:106A0000401EA0630022022306211046FAF73AFA3C
:106A10000223002240213A20FAF734FA042302220A
:106A200006210020FAF72EFA0423022240213A2000
:106A3000FAF728FA0623042219460020FEF7B5FBD0
:106A40000623042240213A20FEF78DFB03F0CDF807
:106A500000287ED0002002F085FA0120FAF744FADF
:106A600005235EA200210720FAF701F90220009019
:106A700000233A221B21206BFEF75BFC7D26206B56
:106A8000F600574D64282BD3314605F03FFF0846EA
:106A9000642105F03BFF10301421484342190021C6
:106AA0001A20FAF787F86421206B05F02FFF0846BB
:106AB0000A2105F02BFF1030142148434219002110
:106AC0002420FAF777F80A21206B05F01FFF103118
:106AD000142041434A1900212E20FAF76BF828E0D0
:106AE0000A281BD3642105F011FF08460A2105F08E
:106AF0000DFF103014214843421900211F20FAF7DE
:106B000059F80A21206B05F001FF10311420414390
:106B10004A1900212920FAF74DF80AE00A2105F068
:106B2000F5FE1031142041434A1900212420FAF7C0
:106B300041F805232BA202210720FAF798F8042038
:106B4000009002233A221B21606BFEF7F2FB606B80
:106B500000E0E0E0642847D3314605F0D7FE084660
:106B6000642105F0D3FE103014214843421902215C
:106B70001A20FAF71FF86421606B05F0C7FE08467B
:106B80000A2105F0C3FE10301421484342190221A6
:106B90002420FAF70FF80A21606B05F0B7FE1031D8
:106BA000142041434A1902212E20FAF703F844E049
:106BB0004C4B000052455345540A0000590A00004E
:106BC0004E0A00007CDB000088DB000094DB000044
:106BD000A0DB0000AC010020BC0B0020523A0A00F0
:106BE00083E50000473A0A000A281BD3642105F018
:106BF0008DFE08460A2105F089FE10301421484315
:106C0000421902211F20F9F7D5FF0A21606B05F018
:106C10007DFE1031142041434A1902212920F9F741
:106C2000C9FF0AE00A2105F071FE1031142041432A
:106C30004A1902212420F9F7BDFF0523FFA20421F0
:106C40000720FAF714F80620009004233A221B21AB
:106C5000A06BFEF76EFBA06B64282BD3314605F0CA
:106C600055FE0846642105F051FE103014214843BA
:106C7000421904211A20F9F79DFF6421A06B05F049
:106C800045FE08460A2105F041FE10301421484314
:106C9000421904212420F9F78DFF0A21A06B05F089
:106CA00035FE1031142041434A1904212E20F9F7F2
:106CB00081FF28E00A281BD3642105F027FE08463F
:106CC0000A2105F023FE1030142148434219042103
:106CD0001F20F9F76FFF0A21A06B05F017FE103196
:106CE000142041434A1904212920F9F763FF0AE0DF
:106CF0000A2105F00BFE1031142041434A190421EA
:106D00002420F9F757FFA06BC2B2606BC1B2206BB1
:106D1000C0B2F9F783FEF8BDC94908607047C84999
:106D200048607047F8B502F01AF9C64DC64C002805
:106D300015D002F014F9FF262D36012837D002F0C5
:106D40000EF90627C14D02287ED002F008F903286B
:106D50007BD0FEF7B3F9AF20FAF7C2F8F8BD02F026
:106D600041FF002820D0002002F0F3F80120FAF7BC
:106D7000BBF8FAF770F804230022302110200095A8
:106D8000F9F754FF0023B2A205211220F9F76FFF93
:106D90000023B0A205211720F9F769FF0023AEA256
:106DA00005211C20F9F763FF00206073D3E7FEF78D
:106DB00089F8002802D001282DD116E002F018FF32
:106DC000002803D102F017FF002824D0002002F091
:106DD000A3FA002002F0C0F8607B032802D2401C16
:106DE000607318E00020607315E002F001FF0028D6
:106DF00003D102F000FF00280DD0002002F08CFA31
:106E0000002002F0A9F8607B002802D0401E6073C9
:106E100001E00320607302F0E8FE00289BD0002010
:106E200002F0A0F80120FAF75FF819277F01394630
:106E30000720FAF78DFF39460820FAF789FF304618
:106E400002F084F8304601E0A8E06BE202F07BF843
:106E5000607B00282FD0012853D0022878D0032847
:106E6000A4D10623052240210020FAF70BF87C4824
:106E700000900423002230211020F9F7D7FE0521CD
:106E8000002378A20846F9F7F2FE002371A205213B
:106E90000A20F9F7ECFE00236FA205210F20F9F775
:106EA000E6FE002370A205212720F9F7E0FE00206E
:106EB000FFF732FF4FE70623052240210020F9F7B4
:106EC000E1FF04230022302110200095F9F7AEFEE7
:106ED000002367A205211220F9F7C9FE00235DA255
:106EE00005211720F9F7C3FE002362A205211C200B
:106EF000F9F7BDFE0120FFF70FFF0020FFF70FFF9E
:106F000029E70623052240210020F9F7BBFF0423CF
:106F10000022302110200095F9F788FE002357A2A7
:106F200005210E20F9F7A3FE00234AA20521132014
:106F3000F9F79DFE002352A205211820F9F797FECC
:106F40000120FFF7E9FE0120FFF7E9FE03E7FFE775
:106F50000623052240210020F9F794FF0423002294
:106F6000302110200095F9F761FE002346A205218B
:106F70000B20F9F77CFE002336A205211020F9F73B
:106F800076FE002341A205211520F9F770FE0120AD
:106F9000FFF7C2FE0220FFF7C2FEDCE6607B00289E
:106FA00009D0274C012809D0022877D00328A7D17F
:106FB000FEF784F8CFE6FFF75AFCCCE6FDF782FF38
:106FC000002802D001281CD10FE002F014FE002896
:106FD00017D0002001F0C0FFA0680F2802D2401C8B
:106FE000A0600EE00F20A0600BE002F004FE00287D
:106FF00007D0002001F0B0FFA068002801D0401E9B
:10700000A06002F0F2FD002874D0002001F0AAFF79
:107010000120F9F769FF05231EA201210720F9F7D6
:1070200026FE009703233A220621A068FEF781F985
:10703000A06800285FD00F2864D030E0423A0A00F0
:10704000FC0B0020EAD00000AC01002083E500002A
:10705000330A00002E0A00004C45440A00000000DC
:107060006AD10000440A00004F46460A00000000B2
:10707000410A00005247420A00000000420A000094
:107080004A554D500A000000430A0000534841444D
:10709000450A000053504545440A000082E00A2892
:1070A00037D30523FFA203210C20F9F7E0FD64216B
:1070B000A06805F02BFC08460A2105F027FC1030DB
:1070C00014214843421903211620F9F773FD0A21C0
:1070D000A06805F01BFC1031142041434A1903211C
:1070E0002020F9F767FD0523EEA203212A20F9F7F6
:1070F000BEFD32E049E00523EBA203210C20F9F7A5
:10710000B6FD2AE00523EAA203210C20F9F7AFFD22
:1071100023E00523E3A203210720F9F7A8FD0523B7
:10712000E0A203211120F9F7A2FD0A21A06805F0D1
:10713000EDFB1031142041434A1903211B20F9F7BC
:1071400039FD0523D7A203212520F9F790FD05235A
:10715000D4A203212F20F9F78AFDA0687821401CD2
:107160004843F9F7B8FBD4490C20FAF7F1FD314652
:107170000720FAF7EDFD31460820FAF7E9FD304621
:1071800001F0E4FE304601F0DEFE05230322062175
:107190000020FEF70AF80523032240213A20FDF7DC
:1071A000E2FFD8E5FDF78EFE002802D001281CD1B1
:1071B0000FE002F020FD002817D0002001F0CCFEE7
:1071C000E0680F2802D2401CE0600EE00F20E06073
:1071D0000BE002F010FD002807D0002001F0BCFEFB
:1071E000E068002801D0401EE06002F0FEFC0028AC
:1071F0007ED0002001F0B6FE0120F9F775FE0523D0
:10720000AE4A01210720F9F732FD009703233A2205
:107210000621E068FEF78DF8E06800282CD00F28E2
:1072200031D00A2836D305239EA203210C20F9F77A
:107230001EFD6421E06805F069FB08460A2105F09F
:1072400065FB103014214843421903211620F9F739
:10725000B1FC0A21E06805F059FB103114204143CC
:107260004A1903212020F9F7A5FC05238DA203214B
:107270002A20F9F7FCFC31E005238BA203210C2026
:10728000F9F7F5FC2AE0052389A203210C20F9F780
:10729000EEFC23E0052383A203210720F9F7E7FC96
:1072A000052380A203211120F9F7E1FC0A21E068FF
:1072B00005F02CFB1031142041434A1903211B20F7
:1072C000F9F778FC052377A203212520F9F7CFFCF5
:1072D000052374A203212F20F9F7C9FCE068F9F710
:1072E000E3FA75490C20FAF733FD3146072000E038
:1072F0000BE0FAF72DFD31460820FAF729FD30465C
:1073000001F024FE304601F01EFE05230322062173
:107310000020FDF74AFF0523032240213A20FDF714
:1073200022FF18E5607B002808D0012871D00228D0
:1073300070D00328F5D1FDF7C1FE0CE5FDF7C2FDC5
:107340005F4C002802D001281CD10FE002F053FC52
:10735000002817D0002001F0FFFDE06B0F2802D2BB
:10736000401CE0630EE00F20E0630BE002F043FC02
:10737000002807D0002001F0EFFDE06B002801D0CD
:10738000401EE06302F031FC00287ED0002001F0B6
:10739000E9FD0120F9F7A8FD0523484A012107204E
:1073A000F9F765FC009703233A220621E06BFDF70D
:1073B000C0FFE06B00282ED00F2833D00A2838D326
:1073C000052338A203210C20F9F751FC6421E06B5E
:1073D00005F09CFA08460A2105F098FA10301421AD
:1073E0004843421903211620F9F7E4FB0A21E06B18
:1073F00005F08CFA1031142041434A190321202052
:10740000F9F7D8FB052327A203212A20F9F72FFC3F
:1074100033E079E075E0052323A203210C20F9F77E
:1074200026FC2AE0052322A203210C20F9F71FFCE9
:1074300023E005231BA203210720F9F718FC0523ED
:1074400018A203211120F9F712FC0A21E06B05F0C4
:107450005DFA1031142041434A1903211B20F9F72A
:10746000A9FB05230FA203212520F9F700FC052322
:107470000CA203212F20F9F7FAFB12490020086122
:10748000E06B410043185B1C00E02DE0A06BC2B232
:10749000606BC1B2206BC0B2F9F734FA06490C2018
:1074A00012E00000200A0000464153540A00000088
:1074B000534C4F570A0000008813000094700000DE
:1074C000BC0B002058030020FAF742FC314607208D
:1074D000FAF73EFC31460820FAF73AFC304601F054
:1074E00035FD304601F02FFD052303220621002043
:1074F000FDF75BFE0523032240213A20FDF733FE12
:1075000029E4FDF7DBFD26E4FDF7D8FD23E4F8B51B
:1075100002F06EFBF94D00280AD0002001F0FCFEBD
:10752000E87B401CC0B2E873102801D30020E87348
:1075300002F061FBF24E00282CD0002001F00CFD7F
:10754000FDF7C0FC002802D0012823D112E0012061
:10755000FDF79EFDE87BEA4A80008019C032C16BCE
:107560009269914204D27D22D2008918C16311E050
:10757000C2630FE00120FDF78BFDE87BE14A80004C
:107580008019C16B914204D97D22D200891AC1634E
:1075900000E0C26302F029FB002877D0002001F050
:1075A000E1FCE87BD84C401C0A2812D303230122BB
:1075B00040210020F9F766FCE87B2C21401C484361
:1075C00000190090032301222B211520F9F72EFB2F
:1075D00011E00323012240210020F9F753FCE87B4E
:1075E0002C21401C4843001900900323012227212D
:1075F0001120F9F71BFBE87BC44980008019C06BA0
:10760000C34CC44F884242D3C34905F07FF90846B2
:10761000BE4905F07BF910301421484302190321BB
:107620000A20F9F7C7FAE87BB84980008019C06BD7
:1076300005F06CF90846394605F068F91030142158
:107640004843021903211420F9F7B4FAE87B3946BC
:1076500080008019C06B05F059F908467D21C900EA
:1076600005F054F9103014214843021903211E205B
:10767000F9F7A0FA052303222B212820F9F702FCB1
:107680000523A6A203212B20F9F7F1FA6DE0B842F9
:107690003FD30523A2A203210620F9F7E8FAE87BED
:1076A0009A4980008019C06B05F030F908463946C8
:1076B00005F02CF9103014214843021903210F2042
:1076C000F9F778FAE87B394680008019C06B05F03D
:1076D0001DF908467D21C90005F018F91030142164
:1076E0004843021903211920F9F764FA05230322FC
:1076F00026212320F9F7C6FB052388A20321262093
:10770000F9F7B5FA052386A203213020F9F7AFFA7D
:107710002BE0052382A203210A20F9F7A8FAE87BCF
:10772000394680008019C06B05F0F0F808467D21CD
:10773000C90005F0EBF81030142148430219032169
:107740001420F9F737FA0523032221211E20F9F727
:1077500099FB052371A203212120F9F788FA05235B
:107760006FA203212B20F9F782FA052303220621B9
:107770000020FDF71AFD0523032240213A20FDF7E2
:10778000F2FCF8BDF8B501F0EAFB002821D001F0C9
:10779000E6FB19277F010026594C012840D001F053
:1077A000DEFB2546C035022872D001F0D8FB274603
:1077B000803703286DD001F0D2FB04286AD001F095
:1077C000CEFB052867D0FDF779FCAF20F9F788FBE1
:1077D000F8BD02F007FA0028F7D0002001F0B9FB4D
:1077E0000120F9F781FBF9F736FB4E48009004239E
:1077F000002230211020F9F719FA00234AA20521AE
:107800000E20F9F734FA002348A205211320F9F7D6
:107810002EFA0023464A05211820F9F728FAD4E762
:1078200002F0E6F9002803D102F0E5F900280BD0B8
:10783000002001F071FD002001F08EFBE0680028BF
:107840002AD001282BD0E66002F0CFF90028BCD066
:10785000002001F087FB0120F9F746FB394607209D
:10786000FAF776FA39460820FAF772FAFF252D352D
:10787000284601F06BFB284601F065FB6660E06876
:1078800000280FD001281BD0022827D0E6609CE7F3
:1078900056E0CFE168E2E7E30120E060D4E70220B0
:1078A000E060D1E70523234A01210320F9F7DFF93E
:1078B0001F4A0321052320320846F9F7D8F984E747
:1078C00005231DA201210320F9F7D1F9184A03214C
:1078D000052320320846F9F7CAF976E7144A05234A
:1078E000183201210320F9F7C2F9114A03210523B7
:1078F00020320846F9F7BBF967E70000AC01002029
:107900003C0B0020701700006CDC0000A08601001A
:1079100083E500001027000040420F00570A0000D6
:10792000200A00006AD00000320A00002E0A00007F
:107930000C2F0000005000002054454D50200A003C
:10794000FDF7C0FA002802D001282DD116E002F080
:107950004FF9002803D102F04EF9002824D000206E
:1079600001F0DAFC002001F0F7FA2069052802D2C4
:10797000401C206118E00120206115E002F038F978
:10798000002803D102F037F900280DD0002001F0C3
:10799000C3FC002001F0E0FA2069012802D9401E52
:1079A000206101E005202061E068002805D0012861
:1079B00061D002287ED0E66007E702F016F90028C1
:1079C0004CD0002001F0CEFA0120F9F78DFA3946AB
:1079D0000720FAF7BDF939460820FAF7B9F9FF256B
:1079E0002D35284601F0B2FA284601F0ACFA0523FD
:1079F000FF4A01210320F9F73AF92069030005F055
:107A000010F8062B040B131B232B0523F94A032123
:107A10000720F9F72CF921E0F64A05230832032163
:107A20000D20F9F724F919E0F24A05231032032159
:107A30000D20F9F71CF911E0EE4A05231832032155
:107A40000D20F9F714F909E0EA4A05232032032151
:107A50000720F9F70CF901E0032020610523032238
:107A600006210020FDF7A1FB0523032240213A2037
:107A7000FDF779FBA9E602F0B8F800286ED00020E7
:107A800001F070FA0120F9F72FFA39460720FAF7CA
:107A90005FF939460820FAF75BF9FF262D363046A4
:107AA00001F054FA304601F04EFAE86900280FD090
:107AB000052300E05FE0D04A01210320F9F7D7F861
:107AC0002069030004F0ADFF064821283038404803
:107AD000F9F7C1F9C9480022009003231421104688
:107AE000F9F7A4F80023C6A203210120F9F7BFF893
:107AF0000023C6A204210120F9F7B9F80023C6A289
:107B000005210120F9F7B3F85FE60523B94A0321FF
:107B10000720F9F7ACF821E0B64A05230832032123
:107B20000D20F9F7A4F819E0B24A05231032032119
:107B30000D20F9F79CF811E0AE4A05231832032115
:107B40000D20F9F794F809E0AA4A05232032032111
:107B50000720F9F78CF801E00320206105230322B8
:107B600006210020FDF721FB0523032240213A20B6
:107B7000FDF7F9FA29E602F038F800284DD0002088
:107B800001F0F0F90120F9F7AFF939460720FAF7CB
:107B9000DFF839460820FAF7DBF8FF252D352846AF
:107BA00001F0D4F9284601F0CEF9924A0523243A8F
:107BB00001210320F9F75BF82069030004F031FF8D
:107BC000062B040B131B232B05238A4A03210720B2
:107BD000F9F74DF821E0874A0523083203210D20EB
:107BE000F9F745F819E0834A0523103203210D20E7
:107BF000F9F73DF811E07F4A0523183203210D20E3
:107C0000F9F735F809E07B4A0523203203210720E4
:107C1000F9F72DF801E00320206105230322062156
:107C20000020FDF7C2FA0523032240213A20FDF788
:107C30009AFACAE5E068002805D0012806D0022893
:107C400075D0E660C1E5FDF739FABEE5E8690028C0
:107C500009D0286A00280AD0FDF734F900280CD092
:107C6000012834D120E0E660FDF728FAADE50120D7
:107C70003860042001F04AFBA7E501F0B9FF0028B5
:107C800003D101F0B8FF002821D0002001F044FB0F
:107C9000002001F061F93868012802D00120386025
:107CA00015E00220386012E001F0A2FF002803D1A5
:107CB00001F0A1FF00280AD0002001F02DFB0020D8
:107CC00001F04AF9386802281BD00220386001F020
:107CD0008CFF0028ADD0002001F044F97D24E400A1
:107CE00021460720FAF734F821460820FAF730F841
:107CF0000120F9F7F9F83868012805D0022829D1C0
:107D000016E001203860E2E7032301224021002031
:107D1000F9F7B8F8052343A201210320F8F7A7FFDC
:107D20000321052341A20846F8F7A1FF12E018E05D
:107D30000323012240210020F9F7A4F801233DA2EA
:107D400019460520F8F793FF0321052337A20846BB
:107D5000F8F78DFFAF20F9F7C3F80020F9F7C4F862
:107D600033E5FFF7D4FB30E5E068002805D00128B3
:107D700006D0022868D0E66027E5FDF79FF924E5E4
:107D800038682F4E2F4C012802D002287ED1C6E041
:107D9000FDF798F8002802D001285DD117E001F026
:107DA00027FF002803D101F026FF002854D000202F
:107DB00001F0B2FA002001F0CFF87D21286B890193
:107DC000884202D20A30286346E0296344E001F089
:107DD0000FFF002803D101F00EFF00283CD0002047
:107DE00001F09AFA002001F0B7F87D2149012CE05A
:107DF00000500000482F000038790000BAE0000071
:107E00002050555243484153450A000041542041F7
:107E1000505020544F0A0000454E41424C4521200D
:107E2000200A00004E49434B454C0A0020434F496D
:107E30004C200A00544954414E49554D0A00000057
:107E40001027000035E300000BE1286B884202D9BF
:107E50000A38286300E0296301F0C7FE002815D026
:107E6000002001F07FF80120F9F73EF80523FF4AD2
:107E700001210320F8F7FBFE0123FDA203210B20C3
:107E8000F8F7F5FE0123FBA2032100E0DCE010205F
:107E9000F8F7EDFE0123F6A203211520F8F7E7FE1F
:107EA0000123F3A203211C20F8F7E1FE3146286BE1
:107EB00004F02CFD7D260846F600314604F026FD30
:107EC00010300A214843021903212320F8F754FEF9
:107ED0003146286B04F01AFD0846642104F016FDB3
:107EE00010300A214843021903212A20F8F744FEE2
:107EF0006421286B04F00AFD08460A2104F006FDFF
:107F000010300A214843021903213120F8F734FECA
:107F1000AF20F8F7E5FF0020F8F7E6FF94E0FCF764
:107F2000D1FF002802D001282DD116E001F060FE1B
:107F3000002803D101F05FFE002824D0002001F0CA
:107F4000EBF9002001F008F8CB49686B884202D2B7
:107F50000A30686317E0696315E001F049FE002804
:107F600003D101F048FE00280DD0002001F0D4F923
:107F7000002000F0F1FFC149686B884202D90A383D
:107F8000686300E0696301F030FE00285CD00020E7
:107F900000F0E8FF0120F8F7A7FFB44A01231032F0
:107FA00019460520F8F763FE0123B1A203210B2037
:107FB000F8F75DFE0123AFA203211020F8F757FE6A
:107FC0000123ABA203211520F8F751FE0123A8A23B
:107FD00003211C20F8F74BFE3146686B04F096FC39
:107FE0007D260846F600314604F090FC10300A2148
:107FF0004843021903212320F8F7BEFD3146686B80
:1080000004F084FC0846642104F080FC10300A214E
:108010004843021903212A20F8F7AEFD6421686B5A
:1080200004F074FC08460A2104F070FC10300A21A8
:108030004843021903213120F8F79EFDAF20F8F7DD
:108040004FFF0020F8F750FF0523032206210020F0
:10805000FDF7ABF80523032240213A20FDF783F812
:1080600015E4FDF72BF812E4E068002805D001289C
:1080700006D002287DD0E66009E4FDF71FF806E48B
:10808000FCF720FF002802D0012829D115E001F0DB
:10809000AFFD002803D101F0AEFD002820D0002064
:1080A00001F03AF9002000F057FFF868002801D0ED
:1080B000FE6015E00120F86012E001F099FD002853
:1080C00003D101F098FD00280AD0002001F024F926
:1080D000002000F041FFF86801281BD00120F86063
:1080E00001F083FD002836D0002000F03BFF7D2406
:1080F000E40021460720F9F72BFE21460820F9F776
:1081000027FE0120F8F7F0FEF868002804D00128C7
:108110001BD10EE0FE60E3E70523544A0121032052
:10812000F8F7A5FD0321052355A20846F8F79FFDA2
:108130000BE005234D4A01210320F8F798FD0321A8
:10814000052351A20846F8F792FDAF20F8F7C8FEC4
:108150000020F8F7C9FE0523032206210020FDF7C1
:1081600024F80523032240213A20FCF7FCFF23E4F6
:10817000FFE7FCF7A3FF1FE438B500F0F0FE00288E
:1081800009D000F0ECFE01282CD0FCF797FFAF20BF
:10819000F8F7A6FE38BD01F025FD0028F7D0002035
:1081A00000F0D7FE0120F8F79FFEF8F754FE38489C
:1081B00000900423002230211020F8F737FD00231F
:1081C00034A205211020F8F752FD002329A2052131
:1081D0001520F8F74CFD00232FA205211A20F8F7EF
:1081E00046FDD4E701F004FD002803D101F003FDB2
:1081F00000280CD0002001F08FF8002000F0ACFE29
:10820000F8F7B7FE01284FD00120F8F7ACFE01F0D7
:10821000ECFC002820D0002000F0A4FE0120F8F79C
:1082200063FE1924640121460720F9F791FD2146D8
:108230000820F9F78DFDFF242D34204600F086FE3E
:10824000204600F080FEF8F794FE002830D0012888
:1082500041D00020F8F787FE0523032206210020E5
:10826000FCF7A3FF05230322402119E0247E000030
:10827000300A00002E0A00007C150000DC0500001A
:108280002020534320200A002020444320200A00BD
:10829000EACF0000310A00004254480A0000000002
:1082A0003A20FCF760FF72E70020F8F75CFEAEE7CB
:1082B0000623032240210020F8F7E4FD0523FFA256
:1082C00001210C20F8F7D3FC0523FEA2032107208F
:1082D000F8F7CDFCC0E70623032240210020F8F781
:1082E000D1FD0523F5A201210C20F8F7C0FC0523E0
:1082F000F6A203210C20F8F7BAFCADE7F5480068B8
:10830000C0B2704710B5FFF7F9FF030004F089FB16
:108310000604070A0D101316FFF72EFF10BDFFF716
:1083200031FA10BDFEF7FEFC10BDFDF7F3FF10BDE6
:10833000FDF741FA10BDFCF75AFF10BD0020FCF715
:10834000A4FE10BDF8B5E34B00271F605F609F607F
:10835000DF60032018615F619F61DF611F6201259B
:108360005D62DD489862DF62DC4C1C635F639F6383
:10837000DB49DA6B8869A24201D3824201D9D94A2A
:10838000DA631A6CA24201D3824201D9D64A1A6436
:108390005A6CA24201D3824201D9D44A5A649A6CDF
:1083A000A24201D3824201D9D14A9A64DA6CA24234
:1083B00001D3824201D9CF4ADA641A6DA24201D3B5
:1083C000824201D9CC4A1A655A6DA24201D3824237
:1083D00001D9CA4A5A659A6DA24201D3824201D993
:1083E000C74A9A65DA6DA24201D3824201D9C54AD1
:1083F000DA651A6EA24201D3824201D9C24A1A66D4
:108400005A6EA24201D3824201D9C04A5A669A6E7C
:10841000A24201D3824201D9BD4A9A66DA6EA242D3
:1084200001D3824201D9BB4ADA661A6FA24201D354
:10843000824201D9B84A1A675A6FA24201D38242D6
:1084400001D9B64A5A679A6FB54EA24201D3824209
:1084500000D99E67DD67A24840380560C8224260A7
:1084600064228260C760076147618761C7610762F4
:1084700047628262AB4AC262FF2202634263826346
:10848000C7630D604F608F60CF600F614F618E6179
:10849000CF610F62984848628F620C63A2484863BC
:1084A000FCF7FCFDF8BDF8B50120F8F71DFD002331
:1084B0009EA219460120F8F7DAFB012100239EA2B3
:1084C0000846F8F7D4FB00239EA202210120F8F70A
:1084D000CEFB00239EA203210120F8F7C8FB052351
:1084E0009EA204210A20F8F7C2FB05239CA20421C6
:1084F0002C20F8F7BCFB9B48062300900422194669
:108500000020F8F793FB98480090062304224021AE
:108510003A20F8F78BFB0621022001F09DFE002691
:10852000924D0127924C00280ED027710F21012077
:1085300001F092FE002822D06771AF20F8F7D0FC3E
:108540000020F8F7D1FCF8BD20790028EED0267184
:10855000884800900623042240213A20F8F766FB61
:108560008548F9F727FEF8F776FC59202860162091
:1085700028608820286001F0E4FB2E60D6E760794F
:108580000028DAD066717D4806230090042219463F
:108590000020F8F74BFBFFF7D5FE7748F9F70AFE06
:1085A000F8F759FC59202860162028608820286098
:1085B00001F0C7FB2E60C0E708B50120F8F794FC76
:1085C000FF20F8F777FCAE20F8F78AFCF8F743FCB9
:1085D0006B4800900423022240210020F8F726FB7C
:1085E000AF20F8F77DFC6448F9F7E4FDAE20F8F71A
:1085F00077FCF8F730FC0020F8F776FC08BD08B5EA
:108600000120F8F771FCFF20F8F754FCAE20F8F7D2
:1086100067FCF8F720FC5B4800900423022240210D
:108620000020F8F703FBAF20F8F75AFC7D2000018B
:10863000F9F7C0FD0020F8F757FC08BD08B5012088
:10864000F8F752FCFF20F8F735FCAE20F8F748FCAD
:10865000F8F701FC4C48009004230222402100203E
:10866000F8F7E4FAAF20F8F73BFC4348F9F7A2FD2E
:10867000AE20F8F735FCF8F7EEFB0020F8F734FCF5
:1086800008BD08B500F058FC00280AD000F022FC14
:10869000002806D100F037FC002802D10820F9F7A5
:1086A000F5FF0120F8F720FCFF20F8F703FCAE20CF
:1086B000F8F716FCF8F7CFFB344869E05455524EF2
:1086C0000A000000204F46460A000000204F4E20BE
:1086D0000A0000003C0B0020A00F000070170000F3
:1086E000FC0B002010270000204E00003075000019
:1086F000409C000050C3000060EA000070110100BF
:1087000080380100905F0100A0860100B0AD01003B
:10871000C0D40100D0FB0100E0220200F0490200B9
:1087200000710200C0270900AC0D00002052455323
:10873000544F5245200A000020464143544F52599D
:10874000200A00002044454641554C54200A0000B0
:1087500053455454494E47532E0A0000590A00000D
:108760004E0A00007CDB000088DB000000010050A6
:10877000CC010020A0DB0000DC05000094DB000041
:108780005ACB00005ACA0000DACA00005ACD0000D5
:1087900000900323012240210020F8F747FA00232C
:1087A000FFA204211F20F8F762FA0023FDA2042192
:1087B0001420F8F75CFA0023FBA204211B20F8F731
:1087C00056FA0023F9A204212420F8F750FA0023D6
:1087D000F7A204212B20F8F74AFAAF20F8F780FB24
:1087E000F448F9F7E7FCAE20F8F77AFBF8F733FB2B
:1087F0000020F8F779FB08BDF8B53720F9F7ACFA97
:1088000000250126EC4C00280CD1FF21F531372042
:10881000F9F79EFAA079002801D0A57100E0A671B1
:10882000F8F719FBA079002829D0E079002825D095
:10883000E5710120F8F758FBE0480090032301227E
:1088400030211020F8F7F2F9DD48009006230322CA
:1088500014210020F8F7EAF90023DA4A0321202046
:10886000F8F705FA0023D8A204211C20F8F7FFF935
:10887000AF20F8F735FB0020F8F736FBF8BDE079BC
:108880000028FBD1E671F8F7E6FAF8BDF8B5D04854
:10889000C94EC068CF490025203E884203D9B5742F
:1088A000FFF7AAFFF8BDB07C002803D10120B07407
:1088B000F8F7D1FAF9F7BCFF032802D03079012884
:1088C00017D00E20F9F748FAC34F3946C03100914E
:1088D00000287ED00120F074F9F7AAFFBE4C0300F7
:1088E000803404F09EF809B8F3ECF1F0EFECEEED13
:1088F000EC000120F8F7F8FA0023B8A2194601208D
:10890000F8F7B5F901210023B7A20846F8F7AFF947
:108910000023B8A202210120F8F7A9F90023B8A288
:1089200003210120F8F7A3F90023B8A204210120B4
:10893000F8F79DF90023ACA205210120F8F797F97B
:10894000AF20F8F7CDFA0020F8F7CEFA00F0F4FAED
:10895000002805D07D21C9002E20F9F7F9F9F8BDCE
:108960002E20F9F7F9F90028F9D10120F8F7BCFA1F
:108970000023A9A219460120F8F779F90121002363
:1089800099A20846F8F773F90023A6A20221012054
:10899000F8F76DF90023A6A203210120F8F767F983
:1089A0000023A6A204210120F8F761F900238EA27A
:1089B00005210120F8F75BF9AF20F8F791FA0020C4
:1089C000F8F792FAA04C59202060162020608820E9
:1089D00000E004E0206001F0B4F92560F8BDF9F78B
:1089E00027FF052800D077E7F07C00282FD0F5740A
:1089F000FBF7D2FE002828D100984068C0B2F7F7F4
:108A0000FAFFF9F7AAFF00280FD1F9F714FF401C6D
:108A1000FDF77DFC0E20F9F79FF98C49091A386A99
:108A2000081838620120F8F70EFE00211120F9F72E
:108A30008FF900211220F9F78BF900211320F9F7A3
:108A400087F900211420F9F783F9F8F704FA0720D1
:108A5000F9F71CFE40E70120F8F742FA0121022055
:108A600001F007FC0321022001F003FC0221012098
:108A700001F0FFFB0721022001F0E0FBF9F7BEFE49
:108A80000120F9F7B2FEF9F704FE01280AD1FFF739
:108A9000B6FDFFF7F6FDFFF7D1FDF8F7DCF907208B
:108AA000F9F7F4FDF9F7F5FD002808D1FFF7A7FD68
:108AB000FFF782FDF8F7CFF90820F9F7E7FDB8E1F5
:108AC00098E1FDE0D1E04CE02EE0FFE70120F8F76F
:108AD00007FAF8F751FA0121022001F0CAFB03213D
:108AE000022001F0C6FB0221012001F0C2FB072198
:108AF000022001F0A3FBF9F781FE0120F9F775FED2
:108B0000F7F73FFFFFF7CFFC1620F9F725F900280C
:108B1000D5D14D4C5920206016202060882020603F
:108B200001F00FF9256084E10120F8F7D9F9F8F791
:108B300023FA0121022001F09CFB0321022001F015
:108B400098FB0221012001F094FB0721022001F093
:108B500075FBF9F753FE0120F9F747FEFFF7D2FB4B
:108B600067E10120F8F7BCF9F8F706FA01210220C5
:108B700001F07FFB0321022001F07BFB0221012099
:108B800001F077FB0721022001F058FBF9F736FED0
:108B90000120F9F72AFEF7F7F4FE162058E000004E
:108BA0002E0A0000560A0000310A0000300A0000B8
:108BB000370A0000DC050000CC010020B6E100000F
:108BC000BAE00000784B0000494E5055540A0000AE
:108BD00028030020282300003C0B0020535445505C
:108BE000313A2020200A00002020202020202020B0
:108BF000200A00004C4F4E4720505245530A0000B7
:108C00005320534D4F4B20544F0A0000444F574EB2
:108C10004C4F41442E0A000053544550323A202014
:108C2000200A0000434C49434B205448450A0000A9
:108C3000444F574E4C4F4144200A00004255545473
:108C40004F4E2E20200A000000010050442F00004B
:108C5000F9F782F8002802D10820F9F717FDF86823
:108C6000012801D1FCF731F9E3E00120F8F738F9E8
:108C7000FF20F8F71FF9F8F77FF90321022001F030
:108C8000DDFA0221012001F0D9FA0721022001F0CA
:108C9000D5FA3575FBF78BFAF86801280DD02069F5
:108CA000A0616D49884200D3A5617D21C9002F20B4
:108CB000F9F74EF8FBF773FDBBE0FCF7E2F8F4E7D9
:108CC0000120F8F70DF91620F9F746F80099624AE5
:108CD000496AD2438918884203D20020F8F7EAF89B
:108CE00002E06420F8F7E6F8F8F746F902210120DF
:108CF00001F0BFFAF9F782FD5848816810229143CC
:108D000081600221084601F0B4FA0120F9F76DFDF7
:108D10006561FD627D630020FBF7C9FAE561306B98
:108D2000002804D0401E3063F9F713F903E0012155
:108D3000022001F09EFA2A20F9F70EF8002802D14D
:108D40004748C0686062786A002809D0F8F711F9CE
:108D500001280CD01620F8F7FFFF002815D017E0E7
:108D60000020F9F793FC0020FBF79EFA61E0E06A2F
:108D700000280DD01920F8F7EFFF002808D1F8F7E8
:108D8000F2F80820F9F782FC02E00820F9F77EFCEF
:108D90001620F8F7E1FF00281CD0307D00280CD009
:108DA0003575FF2191310F20F8F7D2FFFF21F53102
:108DB0002820F8F7CDFFF8F74EF80321022001F044
:108DC0003DFAFBF75BFAF9F7D1FD00212D20F8F70A
:108DD000BFFF2EE00120F8F787F8AE20F8F780F803
:108DE0000321022001F045FA0020F8F779F801206C
:108DF00030751EE00020F8F773F8F9F7FFFC01204A
:108E0000F9F7F3FC1648C06860626561FD627D6336
:108E100000F092F8002805D01020F8F79DFF0028F8
:108E200005D006E00F491020F8F792FF01E0F9F7AE
:108E300033FC0020F8F758F8F8BD0B48806A7047FB
:108E40000A49C87170470849803948617047064926
:108E500040314861704700000F27000080400050FB
:108E600028030020DC050000BC0B0020AC01002022
:108E700070477047704710B5FF4C5920206016208E
:108E800020608820206003220621022001F0ACF936
:108E900003220F21012001F0A7F90322114600202F
:108EA00001F0A2F9022200230621104601F0F5F993
:108EB000F24A0021022001F050FA0023022203218D
:108EC000184601F0EAF9EE49EE4801F042FA0020B6
:108ED000206010BD10B5EC488069002807D001283B
:108EE0000BD00621022001F0B7F9C0B210BD062157
:108EF000022001F0B1F9C0B210BD0F21012001F034
:108F0000ABF9C0B210BD10B5DF488069002807D0AA
:108F100001280BD00F21012001F09EF9C0B210BD35
:108F20000F21012001F098F9C0B210BD06210220E6
:108F300001F092F9C0B210BD10B50321002001F07C
:108F40008BF9C0B210BDD14908627047CF49C861E2
:108F50007047CE4948717047CC49C8707047CB48BC
:108F600000787047C94948707047F8B5F9F791FB28
:108F7000002870D00020FCF79EF80120F7F7B4FF1E
:108F80000120FFF7EFFF0120FFF7E6FFF9F750FCA4
:108F9000072832D1F9F7E1FC00282ED1FFF7DCFFDA
:108FA000B94D00246C60E868002804D0012837D04F
:108FB000022822D160E03020F8F7CEFE00281CD134
:108FC00028213020F8F7C4FE0720F8F7C5FEAE4C84
:108FD0007D27FF00C034002806D12E6B394630466D
:108FE00003F094FC002909D0A949286B88420FD3CB
:108FF000A16988420AD2C019286364E0A069864248
:1090000002D2F01928635EE028635CE029635AE02D
:10901000A169884202D26430286354E0296352E097
:109020003120F8F799FE00284DD164213120F8F75E
:109030008FFE9548E96F01228030002903D0012975
:109040000ED0EA673FE0FF2381683C33994203D2A8
:10905000491D816037E062E0EA67C821416032E083
:109060004B224168D200914202D20A3141602AE08B
:10907000EC676421816026E03220F8F76DFE00285D
:1090800021D128213220F8F763FE19214901072058
:10909000F8F75EFEFF202D30FFF758FF002111206A
:1090A000F8F756FE00211220F8F752FE0021132097
:1090B000F8F74EFE00211420F8F74AFEA86B0F289F
:1090C00001D2401CA863F9F7B3FB032827D1FFF7AF
:1090D00046FF002823D1FFF73FFF0120F7F704FFE9
:1090E0000120FFF736FF1924640121460720F8F715
:1090F0002FFE21460820F8F72BFEFF222D321046C6
:10910000FFF724FF1046FFF71EFFFFF7F7F80528CB
:1091100006D2FFF7F3F8401CC0B2FBF7B6FFF8BD6C
:109120000020FBF7B2FFF8BDF8B5F9F7B2FA002856
:1091300074D00120FBF7BFFF0120F7F7D5FE012017
:10914000FFF710FF0120FFF707FFF9F771FB072872
:1091500030D1F9F702FC00282CD1FFF7FDFE4A4C74
:1091600000256560E068002804D0012833D002287B
:1091700020D158E03020F8F7EFFD00287AD12821DF
:109180003020F8F7E5FD0820F8F7E6FD7D27FF0021
:10919000404E002806D1256B3946284603F0B6FB21
:1091A000002908D03C49206B88420DD3B04209D930
:1091B000C01B20635EE0B54202D9E81B206359E082
:1091C000266357E0266355E0B04202D96438206335
:1091D00050E026634EE03120F8F7BEFD002849D16B
:1091E00064213120F8F7B4FD2748E16F0122803077
:1091F000002903D001290BD0E2673BE08168642994
:1092000002D9491F816035E0E2672449416031E0BD
:109210004168C82903D90A3941602BE06EE0E5674F
:109220001F49816026E03220F8F796FD002821D101
:1092300028213220F8F78CFD192149010820F8F780
:1092400087FDFF202D30FFF77EFE00211120F8F76B
:109250007FFD00211220F8F77BFD00211320F8F795
:1092600077FD00211420F8F773FDA06B002801D0D2
:10927000401EA06316E0000000010050758E000043
:10928000738E0000718E00003C0B00202002002035
:10929000A086010070170000888A010058020000B3
:1092A0003B010000F9F7C4FA032827D1FFF757FE66
:1092B000002823D1FFF750FE0120F7F715FE01200B
:1092C000FFF747FE1924640121460720F8F740FD07
:1092D00021460820F8F73CFDFF222D321046FFF70B
:1092E00035FE1046FFF72FFEFFF708F8002806D0DE
:1092F000FFF704F8401EC0B2FBF7C7FEF8BD05201B
:10930000FBF7C3FEF8BDF94908717047F7490870CB
:109310007047F64800797047F44988707047F8B58F
:10932000FFF7D8FDF24F002639468031C0370125BE
:10933000EE4C009100280AD0192149010720F8F7C6
:1093400007FD3B20F8F708FD00284DD142E0FFF76C
:10935000DAFD002836D0A07A002834D0A671257214
:1093600000211220F8F7F4FC1620796AF8F7F0FCD7
:109370000098C16A1920F8F7EBFCDE490C20F8F7D9
:10938000E7FC3520F8F7E8FC002803D1C821352098
:10939000F8F7DEFC0720F8F7DFFC002813D10920DE
:1093A000F8F7DAFC00280ED1E0690A2802D90A3859
:1093B000E06100E0E6610920E169F8F7C9FCFFF728
:1093C000D4FD00E0A6720720F8F7C6FC002823D1E0
:1093D000A57121E03C20F8F7BFFC002804D11E2035
:1093E000F8F7BAFC002800D0A571A07900280AD1AE
:1093F000A57100211220F8F7ABFC00213520F8F709
:10940000A7FCFFF7B2FD207A002802D02672FBF7F6
:1094100045FEB948E061A572FFF775FD00280AD046
:10942000192149010820F8F793FC3B20F8F794FC38
:1094300000284DD142E0FFF74DFD002836D0E07AFC
:10944000002834D0E671657200211220F8F780FC04
:109450001620796AF8F77CFC0098C16A1920F8F7A1
:1094600077FCA4490C20F8F773FC3620F8F774FC5D
:10947000002803D1C8213620F8F76AFC0820F8F745
:109480006BFC002813D10A20F8F766FC00280ED1E7
:10949000206A0A2802D90A38206200E026620A20DF
:1094A000216AF8F755FCFFF73FFE00E0E67208205E
:1094B000F8F752FC002823D1E57121E03C20F8F7B1
:1094C0004BFC002804D11E20F8F746FC002800D0F1
:1094D000E571E07900280AD1E57100211220F8F742
:1094E00037FC00213620F8F733FCFFF71DFE607AC9
:1094F000002802D06672FBF7D1FD7F482062E5723A
:10950000FFF71AFD002805D03820F8F725FC0028C1
:109510007ED0ADE077490C20F8F71AFCFF2191319D
:109520000620F8F715FC1620796AF8F711FC009868
:10953000C16A1920F8F70CFC6F490520F8F708FC00
:1095400064213820F8F704FCA5742573E573F9F756
:109550006FF903281CD100210520F8F7F9FB0B2037
:10956000F8F7FAFB002813D17D21C9000B20F8F78A
:10957000EFFBFFF7F4FC401CC0B2FFF7C7FE2574F9
:109580000120FFF7EFFC0120F7F7AEFCF7F763FCD3
:10959000F9F77FF801283FD10D20F8F7DDFB00280F
:1095A000F9D16673F9F744F9032835D0F9F740F992
:1095B000072827D13D20F8F7CFFB002822D105202E
:1095C000F9F764F8F9F7C9F900280FD1607C002891
:1095D0000CD066740020F8F7BCFC7868C0B2F7F7CE
:1095E000B4F97D2109013420F8F7B2FBF9F7B5F998
:1095F000012807D1E07C002804D0E6743E49012010
:10960000F7F739F9A07B0028C5D1A5733B4900E0E5
:1096100003E00E20F8F79CFB2CE1E07B002827D02C
:10962000E673F9F736F8012822D1F9F701F9052890
:109630001ED10720F9F72AF80120F7F755FCFBF7B0
:10964000ABF8002814D1F9F788F9002810D1F9F700
:10965000F2F8401CFCF75BFE0E20F8F77DFB274973
:10966000091A2348026A891801620120F7F7EBFF03
:10967000F9F7DEF80528CFD0207B002803D0267329
:10968000607B401C60730520F8F766FB002871D1F1
:10969000607B04280DD3F8F7FCFF002809D166731E
:1096A0000120F7F721FC0120FAF7FEFD0020F8F772
:1096B000EDFF607B052813D3F8F7EBFF01280FD1EE
:1096C00066730020FFF7BCFB192149011720F8F74A
:1096D0003FFBF9F742F9012812D00120FFF7B3FB55
:1096E000607B032810D004280ED027E02002002041
:1096F0003C0B0020881300002C010000442F0000C8
:109700000020FFF7A0FBEBE7F8F7C3FF012815D116
:10971000FFF7FFFD002811D166730120F7F7E4FB86
:10972000F7F799FB0120FFF714FC0020FFF7EEFD8F
:109730000320F8F7ABFF0120FFF7E5FD607B012870
:1097400034D1F8F7A6FF012830D1FFF7E2FD012858
:109750002CD16673F7F7C8FB0120FFF7FAFB032053
:10976000F8F794FFFFF7FBFB002804D0207C0028CB
:109770000FD01AE01BE0FEF7C1FD401CC0B2FBF7A2
:1097800084FCFEF7BBFD052810D90020FBF77DFC0B
:109790000CE00120F7F7A8FB0120FFF7BDFD012039
:1097A000FFF7E0FB0020FBF786FC267466730620BB
:1097B000F8F7D2FA002800D16673F8F76AFF01289B
:1097C0001AD1FFF7A6FD012816D10C20F8F7C4FA2C
:1097D000002811D1FFF7C3FB401CC0B2FFF796FD74
:1097E000FB490C20F8F7B4FA0120F7F77DFBF7F7F7
:1097F00032FB0120FFF7B6FBE07C002800D1E574C6
:10980000607C002807D1A07C002804D0A67478686A
:10981000C0B2F7F7F0F8FAF7BFFF002819D000211F
:109820001120F8F795FA00211220F8F791FA00219B
:109830001320F8F78DFA00211420F8F789FAF7F7CA
:10984000A0F80120F7F750FBF7F705FB0020FAF727
:1098500077FFFF2191310B20F8F77AFAFF21913140
:109860000D20F8F775FAA6736574DA48816810223E
:1098700091438160F9F771F801287AD1FFF75CFB19
:10988000002807D1FFF726FB002803D0FFF73BFB9A
:10989000002803D0207D00281AD01AE02720F8F7EE
:1098A0005BFA002815D1207D002812D02675F9F723
:1098B00058F8012808D00120FDF72EFA4B210901A4
:1098C0002720F8F745FA04E00020FDF725FAF5E730
:1098D0002575FFF731FB00281CD1FFF7FBFA0028A4
:1098E00018D1FFF710FB002814D03E20F8F734FA07
:1098F000002813D1607D002810D06675B86A002852
:1099000006D0BE624B2109013E20F8F721FA05E09E
:10991000BD62F7E7607D002800D16575FFF70CFB9D
:10992000002807D0FFF7D6FA002803D1FFF7EBFA9B
:10993000002803D0A07D00280AD00AE0A07D0028DE
:1099400000D0A6754B2109013F20F8F701FA00E08D
:10995000A575FFF7F1FA002807D0FFF7BBFA00283A
:1099600003D0FFF7D0FA002804D0E07D002810D003
:1099700010E064E0E07D002800D0E6754020F8F7B4
:10998000EBF900280BD1FF21F5313920F8F7E0F988
:1099900005E0E575FF21F5314020F8F7D9F9FFF72B
:1099A000CBFA002816D0FFF795FA002812D1FFF75E
:1099B000AAFA00280ED0207E002800D0267641206A
:1099C000F8F7CAF900280ED1FF21F5313A20F8F74F
:1099D000BFF908E0207E002800D12576FF21F5316F
:1099E0004120F8F7B5F9FFF7A7FA002828D1FFF7CB
:1099F00071FA002824D0FFF786FA002820D0F8F763
:109A000017FF032820D00D20F8F7A6F9002804D16D
:109A1000FF2191311820F8F79BF94420F8F79CF9C1
:109A2000002811D16A494420F8F792F90320F8F789
:109A30002DFE0120FFF767FC0520FBF726FB03E066
:109A400063494420F8F784F9F8F7F2FE05287DD041
:109A5000F8F783FF002879D1FFF76EFA002807D1C5
:109A6000FFF738FA002803D0FFF74DFA002803D09B
:109A7000607E002839D039E03B20F8F76DF90028E6
:109A80001DD1607E00281AD06676F869022200286F
:109A900004D15149CB68002B03D0CE60012802D0FD
:109AA00008E0CA60FAE74C49C868002819D00128C4
:109AB00019D0CE604B2109013B20F8F749F9192153
:109AC00049010D20F8F744F91927BF01394607204D
:109AD000F8F73EF939460820F8F73AF9A571E5712B
:109AE00004E0CD60E6E7CA60E4E76576FFF724FAB4
:109AF000002831D1FFF7EEF900282DD1FFF703FA46
:109B0000002829D03C20F8F727F9002810D1A07EA2
:109B100000280DD0A67630490869052802D2401CDD
:109B2000086100E00D614B2109013C20F8F710F9B4
:109B3000192149010D20F8F70BF91927BF01394602
:109B40000720F8F705F93946082000E018E0F8F793
:109B5000FFF8A571E57103E0A07E002800D1A5768D
:109B6000FFF7EAF9002807D0FFF7B4F9002803D17E
:109B7000FFF7C9F9002804D0E07E002800D1E5767F
:109B8000F8BD1E20F8F7E8F800280FD1E07E002885
:109B90000CD0E676F7F7EDF901281FD00120F7F792
:109BA000E2F94B2109011E20F8F7D2F819214901E9
:109BB0000D20F8F7CDF81926B60131460720F8F741
:109BC000C7F831460820F8F7C3F8A571E571F8BD6C
:109BD00088130000804000503C0B00200020F7F765
:109BE000C2F9DEE70548407970470448407870477D
:109BF0000248807870470148C078704720020020F2
:109C000070B506460D4600241948864201D9002049
:109C100070BD7D21801BC9004843164902F076FEC5
:109C200001461548704302F071FE1449A2008A589B
:109C3000824204D8621E92008A58824202D8641C72
:109C40007A2CF3D30E49884200D30024002D03D090
:109C5000012D03D0002070BD204670BDE1212046BB
:109C6000C9004843044902F051FE203070BD000095
:109C7000CC0B000010270000E8030000CCEB000034
:109C800092810000F0B5A1B000241E4E5920306032
:109C9000162030608820306020221B4901A8F8F788
:109CA000B6FA01AF1948A50040591949C04302F05E
:109CB0002DFE795988421DD00120F7F715F9F7F7E5
:109CC000CAF8002313A219461846F6F7D0FF00235E
:109CD00013A202211846F6F7CAFF002313A203219C
:109CE0001846F6F7C4FFAF20F7F7FAF80020F7F7A9
:109CF000FBF8FEE7641CE4B2202CD3D300203060D4
:109D000021B0F0BD0001005000FF0100B4ED0000E3
:109D1000431267004552524F523A2020200A000059
:109D20004E4F205345435245540A00002D4B455990
:109D300021202020200A0000EF480068C007C00F43
:109D40007047052000078168012211438160704738
:109D5000052000078169102211438161E7480068EE
:109D6000002800D00047704710B5072802D8011F0F
:109D7000032901D2E24810BDE2490A694007D2082E
:109D8000D200400F02430A61F6F7B2F9002010BD7D
:109D9000F0B58C07A40F4D070C27DA4AA6006D0F0B
:109DA000030002F03EFE0D5F5A524A423A3128212A
:109DB0000D081A136600D069B8433043D06156E0ED
:109DC000D069800880002043D06150E0D069C02174
:109DD0008843A1010843D06149E0D069302188431C
:109DE00021010843D06142E0506980008008890762
:109DF000084350613BE0506903231B0789079843E0
:109E000089080843506132E0506903231B06890723
:109E1000984389090843506129E0506907210905E1
:109E2000884329050843506121E05069072109044E
:109E3000884329040843506119E050690721090348
:109E4000884329030843506111E050690721090242
:109E5000884329020843506109E05069B843304300
:109E6000506104E050698008800020435061002068
:109E7000F0BDA348401CF0BDA24A002807D001282D
:109E80000DD0022813D0032819D09D4870471068C0
:109E9000C90740084000C90F0843106016E0106869
:109EA0000223C9079843890F084310600EE0106829
:109EB0000423C9079843490F0843106006E010685F
:109EC0000823C9079843090F084310600020704712
:109ED0008C4801684022114301608848406800288E
:109EE00000D00047704710B586490B688022934325
:109EF0000B600B685400C007A343C00D03430B6005
:109F000008681043086010BD7F487047F8B50246E6
:109F100008467D4E7D497E4B4118994201D8002567
:109F20000FE07C497C4B4118994202D80125400042
:109F300007E07A49794B41185B42994206D80325DC
:109F40008000002A05D0012A02D002E07448F8BD42
:109F5000744E754F394602F0D9FC044639463046F6
:109F600002F0D4FCC107C90FE207D20F114306D19A
:109F7000022804D0022C02D040086408F2E7801EB8
:109F8000A90340020143A41E21430846F8BD5D49D0
:109F90000A6AC305520A5202DB0D1A430A620A6AB0
:109FA0001F235B029A438304DB0E5B021A430A629F
:109FB0000A6A03239B030004800F9A438003024331
:109FC0000A6270471FB5002058494C680B688A68C0
:109FD000C96801940093029203914A4C216A0903D3
:109FE00001D5504A00E0484A216AC90312D4206AC8
:109FF0008004C10E206A891CC005C00D801C50431E
:10A0000002F084FC216A6A460904890F89005158CC
:10A0100002F07CFC04B010BD10B53A4C206940073A
:10A0200016D020694007400F012813D0206940074F
:10A03000400F022810D020694007400F03280ED09F
:10A040003848A1690907090F491C02F05FFC10BDDF
:10A050002D48F6E73648F4E7FFF7B4FFF1E7354857
:10A06000EFE770B5014600222C48334B08189842A0
:10A0700002D32348C01C70BDFFF75EFE002808D045
:10A08000204D286A000307D428680123184328605C
:10A0900007E01B48001D70BD28680422104328609B
:10A0A00001221046FFF732FF0021224C00E0491C3C
:10A0B000A142FCD3FFF76BFF286A01218904884382
:10A0C0002862286A891088432862002000E0401C2A
:10A0D000A042FCD30220FFF747FE002070BD1749C5
:10A0E00009684843164948610020886105200861D5
:10A0F0000869C003FCD570470001005044020020ED
:10A100000396FFFF00020050001BB700FF1E0AFA73
:10A11000FFE0F5057F0F05FD7FF0FA02C08782FEA4
:10A120002EC200000080510140420F0034EE0000BA
:10A13000008000001027000041787D01040000200D
:10A1400000E000E08307FF22DB0E9A408907090E3A
:10A15000994000280BDA0007000F08388308FA48F6
:10A160009B001818C36993430B43C361704783086E
:10A17000F6489B001818036893430B43036070472D
:10A1800030B4F34A106AF34B196AF34CA1431062DE
:10A190001962F24A1268002A01D030BC104730BC64
:10A1A000704730B4EE4B186AEE4C216AEE4D2A6AC5
:10A1B000186221622A62E94B5B68002BEFD030BC49
:10A1C0001847ECE7E349E9480862E448806800285A
:10A1D00000D000477047DF49E5480862DF48C068A3
:10A1E000002800D00047704710B50346E148112908
:10A1F00011D2D74C9B011B19032449008C40002A23
:10A200000AD0012A08D0022A06D0032A03D11868EE
:10A2100020431860002010BD1868A0431860012A70
:10A2200006D0022AF6D118688A4010431860F1E778
:10A23000186801228A4010431860EBE7112901D306
:10A24000CC487047C24A80018018826801238B4045
:10A250001A43826000207047112901D3C548704716
:10A26000BB4A8001103280180068C840C007C00F88
:10A270007047112901D3BF487047B54A8001801843
:10A28000826801238B409A43826000207047B04A65
:10A2900080018018816000207047F8B50446022ACA
:10A2A00001D1012B02D0012C02D005E0B148F8BD4C
:10A2B0000E2914D00F2912D0A54DA00184461C35BB
:10A2C00040190D46012610353746AF408E40002A12
:10A2D00007D0012A09D0022A0BD0A648F8BDA5480C
:10A2E000F8BD01683943016008E00168314301604D
:10A2F00004E03146026839431143016094496046E5
:10A3000018314018002B03D0012B05D09948F8BD17
:10A310000168B143016002E0016831430160002C33
:10A3200001D0012C06D102210420FFF70BFF0420ED
:10A3300000F0A3FA022C03D0032C01D0042C06D188
:10A3400002210520FFF7FEFE052000F096FA00200E
:10A35000F8BD824A10605160704770B5022801D183
:10A3600001292CD0844B824C002804D0012808D02D
:10A3700002280AD00DE018680125ED07284318606F
:10A3800007E018682043186003E018687B4D2843F5
:10A3900018607B48002902D0012904D006E001683A
:10A3A000A143016002E00168214301606B48C26083
:10A3B00002210320FFF7C6FE032000F05EFA70BD05
:10A3C000F0B501240146283927468F4005210F2585
:10A3D000032609076B4A030002F023FB3E202735C2
:10A3E0003B465358586770797E8993999DAAAFF080
:10A3F000FAEDECEBEAE9E9E9E9E9E9E8E7E6E5E4C1
:10A40000E3E2E1E0DFDEDDDDDDDDDDDDDCDBDAD971
:10A41000D8DBDBDADAD9D9D8D8D7D6B500200863AB
:10A4200048638863C863106023E2486B01231B0301
:10A430001843486310699910084310611069490076
:10A440008843106115E2086B03221202104308636F
:10A450000FE2086B03239B02184308631069012174
:10A46000C9028843106104E2886B28438863086B43
:10A470003F4B1843086310691F21490108431061CD
:10A48000F7E1C86BC0221043C863F2E106280AD086
:10A490000E208B6B864033438B6310690121C90208
:10A4A00088431061E5E10620F3E7886B2843886361
:10A4B0001069FF21E13188431061DAE1486B012323
:10A4C0009B0218434863106920431061D1E1886BF7
:10A4D000302210438863CCE1886B0F231B021843A2
:10A4E000886310690121C90288431061C1E1486B8A
:10A4F00001235B0218434863116902200143116183
:10A50000B7E1886B0322120310438863B1E1C86B83
:10A510002843C863ADE1086B8023184308631069C2
:10A520000421084310611069490288431061A0E1C9
:10A53000C86B30221043C8639BE1CA6B0F20000236
:10A540000243CA6395E196E100ED00E000E400E01B
:10A55000004000504040005000C000004C0200206D
:10A5600080400050C04000500041005000400000BA
:10A57000008000000189FFFF5C40005000800080E7
:10A58000584000504000005031E141E11EE1FCE044
:10A59000D9E0C7E0C0E091E087E07DE073E068E0EB
:10A5A0005DE052E047E040E039E034E024E027E0BD
:10A5B0002BE01CE016E011E00AE0FFE7486B012306
:10A5C0009B0318434863116908200143116150E15E
:10A5D000C86B032212031043C8634AE1886B284307
:10A5E000886346E1CA6B02200243CA6341E1CA6B39
:10A5F00004200243CA633CE113690425AB431361A1
:10A6000013690125ED02AB4313610A6B17388440CF
:10A6100022430A632DE113690825AB4313614A6B9A
:10A620001138844022434A6323E1486BFF22013200
:10A63000104348631DE1486B01235B0218434863E4
:10A64000116902208143116113E14B6B01208002EB
:10A6500003434B63106940084000106109E1486BF7
:10A660000123DB0218434863116910208143116103
:10A67000FFE0486B0123DB0318434863106959026C
:10A6800008431061F5E0106820210843106010694C
:10A69000090508431061ECE0486B04231843486344
:10A6A0001069190608431061E3E0486B082318435A
:10A6B00048631069190608431061DAE00346293B34
:10A6C000022B01D8002300E0042329280AD02C28DB
:10A6D00008D02A2810D02D280ED02B2811D02E28B3
:10A6E0000FD0C6E0486B9D402843486310690121A4
:10A6F000C90288431061BCE0486B9E403043486308
:10A70000B7E0486B9B1C9E403043486310690121B1
:10A71000C90288431061ACE0C86B03229203104366
:10A72000C863A6E0302808D0086B38430863106976
:10A730000121C902884310619BE0086B03231B03BE
:10A7400018430863F3E731280AD00B6B3B430B63D4
:10A75000362814D01169012040028143116188E03C
:10A76000086B03239B031843086310690121490206
:10A7700088431061106989008843106179E010698D
:10A780000121C9028843106173E0322806D03828BD
:10A7900012D011682020014311606AE0486B012348
:10A7A000DB021843486310691021084310611068E8
:10A7B0002021084310605CE0486B0123DB02184352
:10A7C0004863106910210843106152E0332806D015
:10A7D0003A2808D0106802210843106049E0106848
:10A7E0003043106045E010682043106041E04B6B3F
:10A7F0000C2423434B631369E402234313610B6B63
:10A80000214C23430B631369FF2424042343136166
:10A810003C2811D1486B0C23984348631069DB0234
:10A8200098431061086B184BDB43184008631069AC
:10A83000FF231B049843106110690323DB021843B4
:10A840001061886BFF22013210438863086B5A1035
:10A85000104308634A6BC02002434A630A6B0243F9
:10A860000A63886B094A10438863486B5A00104397
:10A8700048630020F0BD0648F0BDC106C90E0120A6
:10A8800088400449086070473E700000C0C0000066
:10A890000189FFFF00E100E0F0B505242407E56829
:10A8A000012636073543E560E568B543E5606B4C46
:10A8B00067690C259B07AF431B0F1F436761A369A3
:10A8C000FF273F04BB43059F3F043B43A361A368AD
:10A8D0003343A360624B1C6A012634431C621C157F
:10A8E00000280FD0186A2043186200290ED00129D1
:10A8F00010D0186A28431862586A000A00021043F0
:10A900005862F0BD186AA0431862EEE7186AA843BF
:10A910001862F1E7186AA84308301862ECE750485B
:10A92000016A4908490001624C498A68CB049A438C
:10A930008A60026A02218A4302624B4B494A1A60CA
:10A94000826A520852008262826A8A438262C26AC2
:10A9500052085200C262C26A8A43C26270474049CA
:10A960004A6A120A120202434A6270473C490A15B7
:10A97000002803D0086A104308627047086A9043B1
:10A980000862704736490C22002805D0012807D0FC
:10A99000086A104308627047086A9043086270476B
:10A9A000086A904308300862704770B52C4C206BE1
:10A9B0002E4E2F4DC00709D02968002901D03068DC
:10A9C0008847206BC008C000401C2063206B8007B4
:10A9D00009D56968002901D070688847206BC008D4
:10A9E000C000801C2063206B400709D5A96800299E
:10A9F00001D0B0688847206BC008C000001D2063EC
:10AA000070BD1748016BC908C900491C0163016A80
:10AA10000122D2021143016270471148006BC00746
:10AA200001D001207047002070470D490A6A80005C
:10AA300052054018002A03DB00680005000D70472E
:10AA4000096A002902DB006880B27047006880B2A2
:10AA50000104FAD501210904401A70470002005090
:10AA600000000E400000002080E100E04C0C0020BF
:10AA70005C020020F8B5F54D6C68F54EE00705D096
:10AA8000012068603068002800D08047A00705D505
:10AA900002206860B068002800D08047600705D5B4
:10AAA000042068603069002800D08047200705D561
:10AAB00008206860B069002800D080472C696F6961
:10AAC000E00611D5E3480068002804D02869E2496F
:10AAD0000840286104E028690121090588432861AC
:10AAE0007068002800D08047E002DC4C0FD5D948C0
:10AAF0000068002803D028692040286103E0286905
:10AB0000102188432861F068002800D08047F806AB
:10AB100011D5D0480068002804D06869CE490840A3
:10AB2000686104E06869012109058843686170690A
:10AB3000002800D08047F8020FD5C64800680028DA
:10AB400003D068692040686103E06969102081438F
:10AB50006961F069002800D08047F8BDF8B5C04DA4
:10AB60006C68C04EE00705D001206860306800289E
:10AB700000D08047A00705D502206860B068002893
:10AB800000D08047600705D5042068603069002840
:10AB900000D08047200705D508206860B0690028EC
:10ABA00000D080472C696F69E00611D5A94800687C
:10ABB000002804D02869A8490840286104E02869D1
:10ABC00001210905884328617068002800D080476A
:10ABD000E002A24C0FD59F480068002803D02869E6
:10ABE0002040286103E02869102188432861F0682B
:10ABF000002800D08047F80611D596480068002844
:10AC000004D0686994490840686104E068690121DA
:10AC10000905884368617069002800D08047F80200
:10AC20000FD58C480068002803D06869204068610F
:10AC300003E06969102081436961F069002800D050
:10AC40008047F8BD884881680F2212051143816052
:10AC500005200007C268032109050A43C260C268D3
:10AC60008A43C260704779490020C86388637C4981
:10AC7000C86388637D484021016080210160052010
:10AC80000007C268032109050A43C260C2688A43FB
:10AC9000C260754881680F22120591438160704738
:10ACA000F0B54207520F0124130001F0BAFE080567
:10ACB000050505111111111D644D403DAB68D20011
:10ACC0009440A343002900D100242343AB600BE050
:10ACD000634D403DAB68121FD2009440A34300294E
:10ACE00000D100242343AB60C10616D559495A4D03
:10ACF0001038564A103D08265D4F594C096803002C
:10AD000001F08FFE080511212D3D4959650B0029E1
:10AD100004D01069284030431061F0BD10693840FC
:10AD200030431061F0BD002906D010690121284090
:10AD3000C90408431061F0BD106901213840C904FD
:10AD400008431061F0BD002904D050692840304309
:10AD50005061F0BD5069384030435061F0BD00296A
:10AD600006D0506901212840C90408435061F0BD54
:10AD7000516901203940C00401435161F0BD0029EF
:10AD800004D02069284030432061F0BD206938405C
:10AD900030432061F0BD002906D020690121284000
:10ADA000C90408432061F0BD216901203940C00475
:10ADB00001432161F0BD002904D06069284030437F
:10ADC0006061F0BD6069384030436061F0BD0029CA
:10ADD00006D0606901212840C90408436061F0BDC4
:10ADE000606901213840C90408436061F0BDF3B5D2
:10ADF0008BB00C4600200B994F077F0F1A493B0080
:10AE000001F00FFE08050509090C0C101013486924
:10AE10008000800F09E04869800F06E0C86980065D
:10AE2000800F02E0C8690006800F002834D0012896
:10AE300035D0022836D00F4803900648064D0B9EA9
:10AE4000103D00680149064A16E000004000044039
:10AE5000580C0020680200201F000F000F001F0088
:10AE600040001440780C00200002005080E100E017
:10AE7000EFFFEFFF00805101330001F0D2FD181702
:10AE80001717172626262625252525252525253687
:10AE90004F6A839EB7D2EB25FC480390CDE7FC4870
:10AEA0000390CAE7FB4800680390C6E7FA4A916836
:10AEB0000B98C3009B1C01209840E3688143002B42
:10AEC00000D1002001439160DEE0F44A91680B98C4
:10AED000001FC3009B1C01209840E3688143002BA6
:10AEE00000D1002001439160CEE000280AD00A6919
:10AEF000E0682A40002801D0012000E00020024341
:10AF00000A61C1E00A69E6480240E068002801D011
:10AF1000012000E0002002430A61B5E000280BD0C8
:10AF20000A69E0682A40002802D00120000400E0FD
:10AF3000002002430A61A7E00A69D9480240E0689C
:10AF4000002802D00120000400E0002002430A6132
:10AF50009AE000280AD04A69E0682A40002801D017
:10AF6000012000E0002002434A618DE04A69CC489C
:10AF70000240E068002801D0012000E000200243E8
:10AF80004A6181E000280BD04A69E0682A40002825
:10AF900002D00120000400E0002002434A6173E077
:10AFA0004A69BF480240E068002802D0012000043E
:10AFB00000E0002002434A6166E000280AD01169DF
:10AFC000E0682940002801D0012000E00020014372
:10AFD000116159E01169B2480140E068002801D0D0
:10AFE000012000E00020014311614DE000280BD05A
:10AFF0001169E0682940002802D00120000400E027
:10B000000020014311613FE01169A5480140E0685B
:10B01000002802D00120000400E00020014311615B
:10B0200032E000280AD05169E0682940002801D0A8
:10B03000012000E000200143516125E0516998485A
:10B040000140E068002801D0012000E00020014319
:10B05000516119E000280BD05169E06829400028AF
:10B0600002D00120000400E00020014351610BE008
:10B0700051698B480140E068002802D0012000049B
:10B0800000E00020014351610B983B004007400F56
:10B09000001F01F0C6FC0805050505131313132056
:10B0A0007D4A9168FB00DB1C012098402378814396
:10B0B000002B00D10020014391600CE0774A916899
:10B0C000C300DB1C0120984023788143002B00D172
:10B0D00000200143916007230B981D461840810012
:10B0E00062688D400A950591011F0D4689008B40CD
:10B0F00007910C214D4369490993691808910C2166
:10B100004843654940180690002A0CD01146039820
:10B1100001F0FCFB049001210498090788427AD9C8
:10B1200000200DB0F0BD01253B0001F07AFC0805C0
:10B13000050D0D17171F1F2857480168E278090AE7
:10B140000902114301601AE0534A1068FF21090205
:10B150008843E17809020843106010E04F48016815
:10B16000E278090A09021143016008E04B4A1068BD
:10B17000FF2109028843E1780902084310606178E1
:10B18000A0684843642101F0C1FB401E3B0001F070
:10B1900048FC080505050517171717283E4E716866
:10B1A0000A9A9143A2785307059A5B0F934019437B
:10B1B0007160A168069A491ED1600699086110E085
:10B1C000364E7168099A9143A2785307079A5B0F2C
:10B1D000934019437160A168089A491ED16008998B
:10B1E0000861A078030001F01CFC04030507090AAC
:10B1F000022504E0042502E0082500E01025E1789E
:10B200000398491C694301F081FBA16801F07EFBB2
:10B210000490DEE0FFE7012504986904884201D22A
:10B22000022642E00498060C3146049801F06EFBB9
:10B2300001210904884201D9761CB6B2FF200130F1
:10B24000864232D9002506460498000A04900498E4
:10B25000000C01900199049801F058FB01210904A8
:10B26000884203D90198401CC0B2019001222946AE
:10B270006D1C104688400199EDB28842F7DD6D1EC5
:10B28000AA40D5B2102D0DD900204AE7001BB70007
:10B290000080000000000020000004400000144076
:10B2A000EFFFEFFF04987043049031466943049820
:10B2B00001F02CFB82B202923146039801F026FB8A
:10B2C000029A2946514301F021FB04903B0001F012
:10B2D000A8FB0805050E0E191922222C77490868CB
:10B2E000000A0002761EF2B2104308601DE0734AA5
:10B2F0001068FF2109028843761E3106090C0843B5
:10B30000106012E06E490868000A0002761EF2B270
:10B310001043086009E06A4A1068FF210902884367
:10B32000761E3106090C08431060042D0ED004DC93
:10B33000012D07D0022D0ED106E0082D08D0102DCA
:10B3400009D107E0042506E0002504E0012502E01C
:10B35000022500E003250B98C0060AD5A068411E0F
:10B360008EB261784843642101F0D0FA401E80B269
:10B370000AE00298401E86B2607802994843642130
:10B3800001F0C4FA401E80B23B0001F04AFB080500
:10B390000505051414141422484B59680A9A6C07C1
:10B3A0009143059A640F9440214359600699CE60F9
:10B3B000069908610DE0424B5968099A6C07914360
:10B3C000079A640F9440214359600899CE60089908
:10B3D00008610498A5E6F0B5394E034640360125CC
:10B3E000143B2A469A404407640F2B46A340071F8C
:10B3F0002C46BC408540002919D0C1060BD540071A
:10B4000003D5B06B1043B063F0BD2C484030816B66
:10B4100019438163F0BD400703D5F06B2043F0630F
:10B42000F0BD26484030C16B2943C163F0BDC10661
:10B430000BD5400703D5B06B9043B063F0BD1F48F8
:10B440004030816B99438163F0BD400703D5F06BB9
:10B45000A043F063F0BD19484030C16BA943C163FC
:10B46000F0BD10B54407640F8807164A800F23000B
:10B4700001F0D7FA0805050E0E15151C1C0D5069B4
:10B4800003231B078907984389080843506110BDAF
:10B4900050698000800889070843506110BDD16958
:10B4A0003023994300010143D16110BDD169C0230C
:10B4B000994380010143D16110BD000000000440A8
:10B4C000000014400002005070B5FC4DE86AFC4CCE
:10B4D000800708D50220E862E068401CE0606068F0
:10B4E000002800D08047E86AC00705D00120E86244
:10B4F000A068002800D0804770BD10B56421EF4AD5
:10B50000F04C002053681B0C1B041B19536053683C
:10B510001B0C1B041B1953605368DB0302D4401C33
:10B52000FF28F4DBFF2801D0002010BD491E0029B0
:10B53000E7D1E54810BD10B5E44AE1490020886034
:10B540004860C860E2480068C107E24819D0E24B91
:10B5500019680224214319601146521E0029FBD1AB
:10B56000996821439960D54ADC4911600021DC4B80
:10B570001468012C02D0491C9942F9DB994200D091
:10B58000002010BDFEB50446D04E00200190009072
:10B590000122A1691046002902D00C2900D8002000
:10B5A0007D27E3693F01DB1B1146632B00D8002197
:10B5B000084361691346002902D01F2900D80023DF
:10B5C000184302D0C348401FFEBDC2492078091F5E
:10B5D000002803D0012808D00846FEBDE0680028F6
:10B5E00001D00C2806D90846FEBDE068172801D90D
:10B5F0000846FEBDA16810463B2900D800206268BD
:10B6000001213B2A00D80021084302D0B148C01EC6
:10B61000FEBD2069062802D9AE48801EFEBDFFF798
:10B620006CFF0146A64841614069002801D0A64848
:10B63000FEBD2078A14D002856D0FFF75EFF686957
:10B64000012108436861E0690A21C01B01F05EF92D
:10B6500000050F0407430A21A06901F057F9000310
:10B6600038430F0207430A21606901F04FF90001D6
:10B6700038430143924F7961FFF73FFF6869012129
:10B6800008436861786928610A21E06801F03EF9A1
:10B6900000050A04024302920A21A06801F036F96B
:10B6A000029A000310430A02024302920A216068D0
:10B6B00001F02CF9029A0001104301437961FFF770
:10B6C0001CFF7869E8602069A861286B082188431D
:10B6D00020342178C907090F084328633546761EB0
:10B6E000002DFBD10020FEBDFFF707FF6869400871
:10B6F0004000686160780228A5D1E0681430E060FD
:10B70000A1E710B56D4B5A69D407E40F0C709A6924
:10B710005207520F0A616A4A002804D0012833D028
:10B720006C48401C10BD18690002000F9061186938
:10B730000003000FD0611869C004C00F10621869BF
:10B740000005000F506218698006800F906218692A
:10B750000007000FD062D8688002800F1063D8689D
:10B760000003000F5063D8684004400F9063D8680E
:10B770000005000FD063D8684006400F1064D868F9
:10B780000007000F50642FE0186A0002000F90615C
:10B79000186A0003000FD061186AC004C00F10625D
:10B7A000186A0005000F5062186A8006800F9062C8
:10B7B000186A0007000FD062D8698002800F1063FA
:10B7C000D8690003000F5063D8694004400F9063AC
:10B7D000D8690005000FD063D8694006400F106497
:10B7E000D8690007000F506490690A235843D36951
:10B7F000C0187D231B01C018C861106A0A23584372
:10B80000536AC0188861906A0A235843D36AC018E3
:10B810004861002C13D0106B0A235843536BC01897
:10B82000C860906B0A235843D36BC0188860106CB3
:10B830000A235843526C80184860002010BD106BDA
:10B840000A235843536BC018C860152804D3022339
:10B850004B701438C86001E001204870906B0A23D7
:10B860005843D36BC0188860106C0A235843526C3D
:10B8700080184860E1E710B5114C104A01230128F7
:10B880000BD0022802D01348401C10BD2361906ADF
:10B89000022318439062616004E06370906A184369
:10B8A0009062A1600F4908680202120A4807024329
:10B8B0000A600D490860002010BD000000800040B3
:10B8C0006C02002065A900000892FFFFE803000059
:10B8D000000100500592FFFF000200505713EBA536
:10B8E000FFFFAF001CE400E000E100E0F3B581B031
:10B8F0000C460127A0693B46002802D00C2800D83E
:10B9000000237D25E2692D01521B3946632A00D8A8
:10B9100000210B4361693E46002902D01F2900D84F
:10B9200000263343854E01D03046FEBD632A01D93F
:10B930003046FEBD002801D00C2801D93046FEBD9E
:10B94000002901D01F2901D93046FEBD20780028EA
:10B9500003D0012808D03046FEBDE068002801D0A1
:10B960000C2806D93046FEBDE068172801D93046BC
:10B97000FEBDA0683B2801D93046FEBD60683B286B
:10B9800001D93046FEBD2069062801D93046FEBDEA
:10B99000FFF7B3FD6A4D68616869002801D0304641
:10B9A000FEBD01980021674E002804D0012858D020
:10B9B0006248801EFEBD2078002846D02F70706936
:10B9C00038437061B0692169C008C0004907490F58
:10B9D0000843B0617D20E1690001081A0A2100F0E6
:10B9E00095FF00050F0407430A21A06900F08EFFB0
:10B9F000000338430F0207430A21606900F086FF05
:10BA00000001384301436961FFF777FD68693061E0
:10BA10000A21E06800F07AFF00050F0407430A21BD
:10BA2000A06800F073FF000338430F0207430A21A8
:10BA3000606800F06BFF0001384301436961FFF764
:10BA40005CFD6869F0600020FEBD297070694008E7
:10BA50004000706160780228B4D1E0681430E06082
:10BA6000B0E7A9607D20E1690001081A0A2100F011
:10BA70004DFF00050F0407430A21A06900F046FFAF
:10BA8000000338430F0207430A21606900F03EFFBC
:10BA90000001384301436961FFF72FFD6869306297
:10BAA0002878002805D16078022802D1E068143097
:10BAB000E0600A21E06800F029FF00050F04074359
:10BAC0000A21A06800F022FF000338430F02074359
:10BAD0000A21606800F01AFF0001384301436961E0
:10BAE000FFF70BFD6869F06100210120FFF7C3FE3D
:10BAF000306B0821884320342178C907090F084397
:10BB000030630020FEBD10B504460D490020C8601A
:10BB1000FFF7F3FC002802D00848C01E10BD072C18
:10BB200002D90648801E10BD0648016B6207C9088D
:10BB3000C900520F11430163002010BD0892FFFF9E
:10BB40006C020020008000408307FF22DB0E9A4039
:10BB50008907090E994000280BDA0007000F083802
:10BB600083089B00FF481818C36993430B43C361C4
:10BB700070478308FC489B001818036893430B43E5
:10BB80000360704710B5002807D0012805D00228AF
:10BB900003D0032801D0F54810BDF549496980005C
:10BBA0000830C1404807400F002808D0012809D0BC
:10BBB000022809D007280AD0EC48401C10BDFEF727
:10BBC000A3F910BDEB4810BDFEF726FA10BDEA48F8
:10BBD00010BDF3B581B00D460198E84F02280FD390
:10BBE000002D0DD00124E64E29466143019800F056
:10BBF0008DFE811EB14205D2641E21060843FEBDA2
:10BC00003846FEBD641CFF2CEED93846FEBD10B58B
:10BC1000DC48016801228900002905DA8168C9072A
:10BC200002D08168114381604169090708D54169E3
:10BC3000890605D58169C90702D0816911438161EF
:10BC4000D149086B401C0863D04C2068002809D0FB
:10BC5000A068401EA060002804D1E16820698847E0
:10BC60006068A06010BD10B5C648016A0122890055
:10BC7000002905DA816AC90702D0816A114381620D
:10BC8000416B090708D5416B890605D5816BC9074A
:10BC900002D0816B11438163BB49486B401C4863F0
:10BCA000BA4C14342068002809D0A068401EA06057
:10BCB000002804D1E168206988476068A06010BD51
:10BCC00010B5B348016801228900002905DA8168AE
:10BCD000C90702D08168114381604169090708D50D
:10BCE0004169890605D58169C90702D08169114377
:10BCF0008161A549886B401C8863A44C2834206866
:10BD0000002809D0A068401EA060002804D1E16886
:10BD1000206988476068A06010BD10B59C48016A22
:10BD200001228900002905DA816AC90702D0816AE7
:10BD300011438162416B090708D5416B890605D51E
:10BD4000816BC90702D0816B114381638E49C86B37
:10BD5000401CC8638D4C3C342068002809D0A06882
:10BD6000401EA060002804D1E1682069884760680F
:10BD7000A06010BD84480121016041608160C16004
:10BD80007047F7B507460C46002502990120CE06FC
:10BD9000774A0021002F07D0012F3DD0022F76D007
:10BDA000032F70D07148FEBD774B1B68012B03D168
:10BDB000754B1B69002B02D06C48801CFEBD724B7A
:10BDC00018616B4A926804231A43694B9A606D4A62
:10BDD0001160936803439360002014220346534389
:10BDE0006A4AD150401C0028F7D0674801630465B7
:10BDF0000020FFF7C7FE2146FFF7EBFE411C08D0ED
:10BE000002026049120A4A60000E2843304308606B
:10BE1000C3E05648401CFEBD5B4B5B68012B03D161
:10BE2000594B5B69002B02D05048801CFEBD564B1D
:10BE300001205861906808231843906051480162BE
:10BE4000836A012213438362002014220346534372
:10BE50004E4A1432D150401C0028F6D04A48416363
:10BE600044650120FFF78EFE2146FFF7B2FE411C1C
:10BE70000AD002024349120A4A62000E28433043A4
:10BE800008628AE003E03BE03848401CFEBD3E4BC0
:10BE90009B68012B03D13C4B9B69002B02D033489C
:10BEA000801CFEBD384B9861314A936810221343C1
:10BEB0002F4A9360364A11609368034393600020D1
:10BEC000142203465343314A2832D150401C0028E3
:10BED000F6D02D48816384650220FFF753FE21468A
:10BEE000FFF777FE411C08D002022949120A4A6076
:10BEF000000E2843304308604FE01C48401CFEBD44
:10BF0000214BDB68012B03D11F4BDB69002B02D0D7
:10BF10001648801CFEBD1C4BD861154A9268202330
:10BF20001A43134B9A601A4A1162936A034393624D
:10BF30000020164B3C33142242439950401C0028E9
:10BF4000F9D01148C163C4650320FFF71BFE2146E9
:10BF5000FFF73FFE411C25D002020D49120A4A623A
:10BF6000000E17E000ED00E000E400E00197FFFFA5
:10BF7000000200500080000000805101FFFFFFFF21
:10BF8000FEFFFF0000000140B4020020980C0020DA
:10BF9000000011402843304308620298022803D071
:10BFA0000020FEBDD848FEBD002F05D0012F03D0D4
:10BFB000022F01D0032F03D12137F8B2FEF700FA88
:10BFC000D148401EFEBD002808D0012806D0022816
:10BFD00004D0032802D0CC48401E7047CB4A8100D1
:10BFE0005158CB4A89180A6801235B079A430A60B3
:10BFF0000830C106C90E01208840C64908600020EB
:10C000007047F0B5C24F0024BE02C34D002809D0CE
:10C01000012810D0C14F022816D003281DD0BA48DD
:10C02000401EF0BD0020FFF7CEFF38683043386077
:10C030002C612C6219E00120FFF7C5FF386A3043FC
:10C0400038626C616C6210E00220FFF7BCFF386858
:10C0500030433860AC61AC6207E00320FFF7B3FF08
:10C06000386A30433862EC61EC620020F0BDF0B514
:10C0700004460020A44FA84DBF1C0126002C0AD066
:10C08000012C28D0022C47D0032C03D1EC6C002CBF
:10C0900063D03846F0BD2C6C002C01D03846F0BD82
:10C0A0002E622C6C641C2C6400249D4F05E014252A
:10C0B00065437D59002D03D0641C012CF7DBF0BDD6
:10C0C0002046142568433E50C01941608160C2601B
:10C0D00003612046F0BD6C6C002C01D03846F0BDE9
:10C0E0006E626C6C641C6C6400258D4F143705E027
:10C0F00014246C433C59002C03D06D1C012DF7DB3C
:10C10000F0BD2846142460433E50C0194160816050
:10C11000C26003612846F0BDAC6C002C01D03846EB
:10C12000F0BDAE62AC6C641CAC6400247C4F28375C
:10C1300005E0142565437D59002D03D0641C012CB6
:10C14000F7DBF0BD2046142568433E50C01941601E
:10C150008160C26003612046F0BDEE62EC6C641C3D
:10C16000EC6400246E4F3C3705E0142565437D598F
:10C17000002D03D0641C012CF7DBF0BD20461425F4
:10C1800068433E50C01941608160C260036120462F
:10C19000F0BD10B5002808D0012806D0022804D030
:10C1A000032802D05848401E10BD584A81005158FB
:10C1B000574A89180A6801235B071A430A60083046
:10C1C00040B202210446FFF7BFFC2046C106C90E5B
:10C1D0000120884053490860002010BD002808D085
:10C1E000012806D0022804D0032802D04648401E69
:10C1F00070474649800008584549401801680122A7
:10C200009207114301600020704747490868800683
:10C21000C00F0A6808231A430A603F49096E0029C3
:10C2200000D008477047F3B581B0022401273E498A
:10C23000802540221026030000F0F3FB0A060A0EB8
:10C24000181E22262A2E323D08682843086030E056
:10C250000868A84308602CE00868104308600221C1
:10C260000120FFF771FC2F48046022E0086890432A
:10C270000860284804601CE008683043086018E043
:10C280000868B043086014E008683843086010E0AC
:10C290000868204308600CE00868A043086008E0D4
:10C2A0000868072212029043029A5207520D104367
:10C2B00008600020FEBD1448C01CFEBD10B5044639
:10C2C0001A480068C00713D0194988680122104332
:10C2D000886000210120FFF7A6FF13490A680720A4
:10C2E000000282436007400D02430A60002010BD37
:10C2F0000548001D10BD0C490A6840231A430A6016
:10C3000005490866704700000297FFFF44EE0000F1
:10C310000000014080E100E0B40200200000114074
:10C32000980C002000E100E00040004000010050B7
:10C330000002005070B5F848C069F849CC69F84D62
:10C340002968002900D08847A968002901D0204623
:10C35000884770BDF348C069F1494968002900D099
:10C3600008477047F8B5EC4BD41800F0CFFA0746F1
:10C37000012100074907000F4A10032808D2606A0C
:10C3800088436062606A904360623E09B61E27E09F
:10C39000606A08436062606A10436062BE1EE248E1
:10C3A00086421DDD606A08436062606A9043606295
:10C3B00008253846691C00F0A9FA03290DD2606AE5
:10C3C0000F21090688432907090908436062384696
:10C3D000691C00F09BFA861E02E06D1C102DE8DB44
:10C3E000606AB1B2000C000408436062F8BD10B589
:10C3F000CE48816909050C0F41698901890F09D06F
:10C4000040698001800F012807D0C948611C00F0F5
:10C410007DFA10BDFDF778FDF8E7FDF7D3FDF5E7F0
:10C4200070B505460C46C349002D07D08D4205D096
:10C4300041208003854201D0BF4870BDA07900280B
:10C440000AD0032808D0012806D0052804D00728E0
:10C4500002D0B948401C70BD2079002808D00128BE
:10C4600006D0022804D0032802D0B348801C70BD37
:10C470006079002804D0012802D0AF48C01C70BDEC
:10C48000E07900280ED001280CD002280AD0032819
:10C4900008D0042806D0052804D0062802D0A648D3
:10C4A000001D70BD05200007A04A002D0CD08D4254
:10C4B00016D1C36811020B43C360C3688B43C360CA
:10C4C00090680843906016E0C368012109040B439B
:10C4D000C360C3688B43C3609068084390600AE000
:10C4E000C368012189040B43C360C3688B43C360E5
:10C4F00090680843906088482B1898680421084386
:10C50000986098680226304398609868F026B04397
:10C51000E6793607360E30439860A079202640072A
:10C52000002802DAD868304301E0D868B043D86008
:10C53000A07910268007002802DAD868304301E08D
:10C54000D868B043D860D8680826B043A679F60703
:10C55000360F3043D860D868267980088000B60747
:10C56000B60F3043D860D86888436179C907490F4E
:10C570000843D860186A217A000A0002084318624A
:10C580001068C1076D4803D05169814351610FE0C4
:10C59000116AC90306D451698143012000060818B5
:10C5A000506105E0116849070AD55169014351619D
:10C5B000FFF71DFF2A462168FFF7D4FE002070BD5B
:10C5C0005D48801D70BD10B55A49584A0023544C2F
:10C5D00088420DD153488169C900FCD5906801217A
:10C5E00049048843906063600D2000F0D9F810BDC5
:10C5F0004121890388420DD148488169C900FCD591
:10C6000090680121890488439060A3600C2000F0A9
:10C61000C7F810BD40488169C900FCD59068012168
:10C6200009048843906023600C2000F0B9F810BD25
:10C6300030B5394BC3185C68CD0764086400ED0F52
:10C640002C435C608C070225002C02DA5C682C43CA
:10C6500001E05C68AC435C604C070425002C02DA06
:10C660005C682C4301E05C68AC435C600C07082507
:10C67000002C02DA5C682C4301E05C68AC435C602F
:10C680002F4DCC0602D55C682C4301E05C68AC43BE
:10C690005C60CC061025002C02DA5C682C4301E0BB
:10C6A0005C68AC435C608C062025002C02DA5C6878
:10C6B0002C4301E05C68AC435C600C064025002C18
:10C6C00002DA5C682C4301E05C68AC435C601D4CA2
:10C6D000C90502D55968214301E05968A143596051
:10C6E000012424030E49184B002806D02502A84235
:10C6F00006D14A601548186030BD0A601C6030BD24
:10C700008A601C6030BD70B5034BC4180023104D07
:10C710002BE0002023E00000000005400040154011
:10C720001803002000001540FFFF00000002005029
:10C7300000805101000010000298FFFF000000037C
:10C74000000800000001000000E100E000200000FF
:10C7500000040000401CA84201D3154870BDA66922
:10C760007604F7D42068C8545B1C9342D1D30020D0
:10C7700070BD70B50F4BC41800230F4D0CE00020A6
:10C7800004E0401CA84201D3094870BDA669F60028
:10C79000F7D5C85C20605B1C9342F0D3002070BDCD
:10C7A000C106C90E01208840044908607047000096
:10C7B0000198FFFF000005400040000080E100E01C
:10C7C00010B54F4AD3681B091B015B1CD360D368AB
:10C7D0001024A343D360D36820242343D360506044
:10C7E0009160012080F310881069012108431061D5
:10C7F000BFF36F8F1069C007FCD180F310881068F9
:10C80000400605D510684021084310603D4810BD22
:10C81000002010BD10B53A4AD3681B091B01D36034
:10C82000D3681024A343D360D3682024A343D360E8
:10C83000506000209060012080F31088106901236F
:10C8400018431061BFF36F8F1069C007FCD180F3EC
:10C8500010881068400605D5106840210843106014
:10C86000284810BD90680860002010BD2449CA689F
:10C8700012091201921CCA60CA6810239A43CA6046
:10C88000CA6820231A43CA604860012080F31088D8
:10C890000869012210430861BFF36F8F0869C00760
:10C8A000FCD180F310880868400605D5086840224E
:10C8B00010430860134870470020704770B5124C51
:10C8C000206804254007002805DB206828432060F5
:10C8D0000C20FDF704FC6068284360600849086884
:10C8E00001221043086070BD0548016849084900ED
:10C8F00001607047024801682022114301607047BF
:10C9000000C000508188FFFF0002005030B50B4688
:10C91000014600202022012409E00D46D5409D4219
:10C9200005D31D469540491B25469540401915469F
:10C93000521E002DF1DC30BD0549064A08685043FF
:10C94000054A801808604008704701490860704730
:10C95000240300206D4EC6413930000003460B43CE
:10C960009B0703D009E008C9121F08C0042AFAD2A5
:10C9700003E00B78491C0370401C521EF9D270472B
:10C98000D2B201E00270401C491EFBD27047002267
:10C99000F6E710B504460846114602462046FFF762
:10C9A000EFFF204610BD0000064C0125064E05E0B5
:10C9B0002046E36807C82B4398471034B442F7D3A6
:10C9C000F3F782FB54EE000074EE000070B58C1893
:10C9D0000578401C6B075B0F01D10378401C2A11BE
:10C9E00006D10278401C03E00678401C0E70491CFA
:10C9F0005B1EF9D12B0705D40023521E0DD40B70FA
:10CA0000491CFAE70378401CCB1A921C03E01D78FE
:10CA10005B1C0D70491C521EF9D5A142D8D30020D1
:10CA200070BD30B47446641E2578641CAB4200D2DD
:10CA30001D46635D5B00E31830BC184702E008C880
:10CA4000121F08C1002AFAD170477047002001E088
:10CA500001C1121F002AFBD1704700387CE4C2C21A
:10CA6000828282860E1C000002F2FE0E7EF0C00062
:10CA7000000080700E0EFEF20200C0F0380C0402BE
:10CA8000020202040C38F0C202FEFE0282C0201232
:10CA90000A060602020000000000003870604040F4
:10CAA00041414163371E40787F47000000030F7EFD
:10CAB000700E0300000000477F78471F3820404079
:10CAC0004040404020381F47407F7F414103070ED0
:10CAD0001C3870E0C0C08080800030C00000E030B2
:10CAE000E00000C03000F010101010101000F00036
:10CAF0000000000000C02010101010204000C020D6
:10CB0000101010101020C000F070C0000000C070A5
:10CB1000F00000F0101010101010000718070000AF
:10CB2000010F180700001F111111111110001F1023
:10CB30001010101000070810101010080C00070843
:10CB400010101010100807001F00010E180E010031
:10CB50001F00001F111111111110C06030101010B2
:10CB600010204000C020101010101020C000C02065
:10CB7000101010101020C000F0101010101020C065
:10CB800000F01010101010E0001030608000806085
:10CB9000301000F0101010101010070C18101011A9
:10CBA00011091F00070810101010100807000708CF
:10CBB00010101010100807001F1010101010080798
:10CBC000001F11111111110E00000000011F0100C2
:10CBD0000000001F111111111110000000000000D1
:10CBE000000000000000000E1E3E7EFEFEFEFEBEA7
:10CBF0003E3E3C3878F8F8F8F8F8F8F8F8F8F878A5
:10CC0000383C3E3EBEFEFEFEFE7E3E1E0E00000096
:10CC10000000000000000000000000000000000014
:10CC200000000000000000000000000001FFFFFF06
:10CC3000FFFEFCF8F0E0C103070F0F0703C1E0F0AF
:10CC4000F8FCFEFFFFFFFF010000000000000000F5
:10CC500000000000000000000000000000000000D4
:10CC60000000000000000000000080C0E0FFFF7F27
:10CC70003F1F0F0783C1E0F0F8FCFCF8F0E0C18330
:10CC8000070F1F3F7FFFFFE0C08000000000000093
:10CC90000000000000000000000000000000000094
:10CCA000000000000000001C1E1F1F1F1F1F1F1F71
:10CCB0001F1F0F07070707070707070707070707CC
:10CCC000070F1F1F1F1F1F1F1F1F1F1E1C000000FD
:10CCD00000000000000000000000000000C0E06054
:10CCE00060606060E0C0000000E0E0000000000064
:10CCF000E0E0000000E0E06060606060E0C0000034
:10CD000000E0E06060606060600000000000000023
:10CD100060E0E06060E0E06000000000003F7F60F5
:10CD20006060606078380000003F7F606060606035
:10CD30007F3F0000007F7F66666666667F39000081
:10CD4000007F7F6666666666660000000000000081
:10CD5000607F7F60607F7F6000000000000004064D
:10CD600006E6FE1E060606060602E0FC1E0200009F
:10CD700000000000000000004666767EDECE06065B
:10CD80000000C0E0F078686CE6E2C000000000C07F
:10CD9000F0380C060606FEFC00000000000040789B
:10CDA0003F07000000000040787F676060606060BF
:10CDB00060000000187860606060301C0F070000A1
:10CDC000083F7F61606060301C0F030000003F7F00
:10CDD000606020301C0F0300000000000000000015
:10CDE0000000000000000000000000000000000043
:10CDF000000000000080C0C0E0E0F0F0F0F0F0F0D3
:10CE0000E0E0C0C080000000000000000000000062
:10CE10000000000000000000000000000000000012
:10CE20000000F0FCFFFF0F03010100000000000004
:10CE30000101030FFFFFFCF00000000080C0C0C034
:10CE4000C0C0C0C0C0C0C0C0C0C0C0C0C0C0C0C0E2
:10CE5000C0C0DFDFDFDFC0C0C08000000000000016
:10CE6000000000000707070700000000FFFFFFFFAA
:10CE7000FFFFFFFFFFFFFF0F0703030303070FFF82
:10CE8000FFFFFFFFFFFFFFFFFFFF000000000000AC
:10CE9000000000000000000000000000FFFFFFFF96
:10CEA000FFFFFFFFFFFFFFFFFE00000000FEFFFF90
:10CEB000FFFFFFFFFFFFFFFFFFFF0000000000007C
:10CEC0000000000000000000000000001F1F1F1FE6
:10CED0001F1F1F1F1F1F1F1F1F1F1E1E1F1F1F1F64
:10CEE0001F1F1F1F1F1F1F1F1F0F0000000000001C
:10CEF0000000000000000000000000000000000032
:10CF00000080C0E0E0F0F0787878787878F0F0E0B1
:10CF1000E0C080000000000000000000000000F8F9
:10CF2000FEFFFF07010000000000000000000001FC
:10CF300007FFFFFEF8000000000080C0C0C0C0DF97
:10CF4000DFDFDFC0C0C0C0C0C0C0C0C0C0C0C0C084
:10CF5000C0DFDFDFDFC0C0C0C080FFFFFFFFFFFF1B
:10CF6000FFFFFFFFFFFF0F0703030303070FFFFF91
:10CF7000FFFFFFFFFFFFFFFFFFFFFFFFFFFFFFFFC1
:10CF8000FFFFFFFFFFFFFFFE00000000FEFFFFFFAF
:10CF9000FFFFFFFFFFFFFFFFFFFF0F1F1F1F1F1FF1
:10CFA0001F1F1F1F1F1F1F1F1F1E1E1F1F1F1F1F93
:10CFB0001F1F1F1F1F1F1F1F1F0FC03008442222CB
:10CFC000410101412222440830C00000000000C09D
:10CFD000F0C0030C10204844828282824448201012
:10CFE0000C030070FC700001030100000080E0F001
:10CFF000F8FCFC7EFEFFFF0303070F1F3F7FFFFED1
:10D00000FEFCFCF8F0E0800000000000FEFFFFFFE7
:10D01000FFFFFFF8F0E1C30000003F1E0C80C0E1FD
:10D02000F3FFFFFFFFFFFFFE000000007FFFFFFF99
:10D03000FFFFFF1F0F87C3000000FC78300103874C
:10D04000CFFFFFFFFFFFFF7F000000000001070F81
:10D050001F3F3F7E7FFFFFC0C0E0F0F8FCFEFF7F78
:10D060007F3F3F1F0F07010000000078FCFECE87C6
:10D0700087CEFEFC787878787878787878787878C1
:10D08000787878787878787830000080C0C1C1C32B
:10D09000C3C1C1C0C0C0E0F070383870F0E0C0C09B
:10D0A000C0C0C0C0C0C0C0C08000000103030303F3
:10D0B000030303030303070F0E1C1C0E0F070303D8
:10D0C000038383C3C38383030100000C1E1E1E1E43
:10D0D0001E1E1E1E1E1E1E1E1E1E1E1E1E1E1E1E70
:10D0E0003F7F73E1E1737F3F1E00000000000004FA
:10D0F0000E1C381000000080808F8F8080000000A0
:10D1000010381C0E0400000000000303030303009A
:10D110000000F0FC0E030301010101010103030EF5
:10D12000FCF000000003030303030000000000F014
:10D13000F0303F3F30303030303030303030303011
:10D140003F3F30F0F000000000000000000000034E
:10D150000303030303FFFF0303030303037F7F03AF
:10D1600003030303030000000000000000000000B0
:10D1700000000000000000808080808080000000AF
:10D18000000000000000000000000000000000009F
:10D190000000F0FCFEFFFFFFFFFFFFFFFFFFFFFEB1
:10D1A000FCF000000000000000000000000000F0A3
:10D1B000F0303F3F3F3F3F3F3F3F3F3F3F3F3F3FDD
:10D1C0003F3F30F0F00000000000000000000003CE
:10D1D0000303030303FFFF0303030303037F7F032F
:10D1E0000303030303000000000000000000000030
:10D1F0000000FEFFFFFFFFFFFFFF7F7F7F7F7F7F3E
:10D200007FFFFEFEFEFCFCF8F0C000000000000006
:10D210000000FFFFFFFFFFFFFFFFE0E0E0E0E0E0D6
:10D22000E0F0FFFFFFFFFFFFFF3F000000000000F6
:10D230000000FFFFFFFFFFFFFFFF0F0F0F0F0F0F9C
:10D240000F0F0707070303010000071F3E7C78F854
:10D25000F8FCFFFF7F7F7F3F1F03000000000000FE
:10D2600000000000000000000000000080C0F0F09E
:10D27000783C1C0E0E0F0707C7E7E7C7070F0E0E17
:10D280001E1C3C78F0E0C0800000F0FEFF1F030091
:10D29000000000000000C0E0FFFFFFFFE0C0C0C0D2
:10D2A000C0C0800000031FFFFEF00F7FFFF8C0002A
:10D2B00000000000000003070F0F0F0F0703030318
:10D2C0000303010000C0F8FF7F0F00000103070FF8
:10D2D0001E3C38787070F0E0E0E0E0E0E0F0707064
:10D2E00078383C1E0F0703010000000040E0F0F812
:10D2F000FCF8F0F0F0F8F8FFFFFFFFFFFFF8F8F0A0
:10D30000F0F0F8FCF8F0E0400000E0E0E0F8FFFFAB
:10D31000FFFFFF3F0F070303010101010303070F95
:10D320003FFFFFFFFFFFF8E0E0E00707071FFFFFF9
:10D33000FFFFFFFCF0E0C0C080808080C0C0E0F054
:10D34000FCFFFFFFFFFF1F070707000002070F1F7B
:10D350003F1F0F0F0F1F1FFFFFFFFFFFFF1F1F0FBD
:10D360000F0F1F3F1F0F070200000000081830209A
:10D370000080C0C0E0E0E7E7E0E0C0C0800020300F
:10D380001808000000000000000018181800007CB9
:10D39000FFFFFFFFFFFFFFFFFFFFFFFFFFFF7C001F
:10D3A0000018181800000000000000000000000035
:10D3B0000103070FFF5F5F9F9FFF0F070301C0205F
:10D3C000101008E808101020C00000000000000045
:10D3D000000000003F65E5EA6A3F000000071820F2
:10D3E00040408287824242201807000080C0F0F04F
:10D3F000F83C3C1E0E0F07070707FFFFFFFFFEFE6E
:10D40000FEFCFCF8F0E0C0800000F0FEFFFF0F0122
:10D4100000000000000000000000FFFFFFFFFFFF12
:10D42000FFFFFFFFFFFFFFFFFEF00F7FFFFFF0C0DA
:10D4300000000000000000000000FFFFFFFFFFFFF2
:10D44000FFFFFFFFFFFFFFFF7F0F00000103070F3C
:10D450001F3E3C787070E0E0E0E0FFFFFFFF7F7F61
:10D460007F3F3F1F0F070301000000000000000086
:10D4700000000000000000000000040E1F0E0E0E51
:10D480001E1C3C78F0E0C08000000000000000009E
:10D4900000000000000000F8FE0603030306FEF88B
:10D4A0000000000000031FFFFEF00F7FFFF8C00028
:10D4B0000000000000FFFFFFFFFFFFFFFFFFFFFF77
:10D4C000FFFF000000000000000000000103070F44
:10D4D0001E3C3878707070F870200000000000006A
:10D4E00000000000000000000000001E33E1E133F6
:10D4F0001E0000000000000000000000000000000E
:10D500000000001E33E1E1331E000000001F1F6019
:10D510006060601C1C606060609C9C606060601C5F
:10D520001C606060601F1F00000000000000000021
:10D530000000000000080C0603FFFF03060C0800B3
:10D5400000000000000000000000000000000000DB
:10D550000000000000000078CC8787CC7800000035
:10D5600000000000000000000000000000000000BB
:10D57000000000000000FFFFFFFFFFFFFFFF0000B3
:10D5800000000000000000000000E0F0F8783838EB
:10D59000383838380000FFFFFFFFFFFFFFFF0000B3
:10D5A00038383838383878F8F0E0FFFFFF000000EE
:10D5B00000040C1C3C7CFFFFFFFFFFFFFFFF7C3CD7
:10D5C0001C0C0400000000FFFFFF3F7FFFF0E0E0C5
:10D5D000E0E0E0E0E0E0E0E1E3E7E7E3E1E0E0E035
:10D5E000E0E0E0E0E0E0F0FF7F3F0000000080C00E
:10D5F000C0E0E0E0000000FEFFFFFFFFFE000000D3
:10D60000E0E0E0C0C08000000000E0FCFEFFFFFFA3
:10D61000FF3F1F0F000000FFFFFFFFFFFF000000A4
:10D620000F1F3FFFFFFFFFFEFCE03FFFFFFFFFFF7D
:10D63000FFF0C080000000070F0F0F0F0700000071
:10D6400080C0F0FFFFFFFFFFFF3F000003070F1F39
:10D650003F3F7F7F7FFEFEFCFCFCFCFCFCFEFE7F70
:10D660007F7F3F3F1F0F07030000F808E4E4E4E476
:10D6700008F8FF00FFFFFFFF00FFFF80BFBFBFBF35
:10D6800080FFF8088484848408F8FF00FFFFFFFF10
:10D6900000FFFF80BFBFBFBF80FFF8080404040481
:10D6A00008F8FF00FEFEFEFE00FFFF80BFBFBFBF09
:10D6B00080FFF8080404040408F8FF00F8F8F8F8FC
:10D6C00000FFFF80BFBFBFBF80FFF8080404040451
:10D6D00008F8FF00E0E0E0E000FFFF80BFBFBFBF51
:10D6E00080FFF8080404040408F8FF0080808080AC
:10D6F00000FFFF80BFBFBFBF80FFF8080404040421
:10D7000008F8FF000000000000FFFF80BEBEBEBEA4
:10D7100080FFF8080404040408F8FF00000000007B
:10D7200000FFFF80BCBCBCBC80FFF80804040404FC
:10D7300008F8FF000000000000FFFF80B8B8B8B88C
:10D7400080FFF8080404040408F8FF00000000004B
:10D7500000FFFF80B0B0B0B080FFF80804040404FC
:10D7600008F8FF000000000000FFFF80A0A0A0A0BC
:10D7700080FF1EF0F81EF8F01E00004C929292926C
:10D7800064000609090600FFFFFF111111010609D7
:10D790000906007EFFFF8181C34200048850FFFE1E
:10D7A000DC88000100000703010000000000000009
:10D7B000000C1E1E0C0000307878300000000000C5
:10D7C00000000080C0C080000081C3C38100000150
:10D7D0000303010098A4C202C2A498C02010080844
:10D7E00008081020C03122243800003824223100DB
:10D7F000F0F81818F8F000001F3F30303F1F00000D
:10D800003030F8F80000000000003F3F000000004A
:10D8100070781898F8F00000383C3E37313000003E
:10D8200030389898F87000001C3C31313F1E0000E1
:10D8300080E030F8F80000070706063F3F060000CA
:10D84000F8F89898981800001B3B31313F1F0000F2
:10D85000F0F89898B83000001F3F31313F1F0000AA
:10D86000181818D8F838000000303F3F01000000B9
:10D8700070F89898F87000001E3F31313F1E00008C
:10D88000F0F81818F8F00000193B33333F1F000080
:10D89000F0F81818F8F000809FBFB0B0BF9F80006C
:10D8A0003030F8F8000000808080BFBF80808000AA
:10D8B00070781898F8F00080B8BCBEB7B1B080009E
:10D8C00030389898F87000809CBCB1B1BF9E800041
:10D8D00080E030F8F8000087878686BFBF8680002A
:10D8E000F8F89898981800809BBBB1B1BF9F800052
:10D8F000F0F89898B83000809FBFB1B1BF9F80000A
:10D90000181818D8F838008080B0BFBF8180800018
:10D9100070F89898F87000809EBFB1B1BF9E8000EB
:10D92000F0F81818F8F0008099BBB3B3BF9F8000DF
:10D930000080C0E060606060C0C080000000FCFF4C
:10D940000300000000000003FFFC00003FFFC000D8
:10D950000000000000C0FF3F0000000103030606B6
:10D960000606070301000000000000000000E0E0E0
:10D97000000000000000000606060707FFFF000089
:10D9800000000000000000000000FFFF0000000099
:10D990000000000000000000070700000000000079
:10D9A0000080C0E060606060E0C0800000000F0F99
:10D9B00001000000000080E1FF3F000080E0703CBB
:10D9C0001C0E0703030100000000070706060606F9
:10D9D000060606060606000000C0C060606060E043
:10D9E000C0800000000007070000808080C0E17F49
:10D9F0003F000000F0F08000010101010387FEFC00
:10DA000000000001030706060606070301000000E8
:10DA100000000000000000C0E0E000000000000086
:10DA200080E0781C0701FFFF000000001C1F1B188E
:10DA300018181818FFFF1818000000000000000058
:10DA4000000007070000000000E0E0606060606028
:10DA5000606060000000F8FF7F203030303070E000
:10DA6000C0000000E0E08000000000000080FF7FB8
:10DA7000000000010307060606060303010000007C
:10DA80000000C0C060606060C0C000000000F8FF1F
:10DA9000C3C060606060E0C3830000003FFF81009E
:10DAA000000000000081FF7E000000010303060665
:10DAB000060607030100000060606060606060604F
:10DAC0006060E06000000000000000C0F0781E0709
:10DAD00001000000000000F0FE3F03000000000015
:10DAE0000000000007070700000000000000000021
:10DAF0000000C0C060606060C0C000000000001F87
:10DB0000BFE0C0C0C0C0E0BF1F0000007CFF8301B9
:10DB1000000000000183FF7E0000000103070606ED
:10DB200006060703010000000080C0E0606060603E
:10DB3000C0C0800000007EFF810000000000008166
:10DB4000FFFC000000C1C3070606060603C3FF1F53
:10DB500000000000030306060606030300000000A1
:10DB6000003030000000000000E0E0E00000006055
:10DB70006000000000000018180000000080C06075
:10DB8000301003070C183020103060C080002030A7
:10DB9000180C07030080C060309003070C1833276F
:10DBA000903060C080002733180C0703000000FC91
:10DBB000FE03E1F1F1E103FEFC0098989898989833
:10DBC0000000000000000000000000000080E0787D
:10DBD0001CC6E2C61C78E08000000000000000FFC8
:10DBE000FF00FFFFFFFF00FFFF00999999999999A6
:10DBF00000000000000000000080E0781E07010027
:10DC00000043EF43000001071E78E080E0F81C8F1E
:10DC1000E7F0FFFFFFFFF0E78F1CF9E101010101D1
:10DC200000000000000000000003070606060606CC
:10DC3000060606060606060606060703030F1C3838
:10DC40003367676F6F676733381C0F03000000008E
:10DC500000000000000000000000000000000000C4
:10DC600000000000000000000000000000000000B4
:10DC70000000E0E02020E0E0E02020E060A0A0A0A4
:10DC800060E00000000000003F3F203F3827383FA1
:10DC9000203F302E2D2B303F000000000000E0E040
:10DCA0002020E0E0E02020E0E0E06020E0E0000074
:10DCB000000000003F3F203F3827383F203F3F3FD4
:10DCC0003F203F3F000000000000E0E02020E0E0B7
:10DCD000E02020E060A0A0A060E0000000000000C4
:10DCE0003F3F203F3827383F203F2F272B2D2E3F07
:10DCF000000000000000E0E02020E0E0E02020E064
:10DD000060A0A0A060E00000000000003F3F203FB6
:10DD10003827383F203F372F2D2D323F000000009D
:10DD20000000E0E02020E0E0E02020E0E0E06020F3
:10DD3000E0E00000000000003F3F203F3827383F70
:10DD4000203F33343720373F000000000000E0E080
:10DD50002020E0E0E02020E0E020A0A0A0E0000003
:10DD6000000000003F3F203F3827383F203F342D40
:10DD70002D2D333F000000000000E0E02020E0E017
:10DD8000E02020E060A0A0A060E000000000000013
:10DD90003F3F203F3827383F203F302D2D2D333F48
:10DDA000000000000000E0E02020E0E0E02020E0B3
:10DDB000A0A0A0A020E00000000000003F3F203F06
:10DDC0003827383F203F3F3F213E3F3F00000000C3
:10DDD0000000E0E02020E0E0E02020E060A0A0A043
:10DDE00060E00000000000003F3F203F3827383F40
:10DDF000203F322D2D2D323F000000000000E0E0DA
:10DE00002020E0E0E02020E060A0A0A060E0000092
:10DE1000000000003F3F203F3827383F203F362D8D
:10DE20002D2D303FE0E02020E0E0E02020E0E0E0A9
:10DE30006020E0E060A0A0A060E03F3F203F3827E6
:10DE4000383F203F3F3F3F203F3F302E2D2B303F7C
:10DE5000E0E02020E0E0E02020E0E0E06020E0E002
:10DE6000E06020E0E0E03F3F203F3827383F203FA0
:10DE70003F3F3F203F3F3F3F203F3F3FE0E02020EC
:10DE8000E0E0E02020E0E0E06020E0E060A0A0A092
:10DE900060E03F3F203F3827383F203F3F3F3F2053
:10DEA0003F3F2F272B2D2E3FE0E02020E0E0E02019
:10DEB00020E0E0E06020E0E060A0A0A060E03F3F64
:10DEC000203F3827383F203F3F3F3F203F3F372FFD
:10DED0002D2D323FE0E02020E0E0E02020E0E0E0F7
:10DEE0006020E0E0E0E06020E0E03F3F203F3827B6
:10DEF000383F203F3F3F3F203F3F33343720373FBD
:10DF0000E0E02020E0E0E02020E0E0E06020E0E051
:10DF1000E020A0A0A0E03F3F203F3827383F203F2F
:10DF20003F3F3F203F3F342D2D2D333FE0E0202069
:10DF3000E0E0E02020E0E0E06020E0E060A0A0A0E1
:10DF400060E03F3F203F3827383F203F3F3F3F20A2
:10DF50003F3F302D2D2D333FE010101010D090108A
:10DF600090D010101050D050101010D0101010D0B1
:10DF700010101010E03F404040405F4043405F4081
:10DF80004040505F504040405F4142445F4040400D
:10DF9000403FE010109050505090109050505090D2
:10DFA00010D050505050105050D050501010E03FF2
:10DFB0004040495252524C404F5050504F405F42A7
:10DFC0004242404040405F404040403FE01010D05F
:10DFD000901010D010905050509010D05050509041
:10DFE00010D0101010D01010E03F40405F41464864
:10DFF0005F404F5050504F405F42424E51405F4152
:10E0000046415F40403FE01010D0101010D01090FB
:10E010005050509010D05050509010D050505090C0
:10E020001010E03F40405F4242425F405F42424248
:10E030005F405F42424E51405F5050504F40403F22
:10E04000E010101010D0101010D010101090509040
:10E05000101010D0101010D010101010E03F4040E1
:10E0600040405F4146415F40405C4342435C40402A
:10E070005845424558404040403FFFFF03030303DB
:10E080000B0B131323234343838343432323131390
:10E090000B0B03030303FFFFE0E07F7F6060606022
:10E0A0006868646462626161606061616262646444
:10E0B0006868606060607F7F07070000000000C044
:10E0C000F03C0EE3F1E30E3CF0C00000000000C0A5
:10E0D000F03C0F03000000217721000000030F3CFB
:10E0E000F0C000010303030303030303030303035B
:10E0F000030303030301000E11F1110E00000000E1
:10E100000000000000000000000000000000000E01
:10E1100011F1110E00000000000F10202020100E41
:10E1200010202020100E10202020100E1020202063
:10E13000100F00000000000E11F1110E0000000091
:10E140000000000000000000000000000000000EC1
:10E1500011F1110E0000000000070810101010103F
:10E1600010109254381038549210101010101010D3
:10E17000080700000000FE01010101010101010189
:10E18000010101010101010101010101010101017F
:10E190000101FE00F8F00F101010101010101010F8
:10E1A000101010101010101010101010101010106F
:10E1B00010100F000301FE01010101010101010125
:10E1C00001416171F9CDC14101010101010101016B
:10E1D0000101FE00F8F00F101010101010101010B8
:10E1E0001010101613111010101010101010101025
:10E1F00010100F00030100000000808000000000EC
:10E20000000000132424190000000000303000003A
:10E2100000000000004F00000007000700147F14FA
:10E220007F14242A7F2A12462610C8C43649552254
:10E23000500005070000001C2241000041221C0084
:10E2400014083E081408083E08080050300000106A
:10E2500010101010000080000040201008047C8A7C
:10E2600092A27C008CFE80008CC2A29ACC44829246
:10E270009A6C3038A6FEA05E9A8A8A727C9292923C
:10E28000640602F21E066C9292926C4C9292927C00
:10E29000000044000000563600000814224100141B
:10E2A00014141414004122140802015109063249C1
:10E2B00079413EE03C263CE0FE9292926C7C828268
:10E2C000824EFE8282827CFE92929282FE12121214
:10E2D000027C8292D2F4FE101010FE0082FE8200B8
:10E2E0004080827E02FE1038C682FE80808080FEE2
:10E2F0000E700EFEFE0638C0FE7C8282827CFE22FC
:10E3000022221C3E4151215EFE1232F28C4C92922E
:10E3100092640E82FE820E7E8080807E0E70C070BF
:10E320000E3EC03EC03E82EE38EE820E10E0100E71
:10E330008EE2BA8EE2000000000000000000000043
:10E3400000000000000000000000000000000000CD
:10E3500000000000000000000000000000000000BD
:10E3600000000000000000C0C00000800804021986
:10E370001800000000000000000000000000000085
:10E38000000000000000000000000000000000008D
:10E39000000000000000000000000000000000007D
:10E3A000000000000000000000000000000000006D
:10E3B0000000000000000000000000000202020255
:10E3C000000000000000000010000000000000003D
:10E3D000000000000080404040800F1112140F0028
:10E3E00080C0000000111F100080404040801018C5
:10E3F0001412198040404080081012120D00008055
:10E40000C0000605141F14C0404040400B131111FA
:10E410000E80404040800F1212120C404040C0C09D
:10E4200000001E030080404040800D1212120D803B
:10E4300040404080091212120F00008000000000CE
:10E4400008000000000000000000000000000000C4
:10E4500000000000000000000000000000000000BC
:10E4600000000000000000000000000000000000AC
:10E47000000000000000000000000000000000009C
:10E4800000E08000101F04071C20E02020C0101FA7
:10E4900011110EC0202020600F1010100820E02065
:10E4A00020C0101F10100F20E020A060101F1113BB
:10E4B00018C0404040401F020202008040202060FF
:10E4C000070810120E20E00000E0101F01011F20BD
:10E4D00020E0202010101F1010002020E02030200D
:10E4E000201F0020E0208060101F11061820E0206F
:10E4F0000000101F101010E0E000E0E01F011E01FE
:10E500001F20E08020E0101F11061F804040408047
:10E510000F1010100F40C0404080101F120201C0A9
:10E52000202020C00F1414382F20E02020C0101FFE
:10E5300011031CC020202040091113120E6020E09E
:10E54000206000101F100020E00000E0000F1010FD
:10E550000FC0000000C0010E100E01C000C000C0BE
:10E56000031E011E0320E000E020101C031C1020ED
:10E57000E000E02000101F1000602020E020101CB0
:10E580001310180000000000000000000000000050
:10E590000000000000000000000000F80000000083
:10E5A00000000000003330000000000000100C06E6
:10E5B000100C060000000000000000000000000039
:10E5C00040C07840C07840000000043F04043F048D
:10E5D00004000000007088FC0830000000000018F3
:10E5E00020FF211E00000000F008F000E0180000ED
:10E5F000000000211C031E211E00000000F00888FE
:10E600007000000000001E212324192721100000A3
:10E6100010160E00000000000000000000000000C6
:10E6200000000000000000E01804020000000000EC
:10E63000000718204000000000020418E00000005D
:10E64000000000402018070000000000404080F05B
:10E650008040400000000202010F010202000000A1
:10E66000000000F00000000000000101011F010196
:10E67000010000000000000000000000000080B069
:10E68000700000000000000000000000000000001A
:10E690000000000101010101010100000000000073
:10E6A000000000000000003030000000000000000A
:10E6B00000000000806018040000006018060100DF
:10E6C0000000000000E010080810E0000000000F4B
:10E6D000102020100F000000001010F800000000B3
:10E6E00000000020203F20200000000000700808EB
:10E6F000088870000000003028242221300000002B
:10E7000000300888884830000000001820202011C0
:10E710000E0000000000C02010F8000000000007FC
:10E720000424243F2400000000F80888880808001A
:10E7300000000019212020110E00000000E01088C8
:10E74000881800000000000F112020110E000000AA
:10E7500000380808C838080000000000003F00002A
:10E760000000000000708808088870000000001C8D
:10E77000222121221C00000000E010080810E00007
:10E7800000000000312222110F000000000000C034
:10E79000C000000000000000003030000000000059
:10E7A0000000008000000000000000008060000009
:10E7B000000000000080C060301808000000010365
:10E7C000060C18302000000040404040404040000F
:10E7D00000000404040404040400000000081830CD
:10E7E00060C080000000002030180C06030100000B
:10E7F000007048080808F0000000000000303601F2
:10E8000000000000C030C828E810E0000000071831
:10E81000272423140B0000000000C038E000000093
:10E820000000203C230202273820000008F88888D6
:10E83000887000000000203F202020110E00000002
:10E84000C0300808080838000000071820202010F1
:10E850000800000008F808080810E0000000203F49
:10E86000202020100F00000008F88888E808100019
:10E870000000203F202023201800000008F888888E
:10E88000E80810000000203F200003000000000006
:10E89000C030080808380000000007182020221E99
:10E8A0000200000008F808000008F8080000203FF7
:10E8B000210101213F200000000808F8080800009D
:10E8C00000000020203F2020000000000000080879
:10E8D000F80808000000C08080807F000000000071
:10E8E00008F888C0281808000000203F20012638BA
:10E8F0002000000008F80800000000000000203F91
:10E90000202020203000000008F8F800F8F8080067
:10E910000000203F003F003F2000000008F830C00A
:10E920000008F8080000203F200007183F00000002
:10E93000E01008080810E00000000F102020201050
:10E940000F00000008F808080808F0000000203F49
:10E950002101010100000000E01008080810E0009B
:10E9600000000F18242438504F00000008F8888851
:10E97000888870000000203F2000030C3020000039
:10E980000070880808083800000000382021212283
:10E990001C000000180808F8080818000000000013
:10E9A000203F20000000000008F808000008F808D8
:10E9B0000000001F202020201F0000000878880091
:10E9C00000C838080000000007380E0100000000F1
:10E9D000F80800F80008F8000000033C0700073CB6
:10E9E00003000000081868808068180800002030C4
:10E9F0002C03032C302000000838C800C838080059
:10EA000000000000203F2000000000E0FC3E060364
:10EA1000030303063EF8E00000FFFF0000000000D3
:10EA2000000000FFFF0000073F7C60C0C0C0C06066
:10EA30007C1F0700002020203038FFFF000000006E
:10EA40000000000000000000FFFF000000000000C8
:10EA5000000000000000FFFF000000000000007048
:10EA60007C0E0703030303070EFCF8000000000000
:10EA70000080C0E0703C1E0F030000F0FCCEC7C158
:10EA8000C0C0C0C0C0C0C0000000383E06030303C1
:10EA90000306FEF8000000000000000C0C0C0E1B2A
:10EAA00033F0C000000E3E70E0C0C0C0C060703FD8
:10EAB0000F00000000000080E0781EFFFF00000053
:10EAC0000000E0781E07010000FFFF0000000000CA
:10EAD00003030303030303FFFF030300000080FF9E
:10EAE0003F03030303030303000000000F0F0603AB
:10EAF000030303070EFCF000000E3E78E0C0C0C028
:10EB0000C060783F070000C0F83C0E07030303060F
:10EB10000E18000000FFFF1C0603030303070EFC92
:10EB2000F00000071F7C60C0C0C0C060783F0F00CD
:10EB30000003030303030383E33B1F0700000000FC
:10EB40000000C0F83E07000000000000000000F8D0
:10EB5000FF0700000000000000000000F8FE0E03A8
:10EB600003030306FEF8000000C0F13B1F0C0C0C71
:10EB70000C1F3BF1C000000F3F70E0C0C0C0C0E000
:10EB8000703F0F0000F0FC1E0603030303063EF86F
:10EB9000E000000F3F70E0C0C0C0C06038FFFF0061
:10EBA0000000187860C0C0C0C0603C1F030000AB0C
:10EBB00006FFAB07FFAB0AFFAB03FFAB04FFAB11D4
:10EBC000FFAB12FFABF9FFABFAFF00009281000030
:10EBD0000C7B0000E0740000046F00008C690000F2
:10EBE0005A6400006E5F0000D25A000068560000B0
:10EBF000445200005C4E0000A64A0000224700007C
:10EC0000D0430000A6400000AE3D0000D43A000012
:10EC10002C3800009835000036330000E830000042
:10EC2000B82E0000A62C0000B22A0000D228000056
:10EC30001027000062250000C823000042220000C7
:10EC4000D0200000681F00001E1E0000D41C000021
:10EC5000A81B0000861A00006E1900006A18000048
:10EC6000661700007616000090150000B41400002E
:10EC7000E21300001A1300005C120000A81100004B
:10EC8000FE10000054100000B40F00001E0F000022
:10EC9000880E0000FC0D00007A0D0000F80C00004A
:10ECA000800C0000080C00009A0B00002C0B0000E8
:10ECB000C80A0000640A0000000A0000A60900005B
:10ECC00056090000FC080000AC08000066080000BF
:10ECD00016080000D00700008A0700004E07000059
:10ECE00008070000CC060000900600005E06000049
:10ECF00022060000F0050000BE0500009605000099
:10ED000064050000320500000A050000E20400006E
:10ED1000BA04000092040000740400004C040000D7
:10ED20002E04000006040000E8030000CA030000EF
:10ED3000AC0300008E0300007A0300005C030000B7
:10ED40003E0300002A03000016030000F802000042
:10ED5000E4020000D0020000BC020000A802000093
:10ED600094020000800200006C02000058020000C3
:10ED70004E0200003A020000260200001C020000C1
:10ED800008020000FE010000F4010000E0010000A4
:10ED9000D6010000CC010000B8010000AE01000067
:10EDA000A40100009A01000090010000860100000B
:10EDB000540100007DDD5FDDE4CA9BE27DDD5FDDA7
:10EDC000E4CA9BE22C8145EC14EF0CE9570174E98D
:10EDD000570174E90F4BCADFF01338E48926FCDED3
:10EDE0008926FCDEB4A62ADC2C8145ECA65C77EBF8
:10EDF0002038A9EAA65C77EB570174E9E96EDEEBEF
:10EE00006F93ACEC570174E9570174E96F93ACEC64
:10EE10006F93ACEC9FB71DF30F4BCADFF01338E4D0
:10EE2000956F98E06AEF69E3763806E5FC5CD4E517
:10EE3000956F98E001000000020000000200000051
:10EE4000040000000000000020000000000010008E
:10EE50002000100074EE00000000002028030000D5
:10EE6000CCC9000060EF000028030020C00B0000A8
:10EE70004CCA0000114580510116231BB73280197E
:10EE8000104B102708014D12FE1314F01328DC1349
:10EE90003CC81350B41364A013788C138C7813A05F
:10EEA0006413B45013C83C13DC281BF01426192A31
:10EEB0002827FE14F0FE28DCFE3CC8FE50B4FE6499
:10EEC000A0FE788CFE8C78FEA064FEB450FEC83C98
:10EED000FEDC28FEF014FEFE2C0926551902092836
:10EEE0005512F01314DC1328C8133CB41350A013AC
:10EEF000648C137878138C6413A05013B43C13C83B
:10EF0000281BDC1423195112FE1825F0FE14DCFE18
:10EF100028C8FE3CB4FE50A0FE648CFE7878FE8CBF
:10EF200064FEA050FEB43CFEC828FEDC14FEF029AE
:10EF3000411378031B208C048113F4071B20A010BD
:10EF40008BA005141AA01479208A090C0111AA01BA
:10EF50000CB90101255A0604012509245301E100D9
:04000005000000C136
:00000001FF
